:020000040800F2
:10000000F8A0002045010008FD030008FF030008D8
:1000100001040008030400080504000800000000B3
:1000200000000000000000000000000007040008BD
:1000300009040008000000000B0400080D0400087B
:100040005F0100085F0100085F0100085F01000810
:100050005F0100085F0100085F0100085F01000800
:100060005F0100085F0100085F0100085F010008F0
:100070005F0100085F0100085F0100085F010008E0
:100080005F0100085F0100085F0100085F010008D0
:100090005F0100085F0100085F0100085F010008C0
:1000A0005F0100085F0100085F0100085F010008B0
:1000B0005F0100085F0100085F0100085F010008A0
:1000C0005F0100085F0100085F0100085F01000890
:1000D0005F0100085F0100085F0100085F01000880
:1000E0005F0100085F0100085F0100085F01000870
:1000F0005F0100085F0100085F0100085F01000860
:100100005F0100085F0100085F0100085F0100084F
:100110005F0100085F0100085F0100085F0100083F
:100120005F0100085F0100085F0100085F0100082F
:10013000DFF80CD005F092FB00480047E101000811
:10014000F8A000200648804706480047FEE7FEE783
:10015000FEE7FEE7FEE7FEE7FEE7FEE7FEE7FEE777
:10016000353D00083101000824A005F089FBFBE7BC
:1001700030B58FB001210804CDE9001000240294AD
:1001800002250491CDE907504FF4E010099068462C
:1001900002F04BFB08B18C210DE00F20CDE90A05E0
:1001A0004FF48060CDE90C4002210AA80E9402F0C1
:1001B000F0FC18B1992116A0FFF7D6FF02F0B1FDAF
:1001C0004FF47A71B0FBF1F003F017FD042003F057
:1001D0008CFD00221146501E03F0CDFC0FB030BD47
:1001E00002F01EFAFFF7C4FF00F01AF800F09CF8C6
:1001F00000F040F803F0F4FDFEE700005F45727286
:100200006F725F48616E646C65720D0A00000000D9
:100210002E2E2F5372632F6D61696E2E63000000C6
:10022000124810B5816986B041F00401816180698E
:100230000F4C00F00400049000221621204602F02A
:1002400057FF16200090012001900220039069467C
:10025000204602F0F9FD00210820CDE900010291BD
:100260006946204602F0F0FD06B010BD00100240C5
:1002700000080140254810B5234901604FF4827100
:10028000416000218160C1604FF400720161C0E9EA
:1002900005122822C0E90721416281620A21C16258
:1002A00001F0FEF9002805D0BDE81040272118A074
:1002B000FFF75ABF10BD00B50068134985B08842EA
:1002C00012D11748816941F4805181618069694682
:1002D00000F480500490A0200090022001900320A0
:1002E0000390104802F0B0FD05B000BD006806495B
:1002F000884208D10A48816921F480518161A02196
:10030000084802F080BE70470030014044000020E1
:100310002E2E2F5372632F7370692E63000000001E
:1003200000100240000801402D4810B52B49016023
:100330004FF4E1314160002181600C22C160C0E9CD
:1003400004128161C16101F0A4FA002805D0BDE862
:100350001040242123A0FFF707BF10BD10B500688F
:100360001E4986B088421DD12248816941F48041EE
:1003700081618069204C00F4804004904FF400704B
:10038000009002200190032003906946204602F06D
:100390005BFD00212015CDE9000102916946204650
:1003A00002F052FD06B010BD00680C49884209D128
:1003B0001048816921F4804181614FF4C0610E4889
:1003C00002F021BE704713B54FF6FF730122694654
:1003D000034801F088FB00981CBD00000038014074
:1003E0009C0000202E2E2F5372632F757361727440
:1003F0002E63000000100240000801407047FEE735
:10040000FEE7FEE7FEE770477047704710B502F061
:1004100025F9BDE8104003F075BC00001D4808B583
:10042000816941F001018161806900F00100009063
:10043000032003F093FB002211466FF00B0003F042
:100440009AFB002211466FF00A0003F094FB002291
:1004500011466FF0090003F08EFB00221146501F79
:1004600003F089FB00221146101F03F084FB0022D9
:100470001146901E03F07FFB00221146501E03F030
:100480007AFB0548416821F0E06141F0007141606C
:1004900008BD00000010024000000140704770B528
:1004A000040005D00025A56294F8510010B106E0C3
:1004B000012070BD84F850502046FFF7FCFE02205A
:1004C00084F851002068016821F040010160D4E9FE
:1004D00001010843D4E90312114308436169084349
:1004E000218B01F400710843E1690843216A084344
:1004F000A16A084321680860A069042101EA10404C
:10050000616A0843216848602068C16921F400617C
:10051000C1616565012084F85100002070BD7047FD
:1005200010B5040011D0022084F851002068016841
:1005300021F0400101602046FFF7D8FE00206065F1
:1005400084F8510084F8500010BD012010BD2DE941
:10055000F0411D4617460E460446DDF8188035E08A
:10056000681C33D02DB102F07FF8A0EB0800A84240
:100570002CD32068416821F0E00141606068B0F54B
:10058000827F0BD1A068B0F5004F02D0B0F5806F2C
:1005900004D12068016821F040010160A06AB0F533
:1005A000005F0AD1206801684DF6FF7211400160BA
:1005B0002068016841F400510160012084F8510075
:1005C000002084F850000320BDE8F0812068806896
:1005D00036EA000004D00020B842C1D10020F3E781
:1005E0000120F9E72DE9F84F044690F85000002665
:1005F000994617460D4601280DD04FF0010B84F89F
:1006000050B002F031F8804694F85100B24601280B
:1006100004D0022694E00220BDE8F88F002D7BD0A4
:10062000002F79D0032084F85100C4F854A025632A
:10063000A786E786C4F838A0A4F83CA0A4F83EA09A
:10064000C4F844A0C4F840A0A068B0F5004F04D19D
:100650002068016841F48041016020680168490612
:1006600003D4016841F040010160E068B0F5006F1B
:10067000606804D030B3E08E012823D03EE010B192
:10068000E08E01281AD135F8021B206805E02068A9
:100690008168890706D535F8021BC160E08E401ECF
:1006A000E0860BE0B9F1000F34D0B9F1FF3F05D07F
:1006B00001F0DAFFA0EB080149452BD2E08E0028BB
:1006C000E5D11EE0216815F8010B087306E02068EB
:1006D0008168890706D515F8011B0173E08E401E5D
:1006E000E0860BE0B9F1000F14D0B9F1FF3F05D05F
:1006F00001F0BAFFA0EB080149450BD2E08E0028BB
:10070000E5D14B46012202212046CDF80080FFF7BB
:100710001EFF10B1032613E011E042464946204671
:1007200000F0A2FF18B101262020606508E0A06853
:1007300018B92068C16880680090606D00B101261A
:1007400084F851B084F850A0304665E72DE9F84FA1
:10075000044690F8500000260A9F9A4693460D469C
:100760004FF0010801280ED0012084F8500001F05C
:100770007BFF814694F85100616801280BD0B1F5E8
:10078000827F06D101E0022046E7A16809B904286A
:1007900001D00226BEE055B1BBF1000F07D0BAF17F
:1007A000000F04D094F85100012802D004E0012683
:1007B000B0E0052084F8510000206065C4F838B02E
:1007C000A4F83EA0A4F83CA02563A4F836A0A4F8A1
:1007D00034A02064606420680168490603D401687D
:1007E00041F040010160E068B0F5006F606804D03E
:1007F000F0B3E08E01283CD06BE010B1E08E012810
:100800002FD1216835F8020BC860E08E401EE086CB
:1008100027E000BFB8F1000F0DD0E08E58B120687E
:100820008168890707D535F8021BC160E08E401E3C
:10083000E0864FF00008E08F58B120688168C90752
:1008400007D0C0682BF8020BE08F401EE0874FF006
:100850000108781C05D001F007FFA0EB0900B842A1
:1008600046D2E08E0028D5D1E08F0028D2D136E0E4
:10087000FFE7216815F8010B0873E08E401EE08643
:1008800027E000BFB8F1000F0DD0E08E58B120680E
:100890008168890707D515F8011B0173E08E401E9A
:1008A000E0864FF00008E08F58B120688168C907E2
:1008B00007D0C0680BF8010BE08F401EE0874FF0B7
:1008C0000108781C05D001F0CFFEA0EB0900B8426A
:1008D0000ED2E08E0028D5D1E08F0028D2D13B4641
:1008E000012202212046CDF80090FFF730FE08B12A
:1008F00003260FE04A463946204600F0B5FE18B1FF
:1009000001262020606505E0A06818B92068C1684C
:1009100080680090012084F85100002084F8500085
:10092000304679E62DE9F84F04464068002698469F
:1009300017460D464FF00409B0F5827F01D1A0683B
:1009400090B194F85000012818D04FF0010B84F8B2
:1009500050B001F089FE009094F851004FF0000A69
:1009600001280DD002267EE084F8519013460A46F5
:100970002046CDF80080FFF7E9FE4DE602204BE669
:10098000002D6FD0002F6DD084F85190C4F854A082
:10099000A563A787E787C4F830A0A4F834A0A4F81B
:1009A00036A0C4F840A0C4F844A0A0684FF40047A3
:1009B000B84204D12068016821F4804101602068B8
:1009C0000168490603D4016841F040010160E06814
:1009D000B8B133E020688168C90706D0007B05F80C
:1009E000010BE08F401EE0870BE0B8F1000F23D031
:1009F000B8F1FF3F05D001F037FE0099411A41459B
:100A00001AD2E08F0028E5D11BE020688168C90771
:100A100006D0C06825F8020BE08F401EE0870DE08D
:100A2000B8F1000F08D0B8F1FF3F07D001F01CFE6D
:100A30000099411A414501D3032614E0E08F0028B4
:100A4000E3D16068B0F5827F0AD1A068B84202D0D5
:100A5000B0F5806F04D12068016821F04001016089
:100A6000606D00B1012684F851B084F850A0304682
:100A7000D2E57047704738B50446FE4845F6C05188
:100A80000068B0FBF1F064214843009001F0ECFDF8
:100A90000246206800994B1E009304D2616D41F01C
:100AA0002001616502E081688907F3D5416821F082
:100AB000A00141606421204600F0D6FD18B1606DB0
:100AC00040F020006065A06818B92068C16880689F
:100AD0000090012084F85100606D0028204602D06B
:100AE000FFF7C8FF38BDFFF7C4FF38BD016B4A1CD4
:100AF0000263026809781173C18E491EC186C18ED6
:100B0000002900D1B7E77047016B02680988D160FE
:100B1000016B891C0163C18E491EC186C18E0029EB
:100B200000D1A8E7704730B590F850300024012B71
:100B30000BD0012380F85030002341B13AB190F836
:100B40005150012D05D002242DE0022030BD01249A
:100B500029E0032580F85150436501638286C286EF
:100B600083638387C3870364C16809B1C24900E016
:100B7000C24941648168B1F5004F04D101680A6837
:100B800042F480420A608168002901684A680ED0F8
:100B900042F0A0024A6001680A68520603D40A685B
:100BA00042F040020A6080F85030204630BD42F0EA
:100BB0008002EFE7704708B501684A6822F06002DA
:100BC0004A604168B1F5827F0BD18168B1F5004F71
:100BD00002D0B1F5806F04D101680A6822F04002AA
:100BE0000A60816819B90168CA68896800910121A1
:100BF00080F85110416D11B1FFF73CFF08BDFFF7C0
:100C0000D9FF08BD01680B7B816B4A1C82630B70A6
:100C1000C18F491EC187C18F002900D1CBE7704722
:100C20000168C968826B1180816B891C8163C18FE7
:100C3000491EC187C18F002900D1BCE770477047AA
:100C400038B504468B4845F6C0510068B0FBF1F05A
:100C500064214843009001F007FD02462068416886
:100C600021F0200141600098411E009104D2606D86
:100C700040F02000606503E0206880688007F2D5BE
:100C80006421204600F0F0FC18B1606D40F02000B7
:100C90006065A06818B92068C16880680090616DBF
:100CA000012029B184F851002046FFF7E3FE38BD4A
:100CB00094F8511084F851000429204602D0FFF71F
:100CC000BEFF38BDFFF776FF38BD016B4A1C0263DB
:100CD000026809781173C18E491EC186C18E002930
:100CE00008D101684A6822F080024A60C18F002959
:100CF00000D1A5E7704701680B7B816B4A1C8263BA
:100D00000B70C18F491EC187C18F002908D10168AE
:100D10004A6822F060024A60C18E002900D18FE744
:100D20007047016B02680988D160016B891C0163FF
:100D3000C18E491EC186C18E002908D101684A684A
:100D400022F080024A60C18F002900D178E7704705
:100D50000168C968826B1180816B891C8163C18FB6
:100D6000491EC187C18F002908D101684A6822F055
:100D700040024A60C18E002900D161E77047F0B59A
:100D800090F850500024012D0CD0012580F85050CF
:100D900090F8515000264768012D0BD0B7F5827F9F
:100DA00006D101E00220F0BD87680FB9042D01D003
:100DB00002242AE031B12AB123B190F85150012D1B
:100DC00002D004E0012420E0052580F8515046655A
:100DD00001638386C38682638387C387C16819B131
:100DE00027490164274902E02749016427494164F2
:100DF00001684A6842F0E0024A6001680A685206E7
:100E000003D40A6842F040020A6080F8506020462D
:100E1000F0BDF0B400248568134604261DB942686D
:100E2000B2F5827F0DD090F85020012A0ED0012219
:100E300080F8502090F851700022012F09D0022430
:100E400041E080F85160F0BC0A4698E70220F0BC0F
:100E5000704771B16BB180F85160426581638387DF
:100E6000C38702638286C2864264C168A1B1084911
:100E700013E00FE00C000020090B0008ED0A000849
:100E8000510D0008230D0008F70C0008CB0C0008DA
:100E9000210C0008012416E0FE490164B5F5004F5D
:100EA00004D101680B6823F480430B6001684B6830
:100EB00043F060034B6001680B685B0603D40B686A
:100EC00043F040030B6080F850202046BFE710B588
:100ED000406A01684A6822F003024A60416D41F0AD
:100EE00010014165012180F85110FFF7C3FD10BDCD
:100EF00038B50546446A01F0B7FB02462868006829
:100F000080061ED42068416821F0020141606421FE
:100F1000204600F0A9FB18B1606D40F0200060652C
:100F2000A068002118B92068C26880680090E18636
:100F3000012084F85100606D18B12046FFF79AFD3A
:100F400038BD2046FFF795FD38BD704710B5406AA3
:100F5000FFF7FBFF10BD70B5044690F85000002667
:100F6000012809D0012084F8500094F85100002590
:100F7000012803D002263FE0022070BD89B182B172
:100F8000032084F8510065652163A286E286A5638B
:100F900065642564A587E587A068B0F5004F02D099
:100FA00006E0012628E02068016841F480410160E4
:100FB000A16CB948C862A16CB8488862A16CB848F5
:100FC0000863A06C4563E38E2268216B0C32A06C31
:100FD00002F077F920680168490603D4016841F0FE
:100FE000400101602068416841F0200141602068B3
:100FF000416841F00201416084F85050304670BDB4
:1010000010B50146406A0968096889061ED401685E
:101010004A6822F003024A604168B1F5827F0BD131
:101020008168B1F5004F02D0B1F5806F04D101683D
:101030000A6822F040020A600021C187012180F87D
:101040005110416D11B1FFF715FD10BDFFF7B2FD55
:1010500010BD704710B5406AFFF7FBFF10BD70B5BB
:101060000546446A01F000FB0246286800688006D5
:1010700019D46421204600F0F7FA18B1606D40F0F1
:10108000200060652068416821F003014160002074
:10109000E086E087012084F85100606D18B1204699
:1010A000FFF7E8FC70BD2046FFF7C9FD70BD704733
:1010B00010B5406AFFF7FBFF10BD2DE9F041044673
:1010C00090F85000002601280CD0012084F8500030
:1010D00094F851000025676801280CD0B7F5827F8D
:1010E00007D102E00220BDE8F081A7680FB904280B
:1010F00001D0022651E031B12AB123B194F8510058
:10110000012802D004E0012647E0052084F85100C0
:1011100065652163A386E386A263A387E3872564CD
:10112000656494F8510004283BD0E16C5D48C862C6
:101130005D48E16C8862E16C59480863E06C456386
:10114000E38F2168A26B0C31E06C02F0BAF82068E2
:10115000416841F001014160A06CC562A06C8562EC
:10116000A06C0563A06C4563E38E2268216B0C3292
:10117000A06C02F0A6F820680168490603D4016853
:1011800041F0400101602068416841F02001416068
:101190002068416841F00201416084F850503046B7
:1011A000A1E7E16C4148C8624148C2E72DE9F0413E
:1011B000044600268068042318B96568B5F5827F67
:1011C0000DD094F85050012D11D0012584F85050C5
:1011D00094F851700025012F0BD0022644E084F8CA
:1011E00051302046BDE8F04113460A4665E702202B
:1011F00079E771B16AB184F851306565A163A2875E
:10120000E28725646564A586E586B0F5004F02D0C7
:1012100006E0012628E02068016821F48041016091
:10122000E16C2248C862E16C21488862E16C1C488C
:101230000863E06C4563E38F2168A26B0C31E06CBE
:1012400002F03FF820680168490603D4016841F0C4
:10125000400101602068416841F020014160206840
:10126000416841F00101416084F8505030463AE74E
:1012700008B5002100910F4945F6C0520968B1FB3D
:10128000F2F16422514300910168009A531E0093C9
:1012900017D211E0050C00084D0F0008F10E0008F0
:1012A000CF0E0008B11000085F10000855100008AC
:1012B000011000080C000020426D42F0200242653F
:1012C00002E08A689207E0D50A6822F040020A60CC
:1012D00001684A6822F0E0024A600068C068009035
:1012E00008BD01684A6822F0E0024A6000680168AF
:1012F00021F040010160704738B50446E24845F6E8
:10130000C0510068B0FBF1F06421484300902068B0
:101310004168090601D5DD4961644168490601D586
:10132000DB492164416821F0200141602068416867
:101330004FF00005890702D44068C00727D0A06C91
:10134000A8B14563A06C01F0F4FF2068416821F06A
:10135000020141600098411E009104D2606D40F08E
:101360002000606503E0206880688007F2D5E06CAB
:1013700068B14563E06C01F0DCFF2068016821F092
:10138000400101602068416821F001014160E5876A
:10139000E58665652068C16880680090012084F852
:1013A0005100002038BD704708B5406A01680A68DE
:1013B00022F040020A60C26C002151630268536847
:1013C00023F001035360826C12B1526B002A0BD1DF
:1013D000C187C18641650168CA6889680091012199
:1013E00080F85110FFF7DFFF08BDA74908B509686D
:1013F00045F6C052B1FBF2F1642251430091406ABC
:101400000021826C51630268536823F00203536029
:10141000009A531E009304D2426D42F020024265AE
:1014200003E0026892689207F2D5C26C12B1526B67
:10143000002A07D1C187C1864165012180F851107A
:10144000FFF7B1FF08BDF8B504460068416809061A
:1014500001D58E4961644168490601D58C492164F2
:10146000416821F0200141600126A06C002538B1BF
:1014700021684968890702D58649416300E04563D0
:10148000E06C38B121684968C90702D082494163DC
:1014900000E0456320684168890715D54068C007AA
:1014A00012D0A06C30B101F05CFF10B1A06C4563AC
:1014B00000E00026E06C38B101F053FF18B1E06C99
:1014C0000126456300E0002620684068800708D5B3
:1014D000A06C30B101F045FF10B1A06C456300E095
:1014E000002620684068C00706D0E06C20B101F0FB
:1014F00038FF78B1E06C456366B1E587E5866565E0
:101500002068C16880680090012084F8510020465E
:10151000FFF749FF0020F8BD90F8501001290CD0CA
:10152000012180F8501001684A6822F003024A60E5
:10153000002180F85010084670470220704790F84C
:10154000501001290CD0012180F8501001684A6820
:1015500042F003024A60002180F8501008467047AC
:101560000220704710B50446806C08B101F0E1FE1E
:10157000E06C08B101F0DDFE2068416821F0030154
:101580004160012084F85100002010BD10B5406A70
:101590000021C187C186FFF76DFA10BD38B504463A
:1015A0000068426881684B0605D4CB0703D0530618
:1015B00001D5216C04E08B0707D5130605D5616CB6
:1015C00001B02046BDE83040084711F0600F3FD021
:1015D00093063DD54B060AD594F85130032B34D0F1
:1015E000636D43F004036365C368836800938906F1
:1015F00009D5616D41F00101616581680091016863
:1016000021F040010160606D002821D02068416810
:1016100021F0E0014160012084F85100900718D0CA
:101620002068416821F0030141601C4DE06C18B155
:101630004563E06C01F095FEA06C002808D045637E
:10164000A06CBDE8384001F08CBEC1688068009095
:1016500038BD2046FFF70EFA38BD90F851007047AC
:10166000406D70470120704738B50B460092044624
:1016700000228021FEF76BFF002804D0606D40F04F
:1016800020006065032038BD0C000020E312000834
:1016900071120008EB130008A91300088D1500084B
:1016A00070B5040005D00025A56294F8510010B172
:1016B00004E0012070BD2046FEF7FDFD022084F805
:1016C00051002068016821F040010160D4E9010166
:1016D0000843D4E903121143084361690843218B8D
:1016E00001F400710843E1690843216A0843A16AD3
:1016F000084321680860A069042101EA1040616A7A
:101700000843216848602168E06A08612068C1696F
:1017100021F40061C1616565012084F85100002059
:1017200070BD00002DE9F041044600680169E268DF
:1017300021F44051114301612169A06808436169A6
:1017400008432168CA6841F20C639A430243CA60A5
:1017500020684169A26921F4407111434161FC494B
:1017600020686425322688423CD101F0E7FA00EB7C
:10177000C00101EB001061688900B0FBF1F701F0D6
:10178000DDFA00EBC00101EB00106168B046890092
:10179000B0FBF1F0B0FBF5F06FF01801484307EB38
:1017A000800106EB0110B0FBF5F000F0F00601F04F
:1017B000C5FA00EBC00101EB001061688900B0FBC5
:1017C000F1F0B0FBF5F006EB001601F0B7FA00EB14
:1017D000C00101EB001061688900B0FBF1F701F076
:1017E000ADFA3BE001F0A0FA00EBC00101EB001004
:1017F00061688900B0FBF1F701F096FA00EBC001D7
:1018000001EB00106168B0468900B0FBF1F0B0FB5D
:10181000F5F06FF01801484307EB800106EB01106B
:10182000B0FBF5F000F0F00601F07EFA00EBC0012D
:1018300001EB001061688900B0FBF1F0B0FBF5F03E
:1018400006EB001601F070FA00EBC00101EB00108E
:1018500061688900B0FBF1F701F066FA00EBC001A6
:1018600001EB001061688900B0FBF1F0B0FBF5F00E
:101870006FF01801484307EB800108EB0110B0FB43
:10188000F5F0216800F00F0030448860BDE8F08179
:10189000704770B5040004D094F83900002510B1E9
:1018A00006E0012070BD84F838502046FEF756FD52
:1018B000242084F839002068C16821F40051C160F7
:1018C0002046FFF72FFF2068016921F49041016154
:1018D0002068416921F02A0141612068C16841F412
:1018E0000051C160E563202084F8390084F83A0093
:1018F000002070BD70B5040004D094F839000025B4
:1019000010B106E0012070BD84F838502046FEF783
:1019100025FD242084F839002068C16821F4005195
:10192000C1602046FFF7FEFE2068016921F4904166
:1019300001612068416921F022014161206841690B
:1019400041F0080141612068C16841F40051C16063
:10195000E563202084F8390084F83A00002070BD47
:1019600070B50E46040004D094F83900002510B17B
:1019700006E0012070BD84F838502046FEF7EEFCEA
:10198000242084F839002068C16821F40051C16026
:101990002046FFF7C7FE2068016921F4006101615C
:1019A0002068416921F02A0141612068016941F400
:1019B000804101612068016921F02001314301610A
:1019C0002068C16841F40051C160E563202084F8BB
:1019D000390084F83A00002070BD2DE9F041164628
:1019E0000F46040004D094F83900002510B106E039
:1019F00001204BE784F838502046FEF7AFFC242046
:101A000084F839002068C16821F40051C160204683
:101A1000FFF788FE2068016921F490410161206888
:101A2000416921F02A0141612068016921F00F011B
:101A3000394301612068C16821F400613143C1600C
:101A40002068C16841F40051C160E563202084F83A
:101A5000390084F83A00002018E7704710B50400F8
:101A60000ED0242084F839002046FEF79DFC00208B
:101A7000E06384F8390084F83A0084F8380010BD37
:101A8000012010BD2DE9F041984617460E46044648
:101A9000069D1CE0681C1AD02DB100F0E5FDA0EBFE
:101AA0000800A84213D92068C16821F4D071C16030
:101AB0002068416921F001014161202084F839004A
:101AC00084F83A00002084F838000320DEE620681D
:101AD000006836EA000004D00020B842DAD00020C6
:101AE000D4E60120F9E72DE9F843044690F83900DF
:101AF0001F4616460D46202852D1A5B19EB194F836
:101B0000380001284CD0012084F838004FF000083C
:101B1000C4F83C80212084F8390000F0A5FDA6849B
:101B20008146E68428E00120BDE8F883E08C401E71
:101B3000E084A0684B46B0F5805F4FF000024FF0A4
:101B400080012046009705D0FFF79CFFF8B90FE011
:101B500000380140FFF796FFC8B928882168C0F314
:101B600008004860206908B16D1C05E0AD1C03E069
:101B7000216815F8010B4860E08C0028D6D14B464F
:101B80000022402120460097FFF77CFF08B1032088
:101B9000CAE7202084F8390084F838800020C3E7A1
:101BA0000220C1E72DE9F843044690F83A0099462F
:101BB00016460D4620284ED195B18EB194F83800C6
:101BC000012848D0012084F838000027E76322204C
:101BD00084F83A0000F048FDA6858046E68530E0AE
:101BE0000120A1E7E08D401EE085A0684346B0F5E6
:101BF000805F4FF000024FF020012046CDF80090AA
:101C000004D0FFF73FFF98B103208DE7FFF73AFFBD
:101C10000028F9D1206900282068406803D0C1B2AB
:101C200025F8011B0DE0C0F3080125F8021B08E0B0
:101C3000206900282068406801D000F07F0005F886
:101C4000010BE08D0028CDD1202084F83A0084F8E3
:101C50003870002068E7022066E790F83930202BC2
:101C600018D1A9B1A2B190F83830012B12D001627D
:101C70008284C2840021C163212280F8392080F847
:101C800038100068C16841F08001C16000207047D1
:101C9000012070470220704790F83A30202B22D163
:101CA000F9B1F2B190F83830012B1CD081628285F5
:101CB000C2850021C163222280F83A2080F83810C2
:101CC0000168CA6842F48072CA6001684A6942F0D9
:101CD00001024A610068C16841F02001C160002032
:101CE00070470120704702207047704770B5446A02
:101CF0002068406994F83910C0F3C01000252129EC
:101D000004D118B1E584204600F02EFC206840691B
:101D100094F83A10C0F38010222904D118B1E58557
:101D2000204600F013FCE06B40F01000E06320461A
:101D3000FFF7DBFF70BD704710B5406AFFF7FBFF90
:101D400010BD704710B50146406A096809688906E8
:101D50000CD40021C18401684A6922F080024A61E2
:101D60000068C16841F04001C16010BDFFF7E9FFA4
:101D700010BD70B5044690F83900202830D169B301
:101D800062B394F8380001282AD0012084F8380082
:101D90002162A284E2840025E563212084F83900D1
:101DA000236BFD489862236BFC48D862236BFC4888
:101DB0001863206B134645632668206B321D01F0C3
:101DC00080FA21686FF04000086084F8385020687D
:101DD000416941F080014161002070BD012070BD6A
:101DE000022070BD704710B5406AFFF7FBFF10BDC1
:101DF000704710B50146406A09680968890613D41E
:101E00000021C1850168CA6822F48072CA60016835
:101E10004A6922F001024A6101684A6922F04002DF
:101E20004A61202180F83A10FFF7E2FF10BDF8B5B3
:101E3000044690F83A0020283CD1C1B3BAB394F8D4
:101E40003800012836D0012084F83800A162A2852C
:101E50000025E563222084F83A00636BD14898623C
:101E6000636BD148D862636BCD481863606B1346CF
:101E700045630846666B216802463046091D01F03D
:101E800020FA206801684168009184F83850C168E0
:101E900041F48071C1602068416941F001014161F4
:101EA0002068416941F0400141610020F8BDFFE731
:101EB0000120FBE70220F9E790F8381001290BD048
:101EC000012180F8381001684A6990F83930C2F36E
:101ED000C012212B02D006E0022070471AB14A69D5
:101EE00022F080024A6101684A6990F83A30C2F3F0
:101EF0008012222B0ED16AB1CA6822F48072CA60A5
:101F000001684A6922F001024A6101684A6922F0C7
:101F100040024A61002180F838100846704708B531
:101F200090F83810012907D0012180F8381090F876
:101F30003910212902D006E0022008BD01684A6953
:101F400042F080024A6190F83A100022222911D111
:101F500001680B684B680093CB6843F48073CB60D7
:101F600001684B6943F001034B6101684B6943F021
:101F700040034B6180F83820002008BD10B50446AE
:101F80000068416994F83920C1F3C011212A0BD1AE
:101F900051B1416921F080014161206B08B101F02C
:101FA000C8F9204600F0E0FA2068416994F83A2028
:101FB000C1F38011222A0BD151B1416921F04001B6
:101FC0004161606B08B101F0B4F9204600F0BEFA3F
:101FD000002010BD70B504460068C16821F4F0719E
:101FE000C1602068416921F00101416120684169B7
:101FF0004FF00005090609D5416921F080014161D2
:10200000206B18B14563206B01F093F9206841699A
:10201000490609D5416921F040014161606B18B161
:102020004563606B01F085F9E584E585E563202073
:1020300084F83A0084F83900002070BD70B5044679
:102040000068C16821F0C001C160206841694FF09B
:102050000005090609D5416921F080014161206B25
:1020600018B14563206B01F064F9E584202084F801
:102070003900002070BD70B504460068C16821F4C5
:102080009071C1602068416921F0010141612068BF
:1020900041694FF00005490609D5416921F0400129
:1020A0004161606B18B14563606B01F042F9E585F1
:1020B000202084F83A00002070BD704710B5406AB7
:1020C0000021426B5163026B12B1526B002A09D19D
:1020D000C184C185C163202180F8391080F83A108D
:1020E000FFF7EBFF10BD10B5406A0021026B516392
:1020F000426B12B1526B002A09D1C184C185C16300
:10210000202180F8391080F83A10FFF7D6FF10BD73
:1021100070B5044600680126C16821F4F071C16001
:102120002068416921F001014161206B002538B12F
:1021300021684969090602D51C49416300E04563ED
:10214000606B38B121684969490602D51849416375
:1021500000E045632068416909060CD5416921F01A
:1021600080014161206B30B101F0FBF810B1206BB0
:10217000456300E000262068416949061AD5416997
:1021800021F040014161606BA0B101F0EAF8E8B1D3
:10219000606B45630FE00000451D0008391D000815
:1021A000ED1C0008F31D0008E71D0008E7200008EB
:1021B000BD20000856B1E584E585E563202084F85C
:1021C000390084F83A002046FFF777FF002070BD01
:1021D000704710B5406A0021C184202180F8391071
:1021E000FFF7F6FF10BD10B504460068C16821F086
:1021F000C001C160206841694FF020020B064FF01A
:1022000000010FD5436923F080034361206B48B17F
:10221000F2494163206B01F0A4F848B1206B416B97
:10222000884705E0E18484F839202046FFF7D0FF95
:10223000002010BD704710B5406A0021C1852021E3
:1022400080F83A10FFF7F6FF10BD10B5044600689D
:10225000C16821F49071C1602068416921F00101D9
:102260004161206841694FF020024B064FF00001A8
:102270000FD5436923F040034361606B48B1D849EF
:102280004163606B01F06DF848B1606B416B88474A
:1022900005E0E18584F83A202046FFF7CBFF0020D7
:1022A00010BD10B5406A0021C185C184FFF71DFD36
:1022B00010BD10B590F83A10222901D0022010BDAF
:1022C0008168B1F5805F11D00169002901681FD0D4
:1022D000496801F07F03816A4A1C82620B70C18DDC
:1022E000491E0904090CC18518D02BE00269816AD6
:1022F000002A0268526805D0D2B20A80816A491C5D
:102300008162ECE7C2F308020A80816A891CF7E760
:102310004A68816A4B1C83620A70E0E70168CA68F8
:1023200022F02002CA600168CA6822F48072CA6082
:1023300001684A6922F001024A61202180F83A10BE
:10234000FFF756FD002010BD70B502680446106806
:10235000D168536910F00F0F50D003F0010501F45C
:10236000907635435CD0C20705D0CA0503D5E26B31
:1023700042F00102E263420705D5DA0703D0E26BBF
:1023800042F00202E263820705D5DA0703D0E26B6E
:1023900042F00402E263020705D5DA0703D0E26BDC
:1023A00042F00802E263E26B002A32D0800604D5D4
:1023B000880602D52046FFF77CFF20684069E16B64
:1023C000C0F38010090700D420B3204600F0BEF807
:1023D00020684169490619D5416921F040014161F0
:1023E000606B98B17F494163606B00F0BAFF0028D1
:1023F0000FD0606B416BBDE87040084783060FD576
:102400008B060DD52046BDE8704052E72046FFF709
:102410006CFC70BD2046FFF768FC0020E06370BDD7
:10242000030606D50B0604D52046BDE8704000F033
:10243000A4B84006F3D54806F1D5D168204621F06E
:102440004001D160202184F83910FFF77AFC70BD7B
:1024500090F83810012910D0012100F8381F2421EC
:10246000417050F8381CCA6842F00102CA6020214D
:10247000417000210170084670470220704790F8B3
:102480003810012910D0012100F8381F2421417093
:1024900050F8381CCA6842F00202CA60202141701C
:1024A00000210170084670470220704790F83810EC
:1024B000012910D0012100F8381F2421417050F863
:1024C000381CCA6822F00202CA6020214170002133
:1024D0000170084670470220704790F838100129B3
:1024E00012D0012100F8381F2421417050F8381C07
:1024F000CA6822F00C0242F00802CA602021417032
:1025000000210170084670470220704790F838108B
:10251000012912D0012100F8381F2421417050F800
:10252000381CCA6822F00C0242F00402CA60202162
:10253000417000210170084670470220704710F872
:10254000391F407808437047C06B70470168CA68FC
:1025500022F49072CA6001684A6922F001024A615D
:10256000202180F83A1070470168CA6822F0C00242
:10257000CA60202180F83910704790F8391021295D
:1025800001D0022070478168B1F5805F016A0BD0ED
:102590004A1C0262026809785160C18C491E090414
:1025A000090CC1840ED017E009880268C1F3080144
:1025B000516001690029016A02D0491C0162ECE7FF
:1025C000891CFBE70168CA6822F08002CA600068C3
:1025D000C16841F04001C16000207047D32100086C
:1025E00037220008A3220008704770B5554D0446F5
:1025F0004FF47A712878B1FBF0F053490968B1FBC8
:10260000F0F001F0FAFA48B9102C07D20022214666
:10261000501E01F0B0FA00206C6070BD012070BD4A
:102620004A4810B5016841F010010160032001F033
:1026300095FA0020FFF7D9FFFDF7F0FE002010BD4E
:102640007047434810B54FF0FF31C160002202616E
:10265000C160C260FFF7F4FF002010BD39488168F7
:102660000278114481607047364880687047354869
:1026700040687047334A10B50146137800208B42FA
:1026800003D011705068FFF7B0FF10BD2D480078DF
:10269000704770B50446FFF7E7FF0546601C02D09F
:1026A000284800780444FFF7DFFF401BA042FAD31C
:1026B00070BD4FF0E020016921F002010161704717
:1026C0004FF0E020016941F00201016170472148AB
:1026D000704721480068000C70471F480068C0F32D
:1026E0000B0070471C48416841F001014160704790
:1026F0001948416821F0010141607047164841685E
:1027000041F00201416070471348416821F0020125
:10271000416070471048416841F0040141607047D2
:102720000D48416821F00401416070470B49096878
:1027300001600A49091D09684160084908310968B2
:1027400081607047000000200C0000200020024043
:102750000010024000020101002004E0E8F7FF1F22
:102760002DE9F041FFF780FFFD4C0546206840F061
:102770000100206005E000BFFFF776FF401B022844
:1027800043D820688007F7D5206820F0F80040F093
:1027900080002060FFF768FF00250646656041F273
:1027A000883704E0FFF760FF801BB8422DD86068CF
:1027B00010F00C0FF6D1EC49EA4808600020FFF752
:1027C00014FF10B10120BDE8F081FFF74DFF064670
:1027D000206820F08070206005E000BFFFF744FF14
:1027E000801B022811D820688001F7D46560FFF7AC
:1027F0003BFF0646206820F41020206007E000BF61
:10280000FFF732FF801B642801D90320DBE7206833
:102810008003F5D4206820F480202060606A40F0B6
:1028200080706062A5600020CDE72DE9F84F044676
:102830000078CB4DC00749D06868C0F381000128FB
:1028400007D06868C0F38100022809D16868C00316
:1028500006D52868800339D56068002870D035E037
:102860006068B0F5803F0BD010B1B0F5A02F11D04B
:10287000286820F480302860286820F4802002E056
:10288000286840F480302860606890B1FFF7ECFE63
:1028900006460AE0286840F480202860F0E700BF80
:1028A000FFF7E2FE801B642875D828688003F7D5FF
:1028B0000CE0FFF7D9FE064605E000BFFFF7D4FEA7
:1028C000801B6428F0D828688003F7D42078A74EAE
:1028D00080074FF001094FF000083BD5686810F001
:1028E0000C0F07D06868C0F38100022809D168681E
:1028F000C00306D42868800714D5206901281FD199
:1029000010E02069B0B1C6F80090FFF7ADFE0746B1
:1029100005E000BFFFF7A8FEC01B0228C4D8286846
:102920008007F7D52868616920F0F80040EAC10007
:1029300028600FE0C6F80080FFF796FE074606E025
:10294000E9E000BFFFF790FEC01B022823D82868EB
:102950008007F7D4207800072CD58548A169D9B124
:10296000C0F80090FFF780FE074604E0FFF77CFE0A
:10297000C01B02280FD8686A8007F7D57A484FF441
:10298000FA510068B0FBF1F0009000BF0098411EC2
:102990000091FAD20EE080E0C0F80080FFF764FEFC
:1029A000074604E0FFF760FEC01B022875D8686A7E
:1029B0008007F7D42078400760D5E8690027C00079
:1029C00008D4E86940F08050E861E869012700F028
:1029D0008050009067480168C90513D40168834698
:1029E00041F480710160FFF73FFE824606E000BFC0
:1029F000FFF73AFEA0EB0A0064284ED8DBF800008F
:102A0000C005F5D5E06801280AD008B1052813D023
:102A1000286A20F001002862286A20F0040002E001
:102A2000286A40F001002862E06841F2883B98B1D2
:102A3000FFF71AFE82460BE0286A40F00400286285
:102A4000EEE700BFFFF710FEA0EB0A0159455AD888
:102A5000286A8007F6D50CE0FFF706FE824605E0FF
:102A6000FFF702FEA0EB0A0159454CD8286A8007FF
:102A7000F6D41FB1E86920F08050E861E06988B3BE
:102A80006968C1F38101022945D00228C6F8608037
:102A900004D0FFF7E9FD044638E034E0FFF7E4FD39
:102AA000074604E0FFF7E0FDC01B02282BD828688A
:102AB0008001F7D4206AB0F5803F05D16868A1682D
:102AC00020F4003008436860D4E9080108436968CD
:102AD00021F4741108436860C6F86090FFF7C4FDE4
:102AE000044606E015E000BFFFF7BEFD001B02280C
:102AF00009D828688001F7D50BE000BFFFF7B4FDC7
:102B0000001B022802D90320BDE8F88F2868800145
:102B1000F4D40020F8E70120F6E717A185B00FC92B
:102B20008DE80F0018A00E4A0068049051680D4807
:102B300001F00C03042B10D0082B0ED1C1F38343FA
:102B4000C9031DF8030021D5516804AAC1F340410F
:102B5000515C044A5043B0FBF1F005B070470000EF
:102B60000010024000127A000C00002000004242D7
:102B70008004424200700040020304050607080971
:102B80000A0B0C0D0E0F101001020000A64948435D
:102B9000E3E72DE9F047DFF8948205460E46D8F8C2
:102BA000000000F00700B0420CD2D8F8001021F06D
:102BB00007013143C8F80010D8F8000000F0070002
:102BC000B04262D128789A4C800705D56068A96820
:102BD00020F0F000084360602878C00744D068689F
:102BE000012816D02168022816D0890700294CDA5E
:102BF000616821F0030101436160FFF735FD6968F9
:102C0000074641F2883001290ED00229814618D0AA
:102C100026E021688903E9E78901E7E7FFF724FD5A
:102C2000C11B494501D918E081466068C0F38100A5
:102C30000128F3D118E000BFFFF716FDC11B49457D
:102C40000BD86068C0F381000228F5D10CE000BF0A
:102C5000FFF70AFDC11B494502D90320BDE8F087F3
:102C6000606810F00C0FF3D1D8F80010404601F066
:102C70000701B1420BD9016821F00701314301601E
:102C8000006800F00700B04201D00120E6E7287894
:102C9000400705D56068E96820F4E060084360609B
:102CA0002878000706D56068296920F4605040EA5A
:102CB000C1006060FFF731FF61685E4AC1F3031134
:102CC000515CC8405C4908600020FFF78EFC002082
:102CD000C4E730B585B000200290022001900320A7
:102CE0000390534C4FF480700090A0690D4640F063
:102CF0000400A061A069694600F0040004904F48F8
:102D000000F0A2F8606820F0E0602843606005B041
:102D100030BD4B490120C864704749490020C86450
:102D20007047454800687047434841490068496812
:102D3000444AC1F30221515CC84070473E483C49B7
:102D4000006849683F4AC1F3C221515CC8407047DE
:102D500010B50F21016036490A6853034FF0000295
:102D600002D54FF4A02304E00B68DB0303D54FF436
:102D70008033436000E042604B6803F400338360BB
:102D80000B68DC074FF0010301D0036100E0026132
:102D90000C68C4F3C40444610C6A640702D50524BA
:102DA000C46005E00C6AE40701D0C36000E0C260C3
:102DB0004C6AE40701D0836100E082610A68D201B5
:102DC00002D50222C26100E0C3614A6802F4803287
:102DD0000262496801F47011416210BD0F22026065
:102DE000134A536803F003034360536803F0F0038E
:102DF0008360536803F4E063C36052684FF4E06398
:102E000003EAD20202610948006800F00700086086
:102E10007047704710B5064CA068000603D5FFF751
:102E2000F8FF8020A07210BD00093D000020024084
:102E300000100240345B00080C0000200008014034
:102E400000004242445B00082DE9F84FDFF8ECA295
:102E500000220AF1040B144601274FF00F090BF171
:102E6000040E00BF0B6807FA04F52B40AB4274D187
:102E7000DFF8CCC24E68A6EB0C0866452BD00DDC03
:102E8000032E34D005DC36B3012E19D0022E2FD1FB
:102E90001BE0112E16D0122E2AD119E0B8F5881F8A
:102EA00019D006DCB8F5803F15D0B8F5801F1FD1CA
:102EB00011E0B8F5001F0ED0B8F5041F18D10AE0D4
:102EC000CA6815E0CA68121D12E0CA6808320FE02D
:102ED000CA680C320CE08A682AB1012A4FF0080255
:102EE00003D0456104E0042202E0056100E0002215
:102EF000FF2B01D8064601E000F104064FEA8405E5
:102F000001D9A5F12005D6F800C009FA05F82CEA88
:102F1000080C02FA05F54CEA050CC6F800C04D682D
:102F2000ED006AD5874DAE6946F00106AE61AD6928
:102F300024F0030605F001050095834D06EB050C12
:102F4000DCF80850A6074FEA167809FA08F6B543E8
:102F50007E4EB04202D100261AE04EE07C4EB042D6
:102F600001D1012614E07B4EB04201D102260FE0D0
:102F7000794EB04201D103260AE0784EB04201D129
:102F8000042605E0764EB04201D1052600E0062673
:102F900006FA08F62E43CCF808604D68DAF80060AF
:102FA000ED03554601D51E4300E09E432E604D685B
:102FB000AD0305D5DBF800601E43CBF8006004E0EC
:102FC000DBF800509D43CBF800504D68DEF8006000
:102FD000ED02754601D51E4300E09E432E604D680C
:102FE000AD0205D5554D0C352E681E432E6004E00C
:102FF000524E0C3635689D433560641C102CFFF42E
:1030000031AFBDE8F88F2DE9F04300230F24DFF83E
:1030100038C163E001229A400A405ED0FF2A01D8FD
:10302000074601E000F104074FEA830601D9A6F143
:103030002006D7F8008004FA06F54FF0040928EAC4
:10304000050809FA06F948EA0908C7F80080C568C2
:1030500025EA0205C56023F003056544AF684FEA21
:1030600083764FEA167604FA06F909EA0708374F1D
:10307000B84201D1002719E0354FB84201D10127EC
:1030800014E0344FB84201D102270FE0324FB8426A
:1030900001D103270AE0314FB84201D1042705E0EE
:1030A0002F4FB84201D1052700E00627B74047451A
:1030B00013D1AF6827EA0907AF60204D2E68964309
:1030C0002E602D1D2E6896432E602D1D2E68964372
:1030D0002E602D1D2E6896432E605B1C31FA03F284
:1030E00098D1BDE8F0838068084000D00120704787
:1030F0000AB1016170470904FBE7C2684A40C26037
:10310000704708B541F48032009282618161009974
:103110008161816900918069C00301D5002008BDEB
:10312000012008BD7047054910B514310A680242F4
:1031300002D00860FFF7F6FF10BD00000004014058
:103140000000111000100240000001400008014082
:10315000000C014000100140001401400018014023
:10316000001C014030B560B1FA4A03681421934253
:1031700009D2F94A1A44B2FBF1F189000164F74916
:103180000AE0012030BDF34A52421A44B2FBF1F189
:1031900089000164EF490839C163022180F82110D8
:1031A0001A6843F6F0718A43F0E901142143D0E92B
:1031B00002452C4321430469214344692143846926
:1031C000214311431960002141628162C1620163A0
:1031D0004163012242770177084630BD10B5D0B176
:1031E00001680A6822F001020A6002680021116089
:1031F00002685160026891600268D160D54C026833
:103200001423A24209D2D44C2244B2FBF3F292001E
:103210000264D24A0AE0012010BDCE4C644222442E
:10322000B2FBF3F292000264CA4A083AC26390F811
:10323000403001229A40C36B5A60816380F82110AC
:1032400080F82010002010BD30B590F840500124C7
:10325000AC40C56B6C60046863604368102B036806
:1032600003D099600068C26030BD9A600068C16098
:1032700030BD70B5044690F82000002501280CD020
:10328000012084F8200094F821600020012E06D04F
:1032900084F820000225284670BD022070BD022659
:1032A00084F82160A0632068066826F001060660A5
:1032B0002046FFF7C9FF2068016841F00101016065
:1032C000E9E770B5044690F82000002501280CD0ED
:1032D000012084F8200094F821600020012E06D0FF
:1032E00084F820000225284670BD022070BD022609
:1032F00084F82160A0632068066826F00106066055
:103300002046FFF7A1FFE06A00282068016802D08C
:1033100041F00E0106E021F004010160206801681F
:1033200041F00A0101602068016841F0010101607B
:10333000D9E701680A6822F00E020A6001680A688B
:1033400022F001020A6090F84020C36B012101FACB
:1033500002F25A6080F82110002180F820100846FF
:1033600070472DE9F05F90F821100024022903D066
:1033700004218163012485E001680A6822F00E02BD
:103380000A6001680A6822F001020A60734E734FF6
:103390008036B215DFF8C4C1DFF8C091DFF8BCA1F8
:1033A000DFF8B8B1DFF8B4E101680837130115029E
:1033B0000CF11C0C09F130090AF1440A0BF1580B0D
:1033C0000EF16C0E4FF48018B14227D9B9420ED0DD
:1033D000614512D049451DD0514518D0594518D0E6
:1033E000714501D1424615E05A4EB14201D1012248
:1033F00010E0584E1436B14201D110220AE0554E69
:103400002836B14206D0534A3C32914201D11A4685
:1034100000E02A464F49091F0A602AE0B94213D04A
:10342000614517D0494522D051451DD059451DD081
:10343000714501D142461AE0B14202D14FF080728B
:1034400015E0444EB14201D1012210E0414E143644
:10345000B14201D110220AE03E4E2836B14206D0D8
:103460003C4A3C32914201D11A4600E02A463B498F
:103470004A60012180F82110002180F82010416B62
:1034800001B188472046BDE8F09F2DE9F74F04467B
:1034900090F8210082B0022805D00420A06300200B
:1034A00084F82000FDE020680168890603D54FF408
:1034B0008070A063F5E0294D284E03991C35303605
:1034C000DFF89880DFF89490DFF890A00029244975
:1034D0004FF4806B08F1440809F158090AF16C0AAD
:1034E00003D088423ED1042758E0884201D1022708
:1034F00054E0A84201D1202750E0B04203D100BFE0
:103500004FF400774AE0404503D100BF4FF4005725
:1035100044E0484503D100BF4FF400373EE050453A
:1035200002D14FF4001739E00D497831884201D1BA
:10353000870433E007498842D9D0064914318842CC
:10354000D9D0044928318842DAD002493C31884236
:10355000E2D1DBE708040240F8FFFDBF00000240B3
:1035600008000240A84201D1402717E0B04201D133
:103570005F4613E0404502D14FF480470EE04845D6
:1035800003D100BF4FF4802708E0504502D14FF42B
:10359000800703E0F649884204D1C704FFF764F8C6
:1035A000009082E0F34988429DD0F249143188426C
:1035B000DAD0F04928318842DAD0EE493C318842ED
:1035C000E0D1D9E7884228D9EA4908390A68E849A8
:1035D0007839884210D0A84210D0B04214D040456B
:1035E00015D0484516D0504503D100BF4FF4000018
:1035F00027E0E049884234D1082022E0802020E002
:10360000DC492831884231D14FF4006019E04FF491
:10361000004016E04FF4002013E0D54A803A1268CB
:10362000D34B783B9842E7D0A842E7D0B042EBD0EA
:103630004045ECD04845EDD05045D7D08842D8D150
:103640001806024217D094F84010E26B012000FAED
:1036500001F1516054F8381F41F0010144F8181984
:103660001CE0C44914318842CAD1C7E7C1493C3182
:103670008842CFD1CBE70498401C16D0049830B1D3
:10368000FEF7F2FF0099411A049881420DD954F8CF
:10369000380F40F0200044F8180901206070002025
:1036A0002070012005B0BDE8F08FB1492068884244
:1036B00002D9B04A083A01E0AD4A803A12683A426B
:1036C00080D0AC4A0399121F0029A94911D0884221
:1036D00075D9A749783988427BD0A8427FD0B042BB
:1036E00070D040456FD048456ED050456ED1C8046B
:1036F00086E088422CD99E49783988420ED0A8426B
:1037000012D0B04216D040451BD048451CD0504581
:1037100001D188041AE09749884201D1022015E0BE
:1037200094491431884201D120200FE09149283179
:10373000884202D14FF4007008E08E493C31884243
:1037400002D14FF4005001E04FF40030106032E03D
:10375000874A783A904213D0A84217D0B0421BD083
:10376000404520D0484521D0504501D190041FE06C
:10377000884202D14FF000701AE07E49884201D1A0
:10378000022015E07B491431884201D120200FE04E
:1037900078492831884202D14FF4007008E0754919
:1037A0003C31884202D14FF4005001E04FF4003028
:1037B0006F4980394860012084F8210054E021E0FD
:1037C00007E00CE011E016E018E0FFE769498842E5
:1037D00001D1042014E067491431884201D140200E
:1037E0000EE064492831884201D1584608E0614919
:1037F0003C31884202D14FF4804001E04FF48020F8
:10380000106031E05A4A783A904213D0A84217D05B
:10381000B0421BD040451FD0484520D0504501D173
:10382000D0041EE0884202D14FF0806019E0514977
:10383000884201D1042014E04E491431884201D15C
:1038400040200EE04B492831884201D1584608E01B
:1038500048493C31884202D14FF4804001E04FF4A6
:103860008020434980394860002084F8200019E70F
:103870002DE9F05FC16B0A6801680B68046C4FF0BA
:10388000040808FA04F83C4D3C4E3D4FDFF8F4C004
:10389000DFF8F490DFF8F4A0DFF8D8B0DFF8F0E05C
:1038A00018EA020F76D05FEA437873D50A68920669
:1038B00003D40A6822F004020A604FF48062DFF841
:1038C000B080016813011402414524D9A9420DD0EA
:1038D000B1420FD0B9421AD0614515D0494515D033
:1038E000514501D1120312E0594501D104220EE0E5
:1038F000714501D140220AE0254D1435A94206D078
:10390000234A2832914201D11A4600E02246194941
:10391000091F0A6029E0A94213D0B14215D0B9426B
:1039200020D061451BD049451BD0514502D14FF4F1
:10393000800217E0414502D14FF0806212E0594504
:1039400001D104220EE0714501D140220AE0104D60
:103950001435A94206D00E4A2832914201D11A46A6
:1039600000E02246044908394A60C16A80E011E05B
:103970008000024008040240080002401C0002408F
:103980003000024044000240580002406C000240F7
:103990001C0402404FF0020808FA04F818EA020F6B
:1039A0006BD05FEA837868D50A68920606D40A6805
:1039B00022F00A020A60012180F821104FF40072FF
:1039C000DFF89081016813011402414523D9A9420F
:1039D0000DD0B1420FD0B94219D0614514D049453C
:1039E00014D0514501D1120311E0594501D10222F1
:1039F0000DE0714501D1202209E0574DA94206D0C2
:103A0000554A1432914201D11A4600E022465249E9
:103A10002C390A6028E0A94213D0B14215D0B9422E
:103A20001FD061451AD049451AD0514502D14FF4F3
:103A3000001216E0414502D14FF0007211E05945E5
:103A400001D102220DE0714501D1202209E0424D51
:103A5000A94206D0404A1432914201D11A4600E0F0
:103A600022463C4980394A60002180F82010816A52
:103A700000291BD0BDE8F05F08470825A540154286
:103A800014D01A0712D50A6822F00E020A6090F8C4
:103A90004020C36B012101FA02F25A60816380F871
:103AA0002110002180F82010016BE1E7EBE410B554
:103AB00090F820400023012C07D0012480F82040FA
:103AC00090F82140012C02D008E0022010BD59B12D
:103AD00001290BD002290BD003290BD0012300218F
:103AE00080F82010184610BD8262F8E7C262F6E73F
:103AF0000263F4E74263F2E710B590F82020002358
:103B0000012A08D0012280F8202090F821400022CC
:103B1000012C02D014E0022010BD052910D2DFE8EC
:103B200001F0030507090B0082620AE0C26208E0A7
:103B3000026306E0426304E08262C2620263F9E764
:103B4000012380F82020184610BD90F8210070470E
:103B5000806B70478000024030040240734900F0DF
:103B6000070208684FF6FF03184040EA0220704A37
:103B7000104308607047F0B46C4B1B680C46C3F3ED
:103B80000223C3F10705042D00D90425191D0729B7
:103B900001D2002300E0DB1E012606FA05F1491ED2
:103BA000214099409E40761E16403143F0BC00F003
:103BB000ADB800F01F02012191404009800000F1E2
:103BC000E020C0F80011704700F01F020121914071
:103BD0004009800000F1E020C0F880117047BFF379
:103BE0004F8F52480168524A01F4E061121D11439F
:103BF0000160BFF34F8F00BFFDE710B5401EB0F16D
:103C0000807F01D3012010BD4FF0E02460610F21BF
:103C1000601700F07BF80020A061072020610020E1
:103C200010BD42480068C0F30220704770B50028FC
:103C300006DA00F00F0000F1E02090F8140D03E028
:103C400000F1E02090F80004040901F00700C0F141
:103C50000705042D00D90425011D072901D20020E4
:103C600000E0C01E012124FA00F601FA05F56D1EE0
:103C70002E408140491E21401660196070BD00F041
:103C80001F02012191404009800000F1E020C0F8AE
:103C9000001270474109890001F1E021D1F80012BA
:103CA00000F01F0201209040014201D00120704726
:103CB0000020704700F01F02012191404009800060
:103CC00000F1E020C0F8801270474109890001F13D
:103CD000E021D1F8001300F01F02012090400142C2
:103CE00001D001207047002070474FF0E0210428E8
:103CF000086903D020F004000861704740F0040018
:103D0000FAE7704710B5FFF7FCFF10BD0907090E71
:103D1000002806DA00F00F0000F1E02080F8141D02
:103D2000704700F1E02080F8001470470CED00E0CF
:103D30000000FA052248016841F001010160416874
:103D4000204A1140416001681F4A1140016001682A
:103D500021F480210160416821F4FE0141604FF4AB
:103D60001F0181601949C00308607047144910B5EC
:103D70004868174A10F00C03164803D0042B01D0F2
:103D8000082B09D002604968134AC1F30311515C42
:103D90000268CA40026010BD4A684B6802F47012A3
:103DA0004FF0020413F4803F04EB924202D04B68C0
:103DB0009B0301D5094B00E0054B5A43E2E70000A5
:103DC000001002400000FFF8FFFFF6FE08ED00E0E3
:103DD00000127A000C000020345B000800093D004E
:103DE0002DE9FE4FF3A001F04BFD00F016FE4FF061
:103DF000FF3910B14846BDE8FE8FF4A001F040FD48
:103E000000F0D6FA00F074FB4FF4FA742046FEF787
:103E100040FC43F6982001F057FE07007ED0F2A048
:103E200001F02EFDFF2600234FF496724FF4C87167
:103E30003846009600F01CFEF0A001F021FD384647
:103E400000F032FEFF2000F0EDFEF24801F081FCB0
:103E5000384600F07CFBA2462046FEF71AFCEEA096
:103E600001F00EFD384600F01FFEFF2000F0DAFEE4
:103E7000F0A001F005FD01252B46002250210A206B
:103E8000009500F000FF022300225A210A2000952D
:103E900000F0F9FE0323002264210A20009500F0BF
:103EA000F2FE00244622CDE9004578231146142075
:103EB000029400F042FF4621CDE900457823142208
:103EC0000846029400F039FF4622CDE900457823E8
:103ED00011461420029400F093FFCDE900457823A9
:103EE000822246215020029500F08AFFCDE900543D
:103EF000002314225F212D2001F0D1F80095FF232B
:103F000014225F216920019501F0C9F85F237D2209
:103F1000CDE9004519465520029500E0D6E000F0B5
:103F20000CFF6922CDE9004573234B211046029511
:103F300000F003FFCDE90046C44BC5A200210A20D2
:103F400001F00BFACDE90064C44BC5A214210A208C
:103F500001F003FADFF814B3CDE90046BF4B5A462F
:103F600021210A2001F022FBCDE90064B74BC04AB1
:103F700032210A2001F01AFBCDE90046BD4BBEA25A
:103F80000021822001F023FACDE90064BD4BBEA2DE
:103F90001421822001F01BFABEA001F071FC38460A
:103FA00000F0D5FA4FF4FA60FEF773FBBD4801F05C
:103FB00067FC00F04EFABCA001F062FC384601F04C
:103FC0005BFD47F2305001F07FFD5FEA00087DD0D5
:103FD00000234FF496724FF4C871009600F048FD2C
:103FE000042000F07AFDFF2000F01CFE01230022D7
:103FF00050210A20009500F046FE022300225A219B
:104000000A20009500F03FFE0323002264210A20CD
:10401000009500F038FE4622CDE900457823114690
:104020001420029400F089FE4621CDE90045782352
:1040300014220846029400F080FE4622CDE9004595
:10404000782311461420029400F0DAFECDE90045F1
:104050007823822246215020029500F0D1FECDE93E
:104060000054002314225F212D2001F018F8009540
:10407000FF2314225F216920019501F010F85F23CE
:10408000CDE900457D2219465520029500F055FEE8
:104090006922CDE9004573234B211046029500F0BB
:1040A0004CFECDE90046694B69A200210A2001F0CF
:1040B00054F9CDE90064694B69A214210A2001F08A
:1040C0004CF92121654B5A460A2000E06EE0CDE90B
:1040D000004601F06BFACDE900645C4B644A322182
:1040E0000A2001F063FA0326CDE90064614B77A250
:1040F00000218C2001F06BF90227CDE900755D4BA2
:1041000072A228218C2001F062F9CDE90057594BA9
:104110006EA250218C2001F05AF9CDE90046554B92
:104120006AA278218C2001F052F9CDE90064554B48
:1041300055A20021DC2001F04AF9CDE90075514B70
:1041400051A22821DC2001F042F9CDE900574D4B66
:104150004DA25021DC2001F03AF9CDE90046494B4F
:1041600049A27821DC2001F032F9404600F0A5FA9E
:104170005046FEF78EFAFF2000F054FD554800F03F
:104180009CFA4FF4FA60FEF784FA00F0B1F952A0FD
:1041900001F076FB00F023FB404601F06DFC52A0DD
:1041A00001F06EFB00F04CFC002024E65BA001F067
:1041B00067FB1FE64550445F34494E325F746573B8
:1041C000742044656D6F0D0A00000000652D50617C
:1041D00070657220496E697420616E6420436C655D
:1041E00061722E2E2E0D0A005061696E745F4E654D
:1041F00077496D6167650D0A0000000073686F778D
:1042000020696D61676520666F72206172726179E5
:104210000D0A00004C5B000853656C656374496DC2
:104220006167653A426C61636B496D6167650D0A50
:104230000000000044726177696E673A426C616306
:104240006B496D6167650D0A0000000024000020C5
:104250007761766573686172650000001000002068
:1042600068656C6C6F20776F726C640015CD5B07AE
:10427000B168DE3A1800002020C4E3BAC36162636B
:10428000000000002C000020CEA2D1A9B5E7D7D3B2
:10429000000000004550445F446973706C61790D03
:1042A0000A0000003C35010873686F77204772618F
:1042B000792D2D2D2D2D2D2D2D2D2D2D2D2D2D2DE2
:1042C0002D2D2D2D2D2D2D2D2D0D0A00C4E3BAC31E
:1042D00061626300E4950008476F746F20536C655A
:1042E00065702E2E2E0D0A00636C6F736520355697
:1042F0002C204D6F64756C6520656E74657273203B
:104300003020706F77657220636F6E73756D707497
:10431000696F6E202E2E2E0D0A0000004661696C1A
:10432000656420746F206170706C7920666F7220F4
:10433000626C61636B206D656D6F72792E2E2E0D30
:104340000A00000010B5FF4C012202212046FEF7B2
:10435000CFFEC820FEF79DF9002202212046FEF77D
:10436000C7FEC820FEF795F9012202212046FEF77C
:10437000BFFEBDE81040C820FEF78BB910B5F2A013
:1043800001F07EFA712000F038FAEE4C05E0712061
:1043900000F033FA6420FEF77CF908212046FEF78E
:1043A000A2FE0028F3D0BDE81040EDA001F068BAED
:1043B00010B5FFF7C7FF012000F01FFA032000F03F
:1043C00033FA002000F030FA2B2000F02DFA2B20D9
:1043D00000F02AFA062000F010FA172000F024FA64
:1043E000172000F021FA172000F01EFA042000F038
:1043F00004FAFFF7C3FF002000F0FFF9BF2000F030
:1044000013FA0D2000F010FA302000F0F6F93C20ED
:1044100000F00AFA612000F0F0F9012000F004FA3F
:10442000902000F001FA012000F0FEF92C2000F0AD
:10443000FBF9822000F0E1F9282000F0F5F9502086
:1044400000F0DBF9972000F0EFF9BDE8104000F034
:104450000CBA10B5FFF776FF012000F0CEF903206B
:1044600000F0E2F9002000F0DFF92B2000F0DCF989
:104470002B2000F0D9F9132000F0D6F9062000F027
:10448000BCF9172000F0D0F9172000F0CDF9172063
:1044900000F0CAF9042000F0B0F9FFF76FFF002028
:1044A00000F0ABF93F2000F0BFF9302000F0A5F993
:1044B0003C2000F0B9F9612000F09FF9012000F0E4
:1044C000B3F9902000F0B0F9012000F0ADF92C20F4
:1044D00000F0AAF9822000F090F9122000F0A4F96F
:1044E000502000F08AF9BDE81040972000F09CB9F8
:1044F0002DE9F04132264FF49675102000F07DF939
:1045000000270024FF2000F08FF9641CA4B2B442FD
:10451000F8D37F1CBFB2AF42F3D3132000F06DF984
:1045200000270024FF2000F07FF9641CA4B2B442ED
:10453000F8D37F1CBFB2AF42F3D3122000F05DF975
:104540000A20FEF7A6F8BDE8F04100F084B92DE995
:10455000F047814632274FF49678132000F04DF94A
:104560000024002504FB07F609EB0500305C00F091
:104570005BF96D1CADB2BD42F6D3641CA4B24445D8
:10458000EFD3BDE8F04700F066B92DE9F05F88464B
:104590001E464FF0320A410702D020F007000830D3
:1045A00084B2500702D022F00702083295B25020A0
:1045B00000F023F9F72000F037F96420FEF769F8DE
:1045C000822000F01AF9082000F02EF9502000F0A7
:1045D00014F9472000F028F900F089F9912000F043
:1045E0000CF9902000F009F9200A00F01DF9E0B262
:1045F00000F01AF9280A00F017F9681EC0B200F09E
:1046000013F94FEA182000F00FF908F0FF0000F04E
:104610000BF9300A00F008F9701EC0B200F004F97E
:10462000282000F001F9102000F0E7F80027281BEF
:10463000A6EB0809C11700EB517614E00A9908EBC4
:10464000070000FB0A1B002508E000BF05EBD401B2
:104650001BF8010000F0E8F86D1CADB2B5EBE60FF9
:10466000F4DB7F1CBFB2B945E8DC132000F0C5F8CD
:10467000002716E00A9908EB070000FB0A1B00253B
:104680000AE000BF05EBD4011BF80100C043C0B233
:1046900000F0CAF86D1CADB2B5EBE60FF2DB7F1C83
:1046A000BFB2B945E6DC122000F0A7F80A20FDF7FA
:1046B000F0FFBDE8F05F00F0CEB82DE9F041044610
:1046C000102000F09AF8002643F6982500200146B5
:1046D00001EB4602A35C002203F0C007C02F02D00A
:1046E0001FB1802F01D140F001009B0640061F0E34
:1046F000000E07F0C003C02B02D01BB1802B01D1EC
:1047000040F00100012901D1012A01D04006000E2C
:10471000BB061B0E521C022ADED3491C0229D7D32A
:1047200000F082F8761CAE42D0D3132000F065F87A
:10473000002600204FEA000101EB4602A35C0022A4
:104740001EE000000008014044656275673A20657C
:104750002D506170657220627573790D0A0000003A
:1047600044656275673A20652D50617065722062FC
:104770007573792072656C656173650D0A000000C0
:1047800003F0C007C02F02D01FB1802F01D040F02E
:1047900001009B0640061F0E000E07F0C003C02B51
:1047A00002D01BB1802B01D040F00100012901D1C2
:1047B000012A01D04006000EBB061B0E521C022A25
:1047C000BED3491C0229B7D300F02EF8761CAE42A6
:1047D000AFD300F0C9F8BDE8F04100F03CB810B527
:1047E000022000F00AF8FFF7C9FD072000F005F8E5
:1047F000BDE81040A52000F017B870B57E4C054606
:10480000002204212046FEF773FC002210212046DE
:10481000FEF76EFC284600F0F7F82046BDE8704031
:1048200001221021FEF764BC70B5734C05460122CD
:1048300004212046FEF75CFC002210212046FEF7F2
:1048400057FC284600F0E0F82046BDE87040012201
:104850001021FEF74DBC10B51220FFF7CEFF6420EB
:10486000FDF717FFBDE8104088E570B52020FFF781
:10487000C4FF624D0024285DFFF7D6FF641CA4B27C
:104880002C2CF8D32120FFF7B8FF5C4D00242C35E9
:10489000285DFFF7C9FF641CA4B22A2CF8D322209C
:1048A000FFF7ABFF554D00245635285DFFF7BCFFE1
:1048B000641CA4B22A2CF8D32320FFF79EFF4F4D8F
:1048C00000248035285DFFF7AFFF641CA4B22A2CBA
:1048D000F8D32420FFF791FF484D0024AA35285D26
:1048E000FFF7A2FF641CA4B22A2CF8D370BD70B5E8
:1048F0002020FFF782FF414D0024D435285DFFF7CB
:1049000093FF641C2C2CF9D32120FFF776FF3C4D3C
:104910000024285DFFF788FF641C2A2CF9D322208D
:10492000FFF76BFF364D00242A35285DFFF77CFF2B
:10493000641C2A2CF9D32320FFF75FFF304D00249D
:104940005435285DFFF770FF641C2A2CF9D324200E
:10495000FFF753FF2A4D00247E35285DFFF764FFE3
:10496000641C2A2CF9D370BD70B52020FFF745FFD9
:10497000234D0024A835285DFFF756FF641C2A2C20
:10498000F9D32120FFF739FF1D4D0024D235285DD2
:10499000FFF74AFF641C2A2CF9D32220FFF72DFFD2
:1049A000174E0024FC36305DFFF73EFF641C2A2CB6
:1049B000F9D32320FFF721FF124E0024305DFFF7CB
:1049C00033FF641C2A2CF9D32420FFF716FF0D4E69
:1049D00000242A36305DFFF727FF641C2A2CF9D308
:1049E0002520FFF70AFF0024285DFFF71DFF641C48
:1049F0002A2CF9D370BD000000080140140B0108F7
:104A0000140C01083A0D010801B54FF47A73012224
:104A100069461548FBF7E6FD08BD10B5134C0022AA
:104A200004212046FEF764FB002210212046FEF7F9
:104A30005FFB012202212046FEF75AFB002010BD39
:104A400010B50A4C002204212046FEF751FB00223B
:104A500010212046FEF74CFB20460022BDE8104006
:104A60000221FEF745BB0000440000200008014081
:104A700070B5F94C049E0025206021816281A681D9
:104A80000220E0824E074FEAD10000D0401C608235
:104A9000A282E381258223B1B42B02D0A280E180DF
:104AA00070BDA180E28070BDEB490860704710B511
:104AB00004000BD05A2C09D0B42C07D0B4F5877F52
:104AC00004D0BDE81040E5A000F0DABE0146ECA03D
:104AD00000F0D6FEE048C48110BDDF4910B50A8958
:104AE000022809D004280FD0EDA000F0C9FEBDE8CF
:104AF0001040F6A000F0C4BEC882D7485207008913
:104B0000C00806E0488210BDC882D34892070089D9
:104B10008008002AF6D0401CF4E710B504000AD043
:104B2000012C08D0022C06D0032C04D0BDE8104084
:104B3000EF4800F0A5BE6008C00701D0EDA200E07C
:104B4000EEA2E00701D0EBA100E0ECA1EDA000F0A7
:104B500097FEC148048210BDF0B4BF4CA3888342C5
:104B600034D3E3888B4231D32346E7891E895D899C
:104B7000CFB15A2F1AD0B42F1CD0B7F5877F3FD1B1
:104B80000B46281A401E80B2218AD9B1012916D0BD
:104B9000022904D0032933D1F11A491E8BB2281AF5
:104BA000401E80B20EE003460846EDE7711A491E2A
:104BB0008BB2E9E7301A401E83B2681AE2E7F11AB5
:104BC000491E8BB29E4201D3854203D2F0BCD6A0CF
:104BD00000F056BEA049E58A4C8A0968022D11D022
:104BE000042D0DD1444304EB930490079B075B0F06
:104BF000C025DD400A5D000EAA43D8401043085589
:104C0000F0BC7047444304EBD3048020002A0D5DC0
:104C100003F0070220FA02F001D02843EFE78543B2
:104C20000D55EDE730B500218B4AC3B20DE00020F1
:104C300006E000BF01FB04041568401C80B22B5540
:104C4000548A8442F6D8491C89B2908A8842EED8A8
:104C500030BD2DE9F0471F4616460D468046DDF86B
:104C600020900CE0444606E04A4629462046FFF7DD
:104C700073FF641CA4B2B442F6D36D1CADB2BD4246
:104C8000F0D3BDE8F0872DE9F05F734D9346814680
:104C9000AA880A981C4688464A4502D3EA884245B3
:104CA0000ED2ABA000F0ECFDAA884946B8A000F0F7
:104CB000E7FDEA884146BDE8F05FBEA000F0E0BD38
:104CC000012801D0002635E00025681E00EB4407CE
:104CD00019E009EB05000026A0EB040A0FE000BF75
:104CE000BAF1000F0DD408EB0600001B09D481B205
:104CF0001FFA8AF05A46FFF72FFF761C36B2B742EA
:104D0000EEDC6D1C2DB2AF42E3DCBDE8F09F002568
:104D100009EB06077F1E09E008EB0500401E81B283
:104D2000B8B25A46FFF718FF6D1C2DB2A542F3DB4F
:104D3000761C36B2A642EADBE7E72DE9FE4F1D46B8
:104D4000454B16469A88824206D3DB888B4203D3B2
:104D5000B24201D3AB4204D2BDE8FE4F9FA000F0A7
:104D60008FBD83468A46321A00D5821B91466A1A45
:104D7000002A00DD4A1B90464FF0FF32B34501D2B6
:104D8000012000E010460290AA4500D2012209EB62
:104D90000804002701927F1C0E98FFB2012805D15C
:104DA0000320B7FBF0F100FB1170E8B10120DDE951
:104DB0000C23009051465846FFF765FFB8EB440FAF
:104DC00007DCB3451AD0029944440BEB01001FFAEB
:104DD00080FBB9EB440FDEDBAA450FD001984C44B1
:104DE00050441FFA80FAD6E701200090FF22514676
:104DF00058460D9BFFF747FF0027DFE7BDE8FE8F12
:104E00002DE9FE4F8246144891460C46DDE90D52CD
:104E100081880C9E1F46514506D3C088A04203D30B
:104E2000494501D3B84204D2BDE8FE4F7BA000F053
:104E300027BD0020804662B908E1CDE90065234620
:104E40004A4619465046CDF80880FFF776FF641CA5
:104E5000A4B2BC42F1D3D1E7DC0000204465627506
:104E6000673A20726F74617465203D20302C2039C0
:104E7000302C203138302C203237300D0A00000021
:104E800044656275673A2053657420696D61676592
:104E900020526F746174652025640D0A00000000C3
:104EA00044656275673A20536574205363616C658D
:104EB00020496E70757420706172616D65746572E1
:104EC000206572726F720D0A000000004465627501
:104ED000673A205363616C65204F6E6C792073755F
:104EE00070706F72743A20322034200D0A00000076
:104EF0009C3501086D6972726F7200006E6F6E658D
:104F00000000000044656275673A206D6972726F37
:104F10007220696D61676520783A25732C20793A93
:104F200025730D0A0000000044656275673A20454C
:104F30007863656564696E6720646973706C617914
:104F400020626F756E6461726965730D0A000000FE
:104F500044656275673A205061696E745F4472619E
:104F600077506F696E7420496E7075742065786330
:104F70006565647320746865206E6F726D616C2066
:104F8000646973706C61792072616E67650D0A00E7
:104F900058706F696E74203D202564202C2050616C
:104FA000696E742E5769647468203D202564202042
:104FB0000D0A200059706F696E74203D2025642011
:104FC0002C205061696E742E486569676874203DB5
:104FD00020256420200D0A20000000004465627531
:104FE000673A205061696E745F447261774C696EF4
:104FF0006520496E707574206578636565647320FB
:10500000746865206E6F726D616C20646973706C7A
:1050100061792072616E67650D0A000044656275F2
:10502000673A20496E7075742065786365656473AE
:1050300020746865206E6F726D616C206469737096
:105040006C61792072616E67650D0A00CDE90065BB
:1050500023464A4619465046CDF80880FFF76DFEB4
:10506000CDE9006552463B4621461046CDF8088002
:10507000FFF763FECDE900654A46234639461046F0
:10508000CDF80880FFF759FECDE900653B46524652
:1050900019464846CDF80880FFF74FFEAEE62DE9E9
:1050A000FF4F8046F74885B00F46848813994445E2
:1050B00002D3C088B84205D809B0F348BDE8F04F24
:1050C00000F0DEBB03200024A0EB420015B20FFA73
:1050D00080FA012978D0E7E0264660E04FF0010928
:1050E00008EB040007EB060B02901FFA8BF1CDF8DA
:1050F000009080B24B46089AFFF7C5FDA8EB04006C
:1051000004901FFA8BF1CDF8009080B20123089A29
:10511000FFF7B9FD3819CDE9009081B2A8EB060B75
:105120001FFA8BF00123089AFFF7ADFD381B03909F
:1051300081B2CDF800901FFA8BF00123089AFFF797
:10514000A2FD0498A7EB060B1FFA8BF1CDF8009097
:1051500080B20123089AFFF796FD02981FFA8BF19F
:10516000CDF8009080B20123089AFFF78CFD0398D8
:1051700008EB060B81B2CDF800901FFA8BF00123EB
:10518000089AFFF780FD0198CDF8009081B21FFAD0
:105190008BF00123089AFFF776FD761C36B2AE42FB
:1051A0009CDDBAF1000F05DA0AEB8400801D0FFACE
:1051B00080FA07E0611B0AEB81000A306D1E0FFACE
:1051C00080FA2DB2641C24B2AC4285DD09B0BDE882
:1051D000F08F08EB0400012607EB050902901FFA87
:1051E00089F1009680B2129B089AFFF74CFDA8EB5C
:1051F000040003901FFA89F1009680B2129B089A6E
:10520000FFF741FD3819CDE9006081B2A8EB05092F
:105210001FFA89F0129B089AFFF735FDA7EB040BE4
:105220001FFA8BF11FFA89F00096129B089AFFF77C
:105230002AFD0398A7EB05091FFA89F1009680B2B1
:10524000129B089AFFF71FFD02981FFA89F100963A
:1052500080B2129B089AFFF716FD08EB05091FFAAA
:105260008BF11FFA89F00096129B089AFFF70BFD4D
:105270000198009681B21FFA89F0129B089AFFF7F5
:1052800002FDBAF1000F05DA0AEB8400801D0FFA67
:1052900080FA07E0611B0AEB81000A306D1E0FFAED
:1052A00080FA2DB2641C24B2AC4292DD8EE72DE967
:1052B000F05F814673481E46DDF82CB0838888462F
:1052C0004B4502D3C188414504D2BDE8F05F6FA0D1
:1052D00000F0D6BAB088410700D0012101EBD00020
:1052E000203AF1885043484331684FF0800A0F1844
:1052F00000252EE0002423E0BBF1FF0F3A7804F0F4
:1053000007012AFA01F002EA000201D00AB908E016
:1053100082B108EB050081B209EB040080B20A9A61
:1053200006E008EB050081B209EB040080B25A46A2
:10533000FFF712FCE043400700D17F1C641CA4B2BD
:10534000B088A042D8D83079400700D07F1C6D1CAF
:10535000ADB2F088A842CDD8D7E42DE9FC5F8046F5
:10536000484889460D4681884446DDF834B01E46DB
:105370001746A14203D3C1888246A94222D2BDE882
:10538000FC5F524800F07CBAB088BAF804300119CA
:10539000994203D9F188444629448DB2F188BAF87C
:1053A00006002944814201D944464D460C983346B3
:1053B000CDE900B029462046FFF779FFB0887F1C71
:1053C000204484B23A78002ADED1BDE8FC9F2DE962
:1053D000F05F1D46904606468A46DDF82CB0DFE0B9
:1053E0007F294FF000007DD8AA8875E053232C68F0
:1053F000434314F813308B426DD1532148430221AB
:1054000001EB400004EB0009002736E000242BE00C
:105410004FEAE47004EB507020F00700A4EB0002A8
:10542000BBF1FF0F99F800104FF0800020FA02F056
:1054300001EA000101D009B907E071B10AEB0700E8
:1054400081B2301980B20A9A05E00AEB070081B2F6
:10545000301980B25A46FFF77FFB1D4820400728CD
:1054600001D109F10109641C2889A042D0DC287A05
:10547000400701D009F101097F1C6889B842C5DCE9
:105480002CE02FE0DC000020443601084465627502
:10549000673A205061696E745F4472617743686156
:1054A0007220496E70757420657863656564732039
:1054B000746865206E6F726D616C20646973706CC6
:1054C00061792072616E67650D0A0000003601087F
:1054D00007000080FFE7401C824287DC08F10108DA
:1054E000E8885CE00127AB8854E053222C684243F3
:1054F00014F812C08C454CD107EB4202A45C98F81A
:105500000120944245D1532250430222296802EBE4
:10551000400001EB0009002737E000242CE000BF29
:105520004FEAE47004EB507020F00700A4EB000297
:10553000BBF1FF0F99F800104FF0800020FA02F045
:1055400001EA000101D009B907E071B10AEB0700D7
:1055500081B2301980B20A9A05E00AEB070081B2E5
:10556000301980B25A46FFF7F7FA934820400728CF
:1055700001D109F10109641C2889A042D0DC287AF4
:10558000400701D009F101097F1C6889B842C4DCD9
:1055900002E0401C8342A8DC288908F10208064486
:1055A00098F8001000297FF41BAFD5E62DE9FF4FD6
:1055B000ADF5037D8846DDE990AB814600244FF4CC
:1055C000807715462646394642A800F026F9394626
:1055D00002A800F022F9794842AA83884B4503D3F8
:1055E000C38802A8434510D275A000F049F90DF513
:1055F000077DECE595FBF1F301FB135395FBF1F50A
:1056000030330355641C24B200E00A21002DF1D18F
:105610001146002C08DD031913F8013C8B55761C4C
:10562000641E36B224B2F4E7CDE900BA41464846DA
:10563000869BFFF792FEDAE72DE9FF4F85B070A158
:1056400017468046DDE9126507C902AB4FF00A092B
:1056500083E8070039790898B1FBF9F19A46848804
:105660001AF80120CDE900564046089B0699FFF73D
:105670001EFE397908EB040BB1FBF9F209FB12119C
:105680001FFA8BF01AF80120CDE90056089B069905
:10569000FFF70DFECDE900560BEB940000EB540034
:1056A00080B23A22089B0699FFF701FE797908EB50
:1056B0004400B1FBF9F100EB54001AF80120CDE9E8
:1056C000005680B2089B0699FFF7F1FD797904EB4B
:1056D000440BB1FBF9F209FB12110BEB08001AF8AD
:1056E0000120CDE9005600EB540080B2089B0699DA
:1056F000FFF7DDFD08EB8400CDE9005600EB540018
:10570000A0EB940080B23A22089B0699FFF7CFFDE8
:10571000B979089BB1FBF9F11AF8012004EB840177
:10572000CDE9005601EB080080B20699FFF7BFFDF6
:10573000BA7908EB4B00B2FBF9F109FB112180B2F9
:105740001AF80120CDE90056089B0699FFF7AFFD36
:105750003CE570B50022194B0EE0002107E000BFC8
:1057600002FB04141E68055D491C355589B25C8A2C
:105770008C42F5D8521C92B2998A9142EDD870BDF4
:10578000F0B500230D4A491E12E000240BE000BFD3
:10579000978A03FB05466F434F438519641C7D5D63
:1057A0001768A4B2BD55558AA542F1D85B1C9BB2BF
:1057B000948A9C42E9D8F0BD07000080DC000020FC
:1057C00044656275673A205061696E745F4469731D
:1057D0004E756D20496E70757420657863656564DB
:1057E0007320746865206E6F726D616C20646973DC
:1057F000706C61792072616E67650D0A00000000AF
:10580000303132333435363738390000D2B201E026
:1058100000F8012B491EFBD270470022F6E710B5B5
:1058200013460A4604461946FFF7F0FF204610BD0E
:1058300030B50B46014600202022012409E021FA60
:1058400002F59D4205D303FA02F5491B04FA02F55D
:105850002844151EA2F10102F1DC30BD064C074DB3
:1058600006E0E06840F0010394E807009847103430
:10587000AC42F6D3FAF760FC88360108A836010876
:105880000FB4054B10B503A9044A029800F018F8AC
:1058900010BC5DF814FB0000C703000838000020AE
:1058A00002E008C8121F08C1002AFAD170477047E9
:1058B000002001E001C1121F002AFBD17047000047
:1058C0002DE9FF4F8BB09A460F460546002606E0AD
:1058D00025280BD052460D9990476D1C761C2878D0
:1058E0000028F5D10FB03046BDE8F08F0024A04667
:1058F0000122604900E0044315F8013F203B02FA11
:1059000003F00842F7D128782E2817D115F8010F97
:1059100044F004042A280ED06FF02F022878A0F15A
:10592000300109290AD808EB880102EB410100EB9C
:1059300001086D1CF2E757F8048B6D1C2878692864
:105940003ED006DC0028CDD063280BD0642804D1DB
:1059500036E0732810D075284BD052460D999047E9
:10596000761C85E017F8040B8DF8000000208DF8F8
:105970000100E946012003E057F8049B4FF0FF3097
:1059800061074FF0000401D40AE0641C44450DDABD
:105990008442FADB19F804100029F6D106E0641CF1
:1059A0008442FCDB19F804100029F8D1264404E0F5
:1059B00019F8010B52460D999047641EF8D257E032
:1059C00001CF4FF00A0B002802DA40422D2102E0FD
:1059D000210504D52B218DF82410012103E0E107D6
:1059E00005D02021F7E70DF1200908910CE00021F6
:1059F000F9E701CF4FF00A0BF9E75946FFF718FF17
:105A000001F1300209F8012D0028F6D1ADEB0900B3
:105A100000F1200B600701D44FF00108D84502DDEA
:105A2000A8EB0B0000E000208046002406E009A857
:105A30005246005D0D999047641C761C089884427C
:105A4000F5DB04E0302052460D999047761CB8F102
:105A50000001A8F10108F5DC05E019F8010B524638
:105A60000D999047761CBBF10001ABF1010BF4DC02
:105A70006D1C34E70928010010B5002821D0114B16
:105A80000022001F196803E0814203D80A464968D2
:105A90000029F9D152B11368841A9C4204D10068DC
:105AA00018441060104602E0506000E0186039B100
:105AB00002680B1A934203D10B681A4402604968CA
:105AC000416010BD3C000020F0B50B30154D20F0BA
:105AD00007010024144A0FE003688B420BD38B426A
:105AE00005D95E1A43184768C3E9006700E04368B8
:105AF000136002C004E0021D10680028ECD12046AB
:105B0000002802D1286808B10020F0BD064A0748E5
:105B10001060074A121A22F00702C0E9002401208F
:105B20002860D7E7400000203C000020FC00002057
:105B3000F8900020000000000000000001020304B3
:105B4000060708090000000001020304FFFFFFFF31
:105B5000FFFFFFFFFFFFFFFFFFFFFFFFFFFFFFFF55
:105B6000FFFFFFFFFFFFFFFFFFFFFFFFFFFFFFFF45
:105B7000FFFFFFFFFFFFFFFFFFFFFFFFFFFFFFFF35
:105B8000FFFFFFFFFFFFFFFFFFFFFFFFFFFFFFFF25
:105D6000FFFFFFFFFFFFFFFFF7FFFFFFFFFFFFFF4B
:105D7000FFFFFFFFFFFFFFFFFFFFFFFFFFFFFFFF33
:105D8000FFFFFFFFFFFFFFFFFFFFFFFFFFFFFFFF23
:105D9000FFFFFFFFFFFFFFFFFFFFC3FFFFFFFFFF4F
:105DA000FFFFFFFFFFFFFFFFFFFFFFFFFFFFFFFF03
:105DB000FFFFFFFFFFFFFFFFFFFFFFFFFFFFFFFFF3
:105DC000FFFFFFFFFFFFFFFFFFFFFFFE07FFFFFFDC
:105DD000FFFFFFFFFFFFFFFFFFFFFFFFFFFFFFFFD3
:105DE000FFFFFFFFFFFFFFFFFFFFFFFFFFFFFFFFC3
:105DF000FFFFFFFFFFFFFFFFFFFFFFFFFFF007FFBA
:105E0000FFFFFFFFFFFFFFFFFFFFFFFFFFFFFFFFA2
:105E1000FFFFFFFFFFFFFFFFFFFFFFFFFFFFFFFF92
:105E2000FFFFFFFFFFFFFFFFFFFFFFFFFFFFFFC0C1
:105E300007FFFFFFFFFFFFFFFFFFFFFFFFFFFFFF6A
:105E4000FFFFFFFFFFFFFFFFFFFFFFFFFFFFFFFF62
:105E5000FFFFFFFFFFFFFFFFFFFFFFFFFFFFFFFF52
:105E6000FE0007FFFFFFFFFFFFFFFFFFFFFFFFFF3A
:105E7000FFFFFFFFFFFFFFFFFFFFFFFFFFFFFFFF32
:105E8000FFFFFFFFFFFFFFFFFFFFFFFFFFFFFFFF22
:105E9000FFFFF80003FFFFFFFFFFFFFFFFFFFFFF14
:105EA000FFFFFFFFFFFFFFFFFFFFFFFFFFFFFFFF02
:105EB000FFFFFFFFFFFFFFFFFFFFFFFFFFFFFFFFF2
:105EC000FFFFFFFFE3D003FFFFFFFFFFFFFFFFFF29
:105ED000FFFFFFFFFFFFFFFFFFFFFFFFFFFFFFFFD2
:105EE000FFFFFFFFFFFFFFFFFFFFFFFFFFFFFFFFC2
:105EF000FFFFFFFFFFFFCFEB03FFFFFFFFFFFFFFF2
:105F0000FFFFFFFFFFFFFFFFFFFFFFFFFFFFFFFFA1
:105F1000FFFFFFFFFFFFFFFFFFFFFFFFFFFFFFFF91
:105F2000FFFFFFFFFFFFFFFF03E383FFFFFFFFFF15
:105F3000FFFFFFFFFFFFFFFFFFFFFFFFFFFFFFFF71
:105F4000FFFFFFFFFFFFFFFFFFFFFFFFFFFFFFFF61
:105F5000FFFFFFFFFFFFFFFFFFFE43F3C3FFFFFF56
:105F6000FFFFFFFFFFFFFFFFFFFFFFFFFFFFFFFF41
:105F7000FFFFFFFFFFFFFFFFFFFFFFFFFFFFFFFF31
:105F8000FFFFFFFFFFFFFFFFFFFFFFF9C3F3E3FC8E
:105F9000FFFFFFFFFFFFFFFFFFFFFFFFFFFFFFFF11
:105FA000FFFFFFFFFFFFFFFFFFFFFFFFFFFFFFFF01
:105FB000FFFFFFFFFFFFFFFFFFFFFFFFFFF3E3F91F
:105FC000E3F8FFFFFFFFFFFFFFFFFFFFFFFFFFFF04
:105FD000FFFFFFFFFFFFFFFFFFFFFFFFFFFFFFFFD1
:105FE000FFFFFFFFFFFFFFFFFFFFFFFFFFFFFFE5DB
:105FF000FFFBF3E0FFFFFFFFFFFFFFFFFFFFFFFFE0
:10600000FFFFFFFFFFFFFFFFFFFFFFFFFFFFFFFFA0
:10601000FFFFFFFFFFFFFFFFFFFFFFFFFFFFFFFF90
:10602000FFC8FFFBF3C07FFFFFFFFFFFFFFFFFFF86
:10603000FFFFFFFFFFFFFFFFFFFFFFFFFFFFFFFF70
:10604000FFFFFFFFFFFFFFFFFFFFFFFFFFFFFFFF60
:10605000FFFFFF92FFFBF7007FFFFFFFFFFFFFFF48
:10606000FFFFFFFFFFFFFFFFFFFFFFFFFFFFFFFF40
:10607000FFFFFFFFFFFFFFFFFFFFFFFFFFFFFFFF30
:10608000FFFFFFFFFF30FFF3F4007FFFFFFFFFFF85
:10609000FFFFFFFFFFFFFFFFFFFFFFFFFFFFFFFF10
:1060A000FFFFFFFFFFFFFFFFFFFFFFFFFFFFFFFF00
:1060B000FFFFFFFFFFFFFE5BFFF3F0707FFFFFFFBF
:1060C000FFFFFFFFFFFFFFFFFFFFFFFFFFFFFFFFE0
:1060D000FFFFFFFFFFFFFFFFFFFFFFFFFFFFFFFFD0
:1060E000FFFFFFFFFFFFFFFFFE0BFFF3E1F87FFF66
:1060F000FFFFFFFFFFFFFFFFFFFFFFFFFFFFFFFFB0
:10610000FFFFFFFFFFFFFFFFFFFFFFFFFFFFFFFF9F
:10611000FFFFFFFFFFFFFFFFFFFFFC09FFF385FC11
:106120007FFFFFFFFFFFFFFFFFFFFFFFFFFFFFFFFF
:10613000FFFFFFFFFFFFFFFFFFFFFFFFFFFFFFFF6F
:10614000FFFFFFFFFFFFFFFFFFFFFFFFF94CFFE730
:106150003DFE7FFFFFFFFFFFFFFFFFFFFFFFFFFF92
:10616000FFFFFFFFFFFFFFFFFFFFFFFFFFFFFFFF3F
:10617000FFFFFFFFFFFFFFFFFFFFFFFFFFFFF27EBD
:106180007FE6FDFE3FFFFFFFFFFFFFFFFFFFFFFF7B
:10619000FFFFFFFFFFFFFFFFFFFFFFFFFFFFFFFF0F
:1061A000FFFFFFFFFFFFFFFFFFFFFFFFFFFFFFFFFF
:1061B000F03FBFE19DFE3FFFFFFFFFFFFFFFFFFF3F
:1061C000FFFFFFFFFFFFFFFFFFFFFFFFFFFFFFFFDF
:1061D000FFFFFFFFFFFFFFFFFFFFFFFFFFFFFFFFCF
:1061E000FFFFE43FDFE39DFF3FFFFFFFFFFFFFFFF8
:1061F000FFFFFFFFFFFFFFFFFFFFFFFFFFFFFFFFAF
:10620000FFFFFFFFFFFFFFFFFFFFFFFFFFFFFFFF9E
:10621000FFFFFFFFE4DFFFC67DFF3FFFFFFFFFFF44
:10622000FFFFFFFFFFFFFFFFFFFFFFFFFFFFFFFF7E
:10623000FFFFFFFFFFFFFFFFFFFFFFFFFFFFFFFF6E
:10624000FFFFFFFFFFFFEFFFFFDEFFFF9FFFFFFFEF
:10625000FFFFFFFFFFFFFFFFFFFFFFFFFFFFFFFF4E
:10626000FFFFFFFFFFFFFFFFFFFFFFFFFFFFFFFF3E
:10627000FFFFFFFFFFFFFFFFCFFFFF93FFFF9FFF2A
:10628000FFFFFFFFFFFFFFFFFFFFFFFFFFFFFFFF1E
:10629000FFFFFFFFFFFFFFFFFFFFFFFFFFFFFFFF0E
:1062A000FFFFFFFFFFFFFFFFFFFFCDFFFF33FFFFFC
:1062B0009FFFFFFFFFFFFFFFFFFFFFFFFFFFFFFF4E
:1062C000FFFFFFFFFFFFFFFFFFFFFFFFFFFFFFFFDE
:1062D000FFFFFFFFFFFFFFFFFFFFFFFFC0FFFE1FEE
:1062E000FDFF9FFFFFFFFFFFFFFFFFFFFFFFFFFF20
:1062F000FFFFFFFFFFFFFFFFFFFFFFFFFFFFFFFFAE
:10630000FFFFFFFFFFFFFFFFFFFFFFFFFFFFC9FFD3
:10631000FC8FFFFF9FFFFFFFFFFFFFFFFFFFFFFF60
:10632000FFFFFFFFFFFFFFFFFFFFFFFFFFFFFFFF7D
:10633000FFFFFFFFFFFFFFFFFFFFFFFFFFFFFFFF6D
:10634000C9FFF9FFFDFF8FFFFFFFFFFFFFFFFFFF0B
:10635000FFFFFFFFFFFFFFFFFFFFFFFFFFFFFFFF4D
:10636000FFFFFFFFFFFFFFFFFFFFFFFFFFFFFFFF3D
:10637000FFFFCFFFF0FFF5FF8FFFFFFFFFFFFFFFE6
:10638000FFFFFFFFFFFFFFFFFFFFFFFFFFFFFFFF1D
:10639000FFFFFFFFFFFFFFFFFFFFFFFFFFFFFFFF0D
:1063A000FFFFFFFFE7FFF67FF7FF8FFFFFFFFFFF16
:1063B000FFFFFFFFFFFFFFFFFFFFFFFFFFFFFFFFED
:1063C000FFFFFFFFFFFFFFFFFFFFFFFFFFFFFFFFDD
:1063D000FFFFFFFFFFFFE7FFE33FFDFF8FFFFFFF33
:1063E000FFFFFFFFFFFFFFFFFFFFFFFFFFFFFFFFBD
:1063F000FFFFFFFFFFFFFFFFFFFFFFFFFFFFFFFFAD
:10640000FFFFFFFFFFFFFFFFF3FFEF9F0BFF87FF84
:10641000FFFFFFFFFFFFFFFFFFFFFFFFFFFFFFFF8C
:10642000FFFFFFFFFFFFFFFFFFFFFFFFFFFFFFFF7C
:10643000FFFFFFFFFFFFFFFFFFFFF3FFCE4FA1FFB7
:1064400087FFFFFFFFFFFFFFFFFFFFFFFFFFFFFFD4
:10645000FFFFFFFFFFFFFFFFFFFFFFFFFFFFFFFF4C
:10646000FFFFFFFFFFFFFFFFFFFFFFFFF9FFD72742
:10647000F3FF97FFFFFFFFFFFFFFFFFFFFFFFFFFA0
:10648000FFFFFFFFFFFFFFFFFFFFFFFFFFFFFFFF1C
:10649000FFFFFFFFFFFFFFFFFFFFFFFFFFFFFCFB13
:1064A000D3C3FBFF97FFFFFFFFFFFFFFFFFFFFFFD0
:1064B000FFFFFFFFFFFFFFFFFFFFFFFFFFFFFFFFEC
:1064C000FFFFFFFFFFFFFFFFFFFFFFFFFFFFFFFFDC
:1064D000FE7CD3E1FBFF97FFFFFFFFFFFFFFFFFF06
:1064E000FFFFFFFFFFFFFFFFFFFFFFFFFFFFFFFFBC
:1064F000FFFFFFFFFFFFFFFFFFFFFFFFFFFFFFFFAC
:10650000FFF00F3E1FF1FFFFC7FFFFFFFFFFFFFF81
:10651000FFFFFFFFFFFFFFFFFFFFFFFFFFFFFFFF8B
:10652000FFFFFFFFFFFFFFFFFFFFFFFFFFFFFFFF7B
:10653000FFFFFFC0008F93F8DFFFC7FFFFFFFFFFE4
:10654000FFFFFFFFFFFFFFFFFFFFFFFFFFFFFFFF5B
:10655000FFFFFFFFFFFFFFFFFFFFFFFFFFFFFFFF4B
:10656000FFFFFFFFFFCFFC0393FE5FFFC7FFFFFFAF
:10657000FFFFFFFFFFFFFFFFFFFFFFFFFFFFFFFF2B
:10658000FFFFFFFFFFFFFFFFFFFFFFFFFFFFFFFF1B
:10659000FFFFFFFFFFFFFFA3FFE0CFFF7FFFC7FF6E
:1065A000FFFFFFFFFFFFFFFFFFFFFFFFFFFFFFFFFB
:1065B000FFFFFFFFFFFFFFFFFFFFFFFFFFFFFFFFEB
:1065C000FFFFFFFFFFFFFFFFFF79FFFC0FFF3F7F94
:1065D000E7FFFFFFFFFFFFFFFFFFFFFFFFFFFFFFE3
:1065E000FFFFFFFFFFFFFFFFFFFFFFFFFFFFFFFFBB
:1065F000FFFFFFFFFFFFFFFFFFFFFEFE7FF8F7FF3C
:106600009F7FE3FFFFFFFFFFFFFFFFFFFFFFFFFF96
:10661000FFFFFFFFFFFFFFFFFFFFFFFFFFFFFFFF8A
:10662000FFFFFFFFFFFFFFFFFFFFFFFFFEFFFFF387
:10663000D3F7DFBFE3FFFFFFFFFFFFFFFFFFFFFF1A
:10664000FFFFFFFFFFFFFFFFFFFFFFFFFFFFFFFF5A
:10665000FFFFFFFFFFFFFFFFFFFFFFFFFFFFFCBF8D
:10666000FFC1EBFBCF9FE3FFFFFFFFFFFFFFFFFF3C
:10667000FFFFFFFFFFFFFFFFFFFFFFFFFFFFFFFF2A
:10668000FFFFFFFFFFFFFFFFFFFFFFFFFFFFFFFF1A
:10669000FC0FFFDC71FBEFCFE7FFFFFFFFFFFFFF0A
:1066A000FFFFFFFFFFFFFFFFFFFFFFFFFFFFFFFFFA
:1066B000FFFFFFFFFFFFFFFFFFFFFFFFFFFFFFFFEA
:1066C000FFFFF9BFFFAFFCF9FFEFE7FFFFFFFFFFA1
:1066D000FFFFFFFFFFFFFFFFFFFFFFFFFFFFFFFFCA
:1066E000FFFFFFFFFFFFFFFFFFFFFFFFFFFFFFFFBA
:1066F000FFFFFFFFFBFFFF47FE79F7F7A7FFFFFF55
:10670000FFFFFFFFFFFFFFFFFFFFFFFFFFFFFFFF99
:10671000FFFFFFFFFFFFFFFFFFFFFFFFFFFFFFFF89
:10672000FFFFFFFFFFFFFBFFFE47FF39F7FBA7FF60
:10673000FFFFFFFFFFFFFFFFFFFFFFFFFFFFFFFF69
:10674000FFFFFFFFFFFFFFFFFFFFFFFFFFFFFFFF59
:10675000FFFFFFFFFFFFFFFFFA3FFCEFFF99FBFD8D
:1067600087FFFFFFFFFFFFFFFFFFFFFFFFFFFFFFB1
:10677000FFFFFFFFFFFFFFFFFFFFFFFFFFFFFFFF29
:10678000FFFFFFFFFFFFFFFFFFFFFA3FFCFFFFC917
:10679000FDFC87F87FFFFFFFFFFFFFFFFFFFFFFF0D
:1067A000FFFFFFFFFFFFFFFFFFFFFFFFFFFFFFFFF9
:1067B000FFFFFFFFFFFFFFFFFFFFFFFFFA07FDFFE8
:1067C000FFE0FCFE07C00FFFFFFFFFFFFFFFFFFF23
:1067D000FFFFFFFFFFFFFFFFFFFFFFFFFFFFFFFFC9
:1067E000FFFFFFFFFFFFFFFFFFFFFFFFFFFFF87F40
:1067F000F9FFFFF87E7E0F9FF3FFFFFFFFFFFFFF14
:10680000FFFFFFFFFFFFFFFFFFFFFFFFFFFFFFFF98
:10681000FFFFFFFFFFFFFFFFFFFFFFFFFFFFFFFF88
:10682000F3FFFBFFFFFE3F390F2019FFFFFFFFFFC4
:10683000FFFFFFFFFFFFFFFFFFFFFFFFFFFFFFFF68
:10684000FFFFFFFFFFFFFFFFFFFFFFFFFFFFFFFF58
:10685000FFFFF3FFFBFFFFFF0F980E0FC1FFFFFFCE
:10686000FFFFFFFFFFFFFFFFFFFFFFFFFFFFFFFF38
:10687000FFFFFFFFFFFFFFFFFFFFFFFFFFFFFFFF28
:10688000FFFFFFFFF23FFBFFFFFFC7C00C7FF3FFDF
:10689000FFFFFFFFFFFFFFFFFFFFFFFFFFFFFFFF08
:1068A000FFFFFFFFFFFFFFFFFFFFFFFFFFFFFFFFF8
:1068B000FFFFFFFFFFFFFA3FFBFFFFFFF02009FF95
:1068C000F9FFFFFFFFFFFFFFFFFFFFFFFFFFFFFFDE
:1068D000FFFFFFFFFFFFFFFFFFFFFFFFFFFFFFFFC8
:1068E000FFFFFFFFFFFFFFFFFBFFF3FFFFFFFC00CA
:1068F00001FFF9FFFFFFFFFFFFFFFFFFFFFFFFFFAC
:10690000FFFFFFFFFFFFFFFFFFFFFFFFFFFFFFFF97
:10691000FFFFFFFFFFFFFFFFFFFFFBFFEBFF803FDE
:10692000FE0007FFFCFFFFFFFFFFFFFFFFFFFFFF72
:10693000FFFFFFFFFFFFFFFFFFFFFFFFFFFFFFFF67
:10694000FFFFFFFFFFFFFFFFFFFFFFFFF93FDBD868
:106950001FC7FF800FFFFCFFFFFFFFFFFFFFFFFFD1
:10696000FFFFFFFFFFFFFFFFFFFFFFFFFFFFFFFF37
:10697000FFFFFFFFFFFFFFFFFFFFFFFFFFFFF93EEE
:106980005BEC7FFC3F800FFFFFFFFFFFFFFFFFFF80
:10699000FFFFFFFFFFFFFFFFFFFFFFFFFFFFFFFF07
:1069A000FFFFFFFFFFFFFFFFFFFFFFFFFFFFFFFFF7
:1069B000FCFF1BFF8FFF80001FFFFFFFFFFFFFFF9C
:1069C000FFFFFFFFFFFFFFFFFFFFFFFFFFFFFFFFD7
:1069D000FFFFFFFFFFFFFFFFFFFFFFFFFFFFFFFFC7
:1069E000FFFFFCFF3BFFF9FFFF001FFFFFFFFFFF63
:1069F000FFFFFFFFFFFFFFFFFFFFFFFFFFFFFFFFA7
:106A0000FFFFFFFFFFFFFFFFFFFFFFFFFFFFFFFF96
:106A1000FFFFFFFFFE7EBBFFFFFFFF803FFFFFFF8B
:106A2000FFFFFFFFFFFFFFFFFFFFFFFFFFFFFFFF76
:106A3000FFFFFFFFFFFFFFFFFFFFFFFFFFFFFFFF66
:106A4000FFFFFFFFFFFFFF3EBBFFFFEFFF003FFF2A
:106A5000FFFFFFFFFFFFFFFFFFFFFFFFFFFFFFFF46
:106A6000FFFFFFFFFFFFFFFFFFFFFFFFFFFFFFFF36
:106A7000FFFFFFFFFFFFFFFFFFBE53FFFFF3FE001F
:106A80003FFFFFFFFFFFFFFFFFFFFFFFFFFFFFFFD6
:106A9000FFFFFFFFFFFFFFFFFFFFFFFFFFFFFFFF06
:106AA000FFFFFFFFFFFFFFFFFFFFFF9F13FFFFF849
:106AB000FC047FFFFFFFFFFFFFFFFFFFFFFFFFFF64
:106AC000FFFFFFFFFFFFFFFFFFFFFFFFFFFFFFFFD6
:106AD000FFFFFFFFFFFFFFFFFFFFFFFFFFCF83FF72
:106AE000FFFE180C7FFFFFFFFFFFFFFFFFFFFFFF11
:106AF000FFFFFFFFFFFFFFFFFFFFFFFFFFFFFFFFA6
:106B0000FFFFFFFFFFFFFFFFFFFFFFFFFFFFFFE7AD
:106B1000C3FFFFFFC01CFFFFFFFFFFFFFFFFFFFFE3
:106B2000FFFFFFFFFFFFFFFFFFFFFFFFFFFFFFFF75
:106B3000FFFFFFFFFFFFFFFFFFFFFFFFFFFFFFFF65
:106B4000FFF3E7FFFFFFFE7CFFFFFFFFFFFFFFFFFD
:106B5000FFFFFFFFFFFFFFFFFFFF01FFFFFFFFFF43
:106B6000FFFFFFFFFFFFFFFFFFFFFFFFFFFFFFFF35
:106B7000FFFFFFF9E3FFFFFFF9FDFFFFFFFFFFFF4F
:106B8000FFFFFFFFFFFFFFFFFFFFFFF8000FFFFF0B
:106B9000FFFFFFFFFFFFFFFFFFFFFFFFFFFFFFFF05
:106BA000FFFFFFFFFFFE73FFFEFFE3FDFFFFFFFFA1
:106BB000FFFFFFFFFFFFFFFFFFFFFFFFFFF1FF836F
:106BC000FFFFFFFFFFFFFFFFFFFFFFFFFFFFFFFFD5
:106BD000FFFFFFFFFFFFFFFF33FDFEF88FFFFFFF0B
:106BE000FFFFFFFFFFFFFFFFFFFFFFFFFFFFFFE7CD
:106BF000FFF0FFFFFFFFFFFFFFFFFFFFFFFFFFFFB4
:106C0000FFFFFFFFFFFFFFFFFFFF93EB7EF83FFF5C
:106C1000FFFFFFFFFFFFFFFFFFFFFFFFFFFFFFFF84
:106C2000FFDFFFD87FFFFFFFFFFFFFFFFFFFFFFF3B
:106C3000FFFFFFFFFFFFFFFFFFFFFFFFC3F8FFF8AE
:106C4000FFFFFFFFFFFFFFFFFFFFFFFFFFFFFFFF54
:106C5000FFFFFF9FFBDB1FFFFFFFFFFFFFFFFFFFAC
:106C6000FFFFFFFFFFFFFFFFFFFFFFFFFFFFE1F958
:106C7000FFC3FFFFFFFFFFFFFFFFFFFFFFFFFFFF60
:106C8000FFFFFF7FF3BFF80BCFFFFFFFFFFFFFFF0B
:106C9000FFFFFFFFFFFFFFFFFFFFFFFFFFFFFFFF04
:106CA000F9F3FF0FFFFFFFFFFFFFFFFFFFFFFFFFF6
:106CB000FFFFFFFFFE1F813FFFE3E7FFFFFFFFFF37
:106CC000FFFFFFFFFFFFFFFFFFFFFFFFFFFFFFFFD4
:106CD000FFFFFCF7F87FFFFFFFFFFFFFFFFFFFFF56
:106CE000FFFFFFFFFFFFFECF1C3FFFF3E3FFFFFFB0
:106CF000FFFFFFFFFFFFFFFFFFFFFFFFFFFFFFFFA4
:106D0000FFFFFFFFFE77C1FFFFFFFFFFFFFFFFFF5A
:106D1000FFFFFFFFFFFFFFFFFEE09C3FFFFBCBFFFE
:106D2000FFFFFFFFFFFFFFFFFFFFFFFFFFFFFFFF73
:106D3000FFFFFFFFFFFFFF201FFFFFFFFFFFFFFF22
:106D4000FFFFFFFFFFFFFFFFFFFFFCF19C1FFFF3B3
:106D5000D9FFFFFFFFFFFFFFFFFFFFFFFFFFFFFF69
:106D6000FFFFFFFFFFFFFFFFFFE0FFFFFFFFFFFF52
:106D7000FFFFFFFFFFFFFFFFFFFFFFFF7EFED99F2B
:106D8000FFF79CFF87FFFFFFFFFFFFFFFFFFFFFFF6
:106D9000FFFFFFFFFFFFFFFFFFFFFFFFFFFFFFFF03
:106DA000FFFFFFFFFFFFFFFFFFFFFFFFFFFE3E3E76
:106DB00059CEFFE41CFF23FFFFFFFFFFFFFFFFFF94
:106DC000FFFFFFFFFFFFFFFFFFFFFFFFFFFFFFFFD3
:106DD000FFFFFFFFFFFFFFFFFFFFFFFFFFFFFFFFC3
:106DE0007F1F19CCFFE0C6FEF9FFFFFFFFFFFFFF8B
:106DF000FFFFFFFFFFFFFFFFFFFFFFFFFFFFFFFFA3
:106E0000FFFFFFFFFFFFFFFFFFFFFFFFFFFFFFFF92
:106E1000FFFFFF1F19E5FFC7E07EF9FFFFFFFFFF40
:106E2000FFFFFFFFFFFFFFFFFFFFFFFFFFFFFFFF72
:106E3000FFFFFFFFFFFFFFFFFFFFFFFFFFFFFFFF62
:106E4000FFFFFFFFFF1F93E4FFCFFF7FF9FFFFFF6F
:106E5000FFFFFFFFFFFFFFFFFFFFFFFFFFFFFFFF42
:106E6000FFFFFFFFFFFFFFFFFFFFFFFFFFFFFFFF32
:106E7000FFFFFFFFFFFFFF2F93F4FF9FFF7DF9FF51
:106E8000FFFFFFFFFFFFFFFFFFFFFFFFFFFFFFFF12
:106E9000FFFFFFFFFFFFFFFFFFFFFFFFFFFFFFFF02
:106EA000FFFFFFFFFFFFFFFFFE6FC7F03F3FFF3D0C
:106EB000F9FFFFFFFFFFFFFFFFFFFFFFFFFFFFFFE8
:106EC000FFFFFFFFFFFFFFFFFFFFFFFFFFFFFFFFD2
:106ED000FFFFFFFFFFFFFFFFFFFFE07FCFF27E7F9F
:106EE000FF3DF9FDFFFFFFFFFFFFFFFFFFFFFFFF7C
:106EF000FFFFFFFFFFFFFFFFFFFFFFEFFFFFFFFFB2
:106F0000FFFFFFFFFFFFFFFFFFFFFFFF803FCFF00F
:106F1000FCFFFF39F8F8FFFFFFFFFFFFFFFFFFFF58
:106F2000FFFFFFFFFFFFFFFFFFFFFFFFFFFFFFFF71
:106F3000FFFFFFFFFFFFFFFFFFFFFFFFFFFE078FCA
:106F4000CFF1F9FFFF33FC78FFFFFFFFFFFFFFFFEB
:106F5000FFFFFFFFFFFFFFFFFFFFFFFFFFFFFFFF41
:106F6000FFFFFFFFFFFFFFFFFFFFFFFFFFFFFFF838
:106F7000E3E7E7F1F3FFFF27FF1FFFFFFFFFFFFF3F
:106F8000FFFFFFFFFFFFFFFFFFFFFFFFFFFFFFFF11
:106F9000FFFFFFFFFFFFFFFFFFFFFFFFFFFFFFFF01
:106FA000FFF1F1F3E7F3F7FFFF0FFFFFFFFFFFFF35
:106FB000FFFFFFFFFFFFFFFFFFFFFFFFFFFFFFFFE1
:106FC000FFFFFFFFFFFFFFFFFFFFFFFFFFFFFFFFD1
:106FD000FFFFFFE7F9FDE3E3E7FFFF3FF3FFFDFFFF
:106FE000FFFFFFFFFFFFFFFFFFFFFFFFFFFFFFFFB1
:106FF000FFFFFFFFFFFFFFFFFFFFFFFFFFFFFFFFA1
:10700000FFFFFFFFFFCFFCFCE1E7E7FFFE7FF7FF9D
:10701000FDFFFFFFFFFFFFFFFFFFFFFFFFFFFFFF82
:10702000FFFFFFFFFFFFFFFFFFFFFFFFFFFFFFFF70
:10703000FFFFFFFFFFFFFFDFFCFE75CFCFFFF87FF5
:10704000F7F3FDFFFFFFFFFFFFFFFFFFFFFFFFFF66
:10705000FFFFFFFFFFFFFFFFFFFFFFFFFFFFFFFF40
:10706000FFFFFFFFFFFFFFFFFF9FFEFF749FCFFEAD
:1070700000FFFFF7FFFFFFFFFFFF87FFFFFFFFFF9F
:10708000FFFFFE07FFFFFFFFFFFFFFFFFFFFFFFF09
:10709000FFFFFFFFFFFFFFFFFFFFFF9FFE7F3A3F66
:1070A0008FE005FFFFFFFFFFFFFFFFFE10FFFFFF69
:1070B000FFFFFFE00003FFFFFFFFFFFFFFFFFFFFFA
:1070C000FFFFFFFFFFFFFFFFFFFFFFFFFFBFFE7F91
:1070D000387F8F8019FFFFFFFFFFFFFFFFF9FE3FA3
:1070E000FFFFFFFFC0000019FFFFFFFFFFFFFFFFD3
:1070F000FFFFFFFFFFFFFFFFFFFFFFFFFFFFFF3F60
:10710000FF3FBC7F8F03F3FFFFFFF3FFFFFFFFE7AE
:10711000FF8FFFFFFFFC00E0000CFFFFFFFFFFFF02
:10712000FFFFFFFFFFFFFFFFFFFFFFFFFFFFFFFF6F
:10713000FF3FFF3F9C7F8E03C7FFFFFFF3FFFFFF73
:10714000FF1FFFE7FFFFFFF13FFFF0047FFFFFFF9F
:10715000FFFFFFFFFFFFFFFFFFFFFFFFFFFFFFFF3F
:10716000FFFFFF3FFF9FCD3F8C071FFFFFFFF7FF94
:10717000FFFFFC7FFFF3FFFFFFC6FFFFF8427FFF2B
:10718000FFFFFFFFFFFFFFFFFFFFFFFFFFFFFFFF0F
:10719000FFFFFFFFFF7FFF8FC59F841C7FFF00FF66
:1071A000FFFFFFFFF3FF00FDFFFFFF9DFFFFFE223C
:1071B000FFFFFFFFFFFFFFFFFFFFFFFFFFFFFFFFDF
:1071C000FFFFFFFFFFFFFF7FF7CFC19F8419FFFC89
:1071D000001007FFFFFFCFF83C1CFFFFFF3BFFFF46
:1071E000FE10FFFFFFFFFFFFFFFFFFFFFFFFFFFF9F
:1071F000FFFFFFFFFFFFFFFFFF7FE3E3C08F0013F1
:10720000FFF0FF000047FFFC7FE3FFC67FFFFCF7B6
:10721000FFFFFF18FFFFFFFFFFFFFFFFFFFFFFFF65
:10722000FFFFFFFFFFFFFFFFFFFFFE3FE3F000CE8A
:107230000027FFE1FFE3F803FFC3FFC7FFF13FFFB4
:10724000F9E7FFFFFF88FFFFFFFFFFFFFFFFFFFFE3
:10725000FFFFFFFFFFFFFFFFFFFFFFFFFE3FFFFC02
:10726000004C0027FF87FFF00000001FFF9FFFFC7E
:107270001FFFE38FFFFFFF88FFFFFFFFFFFFFFFF01
:10728000FFFFFFFFFFFFFFFFFFFFFFFFFFFFFE1FEF
:10729000FFFF01000067FC0FFFF807FE01F9FE7F0A
:1072A000FFFF0FFF073FFFFFF988FFFFFFFFFFFF13
:1072B000FFFFFFFFFFFFFFFFFFFFFFFFFFFFFFFFDE
:1072C000FE4FFFFFC1807000003FDFFCFFFFFFF9B2
:1072D000FCFFFFFFC0603C7FFFFFFDC0FFFFFFFF23
:1072E000FFFFFFFFFFFFFFFFFFFFFFFFFFFFFFFFAE
:1072F000FFFFFE27FFFFC1C0080000FF9FFE7FFFCA
:10730000FFFDF9FFFFFFF800C1FFFFFFFFE0FFFFF8
:10731000FFFFFFFFFFFFFFFFFFFFFFFFFFFFFFFF7D
:10732000FFFFFFFFFE33FFFFC0E0003800FFBFFE9E
:107330007FFFFFFFF3FFFFFFFFE03FFFFFFFFFE0E7
:10734000FFFFFFFFFFFFFFFFFFFFFFFFFFFFFFFF4D
:10735000FFFFFFFFFFFFFE1DFFFFE0700418007F2F
:10736000FFFF7FFFFFFFE7FFFFFFFFFFFFFFFFFFC5
:10737000FFF0FFFFFFFFFFFFFFFFFFFFFFFFFFFF2C
:10738000FFFFFFFFFFFFFFFFFE0E7FFFE01004087F
:10739000183FFFFF7FFFFFFFCFFFFFFFFFFFFFFF54
:1073A000FFFFFFFC7FFFFFFFFFFFFFFFFFFFFFFF70
:1073B000FFFFFFFFFFFFFFFFFFFFFE471FFFF00084
:1073C00004088E3FFFFF3FFFFFFFDFFFFFFFFFFFD0
:1073D000FFFFFFFFFFFE078FFFFFFFFFFFFFFFFF26
:1073E000FFFFFFFFFFFFFFFFFFFFFFFFFF63C7FF81
:1073F000FC000C008F3FFFFF3FFFFFFFBFFFFFFFC1
:10740000FFFFFFFFFFFFFFFF03FFFFFFFFFFFFFF88
:10741000FFFFFFFFFFFFFFFFFFFFFFFFFFFFFF304B
:10742000F1FFFF821801873FFFFFBFFFFFFF7FFFD4
:10743000FFFFFFFFFFFFFFFFFFFF8FFFFDFFFFFFCE
:10744000FFFFFFFFFFFFFFFFFFFFFFFFFFFFFFFF4C
:10745000FF381CE1FFF1F001C73FFFFF9FFFFFFE78
:107460007FFFFFFFFFFFFFFFFFFFFFFFE3FFFBFFCC
:10747000FFFFFFFFFFFFFFFFFFFFFFFFFFFFFFFF1C
:10748000FFFFFF3E00047F000103C33FFFFF8FFFAC
:10749000FFFEFFFFFFFFFFFFFFFFFFFFFFFFF8FF04
:1074A000FFFFFFFFFFFFFFFFFFFFFFFFFFFFFFFFEC
:1074B000FFFFFFFFFFBF878300000061C39FFFFF47
:1074C0008FFFFFFDFFFFFFFFFFFFFFFFFFFFFFFF3E
:1074D000FE03FFFFFFFFFFFFFFFFFFFFFFFFFFFFB9
:1074E000FFFFFFFFFFFFFF9FFFF1E600C261C39FA9
:1074F000FFFF9FFFFFF9FFFFFFFFFFFFFFFFFFFF02
:10750000FFFFFFFFFFFFFFFFFFFFFFFFFFFFFFFF8B
:10751000FFFFFFFFFFFFFFFFFFDFFFF0780082614B
:10752000E19FFFFF9FFFFFF3FFFFFFFFFFFFFFFF55
:10753000FFFFFFFFFFFFFFFFFFFFFFFFFFFFFFFF5B
:10754000FFFFFFFFFFFFFFFFFFFFFFFFEFE0000177
:107550008661E1FFFFFF9FFFFFE7FFFFFFFFFFFFE8
:10756000FFFFFFFFFFFFFFFFFFFFFFFFFFFFFFFF2B
:10757000FFFFFFFFFFFFFFFFFFFFFFFFFF3FCFE426
:1075800000010040F0FFFFFF1FFFFFCFFFFFFFFFE5
:10759000FFFFFFFFFFFFFFFFFFFFFFFFFFFFFFFFFB
:1075A000FFFFFFFFFFFFFFFFFFFFFFFFFFFFFFF9F1
:1075B000FFFE04018041D07FFFFF1FFFFF9FFFFF01
:1075C000FFFFFFFFFFFFFFFFFFFFFFFFFFFFFFFFCB
:1075D000FFFFFFFFFFFFFFFFFFFFFFFFFFFFFFFFBB
:1075E000FFFC7FF800338040883FFFFF4FFFF87FAC
:1075F000FFFFFFFFFFFFFFFFFFFFFFFFFFFFFFFF9B
:10760000FFFFFFFFFFFFFFFFFFFFFFFFFFFFFFFF8A
:10761000FFFFFFFF0FE023E7C200CC1FFFFF4FFF7C
:10762000F8FFFFFFFFFFFFFFFFFFFFFFFFFFFFFF71
:10763000FFFFFFFFFFFFFFFFFFFFFFFFFFFFFFFF5A
:10764000FFFFFFFFFFFF80064F8FE300FE07FFFEF7
:1076500047FFE1FFFFFFFFFFFFFFFFFFFFFFFFFF10
:10766000FFFFFFFFFFFFFFFFFFFFFFFFFFFFFFFF2A
:10767000FFFFFFFFFFFFFFFFFC7C9C3FF300FF804D
:10768000FFFE13FC07FFFFFFFFFFFFFFFFFFFFFFF2
:10769000FFFFFFFFFFFFFFFFFFFFFFFFFFFFFFFFFA
:1076A000FFFFFFFFFFFFFFFFFFFFFFF9B1FFF980C3
:1076B0007FC03FFC00003FFFFFFFFFFFFFFFFFFF1A
:1076C000FFFFFFFFFFFFFFFFFFFFFFFFFFFFFFFFCA
:1076D000FFFFFFFFFFFFFFFFFFFFFFFFFFF107FFC0
:1076E000F9C07FF00FFC0003FFFFFFFFFFFFFFFF6C
:1076F000FFFFFFFFFFFFFFFFFFFFFFFFFFFFFFFF9A
:10770000FFFFFFFFFFFFFFFFFFFFFFFFFFFFFFF395
:107710001FFFF9E03FFE01F0007FFFFFFFFFFFFFCB
:10772000FFFFFFFFFFFFFFFFFFFFFFFFFFFFFFFF69
:10773000FFFFFFFFFFFFFFFFFFFFFFFFFFFFFFFF59
:10774000FFE33FFFFCF03FFF80003FFFFFFFFFFF35
:10775000FFFFFFFFFFFFFFFFFFFFFFFFFFFFFFFF39
:10776000FFFFFFFFFFFFFFFFFFFFFFFFFFFFFFFF29
:10777000FFFFFFE73FFFFC783FFFC001FFFFFFFF78
:10778000FFFFFFFFFFFFFFFFFFFFFFFFFFFFFFFF09
:10779000FFFFFFFFFFFFFFFFFFFFFFFFFFFFFFFFF9
:1077A000FFFFFFFFFFE73FFFFC7E1FFFF003FFFF30
:1077B000FFFFFFFFFFFFFFFFFFFFFFFFFFFFFFFFD9
:1077C000FFFFFFFFFFFFFFFFFFFFFFFFFFFFFFFFC9
:1077D000FFFFFFFFFFFFFFCE3FFFFC3F8FFFF807DC
:1077E000FFFFFFFFFFFFFFFFFFFFFFFFFFFFFFFFA9
:1077F000FFFFFFFFFFFFFFFFFFFFFFFFFFFFFFFF99
:10780000FFFFFFFFFFFFFFFFFFCE3FFFFC9FC7FF14
:10781000FC0FFFFFFFFFFFFFFFFFFFFFFFFFFFFF6B
:10782000FFFFFFFFFFFFFFFFFFFFFFFFFFFFFFFF68
:10783000FFFFFFFFFFFFFFFFFFFFFFCC9FFFFC9F4E
:10784000E7FFFE1FFFFFFFFFFFFFFFFFFFFFFFFF41
:10785000FFFFFFFFFFFFFFFFFFFFFFFFFFFFFFFF38
:10786000FFFFFFFFFFFFFFFFFFFFFFFFFFC8CFFF8F
:10787000FD9FE0FFFE3FFFFFFFFFFFFFFFFFFFFF5A
:10788000FFFFFFFFFFFFFFFFFFFFFFFFFFFFFFFF08
:10789000FFFFFFFFFFFFFFFFFFFFFFFFFFFFFFC037
:1078A000E7FC79DFF07FFE7FFFFFFFFFFFFFFFFFB9
:1078B000FFFFFFFFFFFFFFFFFFFFFFFFFFFFFFFFD8
:1078C000FFFFFFFFFFFFFFFFFFFFFFFFFFFFFFFFC8
:1078D000FFC1F0F073DFF07FFCFFFFFFFFFFFFFF52
:1078E000FFFFFFFFFFFFFFFFFFFFFFFFFFFFFFFFA8
:1078F000FFFFFFFFFFFFFFFFFFFFFFFFFFFFFFFF98
:10790000FFFFFFC1FC0307DFF0FFF8FFFFFFFFFFF2
:10791000FFFFFFFFFFFFFFFFFFFFFFFFFFFFFFFF77
:10792000FFFFFFFFFFFFFFFFFFFFFFFFFFFFFFFF67
:10793000FFFFFFFFFFC1FFFFDFDFF27FE3FFFFFF7E
:10794000FFFFFFFFFFFFFFFFFFFFFFFFFFFFFFFF47
:10795000FFFFFFFFFFFFFFFFFFFFFFFFFFFFFFFF37
:10796000FFFFFFFFFFFFFFC1FFFFFFDFF30F07FF79
:10797000FFFFFFFFFFFFFFFFFFFFFFFFFFFFFFFF17
:10798000FFFFFFFFFFFFFFFFFFFFFFFFFFFFFFFF07
:10799000FFFFFFFFFFFFFFFFFFC1FFFFFFDFF380E0
:1079A0001FFFFFFFFFFFFFFFFFFFFFFFFFFFFFFFC7
:1079B000FFFFFFFFFFFFFFFFFFFFFFFFFFFFFFFFD7
:1079C000FFFFFFFFFFFFFFFFFFFFFFC1FFFFFF9F65
:1079D000F3E0FFFFFFFFFFFFFFFFFFFFFFFFFFFFE2
:1079E000FFFFFFFFFFFFFFFFFFFFFFFFFFFFFFFFA7
:1079F000FFFFFFFFFFFFFFFFFFFFFFFFFFE1FFFFB5
:107A0000FF9FF3FFFFFFFFFFFFFFFFFFFFFFFFFFF2
:107A1000FFFFFFFFFFFFFFFFFFFFFFFFFFFFFFFF76
:107A2000FFFFFFFFFFFFFFFFFFFFFFFFFFFFFFE184
:107A3000FFFFFF9FF3FFFFFFFFFFFFFFFFFFFFFFC2
:107A4000FFFFFFFFFFFFFFFFFFFFFFFFFFFFFFFF46
:107A5000FFFFFFFFFFFFFFFFFFFFFFFFFFFFFFFF36
:107A6000FFE1FFFFFF9FF3FFFFFFFFFFFFFFFFFFB0
:107A7000FFFFFFFFFFFFFFFFFFFFFFFFFFFFFFFF16
:107A8000FFFFFFFFFFFFFFFFFFFFFFFFFFFFFFFF06
:107A9000FFFFFFF1FE7FFF9FF3FFFFFFFFFFFFFFF1
:107AA000FFFFFFFFFFFFFFFFFFFFFFFFFFFFFFFFE6
:107AB000FFFFFFFFFFFFFFFFFFFFFFFFFFFFFFFFD6
:107AC000FFFFFFFFFFF0FF7FFF9FE7FFFFFFFFFFCD
:107AD000FFFFFFFFFFFFFFFFFFFFFFFFFFFFFFFFB6
:107AE000FFFFFFFFFFFFFFFFFFFFFFFFFFFFFFFFA6
:107AF000FFFFFFFFFFFFFFF83FFFFF8FE7FFFFFFE5
:107B0000FFFFFFFFFFFFFFFFFFFFFFFFFFFFFFFF85
:107B1000FFFFFFFFFFFFFFFFFFFFFFFFFFFFFFFF75
:107B2000FFFFFFFFFFFFFFFFFFF90F800F8FCFFF6A
:107B3000FFFFFFFFFFFFFFFFFFFFFFFFFFFFFFFF55
:107B4000FFFFFFFFFFFFFFFFFFFFFFFFFFFFFFFF45
:107B5000FFFFFFFFFFFFFFFFFFFFFFFCC0000187EC
:107B6000CFFFFFFFFFFFFFFFFFFFFFFFFFFFFFFF55
:107B7000FFFFFFFFFFFFFFFFFFFFFFFFFFFFFFFF15
:107B8000FFFFFFFFFFFFFFFFFFFFFFFFFFFCF87F8F
:107B9000E0179FFFFFFFFFFFFFFFFFFFFFFFFFFF5C
:107BA000FFFFFFFFFFFFFFFFFFFFFFFFFFFFFFFFE5
:107BB000FFFFFFFFFFFFFFFFFFFFFFFFFFFFFFFCD8
:107BC000FFFFFC123FFFFFFFFFFFFFFFFFFFFFFF75
:107BD000FFFFFFFFFFFFFFFFFFFFFFFFFFFFFFFFB5
:107BE000FFFFFFFFFFFFFFFFFFFFFFFFFFFFFFFFA5
:107BF000FFFE7FFFFF007FFFFFFFFFFFFFFFFFFF95
:107C0000FFFFFFFFFFFFFFFFFFFFFFFFFFFFFFFF84
:107C1000FFFFFFFFFFFFFFFFFFFFFFFFFFFFFFFF74
:107C2000FFFFFFFE7FFFFF81FFFFFFFFFFFFFFFF63
:107C3000FFFFFFFFFFFFFFFFFFFFFFFFFFFFFFFF54
:107C4000FFFFFFFFFFFFFFFFFFFFFFFFFFFFFFFF44
:107C5000FFFFFFFFFFFF1FFFFFFFFFFFFFFFFFFF14
:107C6000FFFFFFFFFFFFFFFFFFFFFFFFFFFFFFFF24
:107C7000FFFFFFFFFFFFFFFFFFFFFFFFFFFFFFFF14
:107C8000FFFFFFFFFFFFFFFF87FFFFFFFFFFFFFF7C
:107C9000FFFFFFFFFFFFFFFFFFFFFFFFFFFFFFFFF4
:107CA000FFFFFFFFFFFFFFFFFFFFFFFFFFFFFFFFE4
:107CB000FFFFFFFFFFFFFFFFFFFFC3FFFFFFFFFF10
:107CC000FFFFFFFFFFFFFFFFFFFFFFFFFFFFFFFFC4
:107CD000FFFFFFFFFFFFFFFFFFFFFFFFFFFFFFFFB4
:107CE000FFFFFFFFFFFFFFFFFFFFFFFFF0FFFFFFB3
:107CF000FFFFFFFFFFFFFFFFFFFFFFFFFFFFFFFF94
:107D0000FFFFFFFFFFFFFFFFFFFFFFFFFFFFFFFF83
:107D1000FFFFFFFFFFFFFFFFFFFFFFFFFFFFFC7FF6
:107D2000FFFFFFFFFFFFFFFFFFFFFFFFFFFFFFFF63
:107D3000FFFFFFFFFFFFFFFFFFFFFFFFFFFFFFFF53
:107D4000FFFFFFFFFFFFFFFFFFFFFFFFFFFFFFFF43
:107D5000FE7FFFFFFFFFFFFFFFFFFFFFFFFFFFFFB4
:107D6000FFFFFFFFFFFFFFFFFFFFFFFFFFFFFFFF23
:107D7000FFFFFFFFFFFFFFFFFFFFFFFFFFFFFFFF13
:107D8000FFFFFF3FFFFFFFFF1FFFFFFFFFFFFFFFA3
:107D9000FFFFFFFFFFFFFFFFFFFFFFFFFFFFFFFFF3
:107DA000FFFFFFFFFFFFFFFFFFFFFFFFFFFFFFFFE3
:107DB000FFFFFFFFFF3FFFFFFFFC0FFFFFFFFFFF86
:107DC000FFFFFFFFFFFFFFFFFFFFFFFFFFFFFFFFC3
:107DD000FFFFFFFFFFFFFFFFFFFFFFFFFFFFFFFFB3
:107DE000FFFFFFFFFFFFFFBFFFFFFFF807FFFFFFE2
:107DF000FFFFFFFFFFFFFFFFFFFFFFFFFFFFFFFF93
:107E0000FFFFFFFFFFFFFFFFFFFFFFFFFFFFFFFF82
:107E1000FFFFFFFFFFFFFFFFFF9FFFFFFFF9C3FF14
:107E2000FFFFFFFFFFFFFFFFFFFFFFFFFFFFFFFF62
:107E3000FFFFFFFFFFFFFFFFFFFFFFFFFFFFFFFF52
:107E4000FFFFFFFFFFFFFFFFFFFFFF9FFFFFFFF3AE
:107E5000E3FFFFFFFFFFFFFFFFFFFFFFFFFFFFFF4E
:107E6000FFFFFFFFFFFFFFFFFFFFFFFFFFFFFFFF22
:107E7000FFFFFFFFFFFFFFFFFFFFFFFFFFDFFFFF32
:107E8000FFF3E3FFFFFFFFFFFFFFFFFFFFFFFFFF2A
:107E9000FFFFFFFFFFFFFFFFFFFFFFFFFFFFFFFFF2
:107EA000FFFFFFFFFFFFFFFFFFFFFFFFFFFFFFDF02
:107EB000FFFFFFE473FFFFFFFFFFFFFFFFFFFFFF79
:107EC000FFFFFFFFFFFFFFFFFFFFFFFFFFFFFFFFC2
:107ED000FFFFFFFFFFFFFFFFFFFFFFFFFFFFFFFFB2
:107EE000FFDFFFFFFFE033FFFFFFFFFFFFFFFFFFAD
:107EF000FFFFFFFFFFFFFFFFFFFFFFFFFFFFFFFF92
:107F0000FFFFFFFFFFFFFFFFFFFFFFFFFFFFFFFF81
:107F1000FFFFFFDFFFFFFFC013FFFFFFFFFFFFFFBC
:107F2000FFFFFFFFFFFFFFFFFFFFFFFFFFFFFFFF61
:107F3000FFFFFFFFFFFFFFFFFFFFFFFFFFFFFFFF51
:107F4000FFFFFFFFFFCFFFFFFF8703FFFFFFFFFFE5
:107F5000FFFFFFFFFFFFFFFFFFFFFFFFFFFFFFFF31
:107F6000FFFFFFFFFFFFFFFFFFFFFFFFFFFFFFFF21
:107F7000FFFFFFFFFFFFFFEFFFFFFF1F83FFFFFF7D
:107F8000FFFFFFFFFFFFFFFFFFFFFFFFFFFFFFFF01
:107F9000FFFFFFFFFFFFFFFFFFFFFFFFFFFFFFFFF1
:107FA000FFFFFFFFFFFFFFFFFFE7FFFFFE3FC3FFF6
:107FB000FFFFFFFFFFFFFFFFFFFFFFFFFFFFFFFFD1
:107FC000FFFFFFFFFFFFFFFFFFFFFFFFFFFFFFFFC1
:107FD000FFFFFFFFFFFFFFFFFFFFFFF7FFFFFC7F3C
:107FE000C7FFFFFFFFFFFFFFFFFFFFFFFFFFFFFFD9
:107FF000FFFFFFFFFFFFFFFFFFFFFFFFFFFFFFFF91
:10800000FFFFFFFFFFFFFFFFFFFFFFFFFFFBFFFF84
:10801000F9FFE7FFFFFFFFFFFFFFFFFFFFFFFFFF8E
:10802000FFFFFFFFFFFFFFFFFFFFFFFFFFFFFFFF60
:10803000FFFFFFFFFFFFFFFFFFFFFFFFFFFFFFF956
:10804000FFFFE3FFE3FFFFFFFFFFFFFFFFFFFFFF78
:10805000FFFFFFFFFFFFFFFFFFFFFFFFFFFFFFFF30
:10806000FFFFFFFFFFFFFFFFFFFFFFFFFFFFFFFF20
:10807000FFFE7FFFCFFFE3FFFFFFFFFFFFFFFFFFDD
:10808000FFFFFFFFFFFFFFFFFFFFFFFFFFFFFFFF00
:10809000FFFFFFFFFFFFFFFFFFFFFFFFFFFFFFFFF0
:1080A000FFFFFFFF1FFF1FFFF3FFFFFFFFFFFFFFAC
:1080B000FFFFFFFFFFFFFFFFFFFFFFFFFFFFFFFFD0
:1080C000FFFFFFFFFFFFFFFFFFFFFFFFFFFFFFFFC0
:1080D000FFFFFFFFFFFFC7FC7FFFF3FFFFFFFFFF77
:1080E000FFFFFFFFFFFFFFFFFFFFFFFFFFFFFFFFA0
:1080F000FFFFFFFFFFFFFFFFFFFFFFFFFFFFFFFF90
:10810000FFFFFFFFFFFFFFFFF021FFFFF3FFFFFF78
:10811000FFFFFFFFFFFFFFFFFFFFFFFFFFFFFFFF6F
:10812000FFFFFFFFFFFFFFFFFFFFFFFFFFFFFFFF5F
:10813000FFFFFFFFFFFFFFFFFFFFFFFFFFFFF9FF55
:10814000FFFFFFFFFFFFFFFFFFFFFFFFFFFFFFFF3F
:10815000FFFFFFFFFFFFFFFFFFFFFFFFFFFFFFFF2F
:10816000FFFFFFFFFFFFFFFFFFFFFFFFFFFFFFFF1F
:10817000FDFFFFFFFFFFFFFFFFFFFFFFFFFFFFFF11
:10818000FFFFFFFFFFFFFFFFFFFFFFFFFFFFFFFFFF
:10819000FFFFFFFFFFFFFFFFFFFFFFFFFFFFFFFFEF
:1081A000FFFFFEFFFFFFFFFFFFFFFFFFFFFFFFFFE0
:1081B000FFFFFFFFFFFFFFFFFFFFFFFFFFFFFFFFCF
:1081C000FFFFFFFFFFFFFFFFFFFFFFFFFFFFFFFFBF
:1081D000FFFFFFFFFE3FFFFFFFFFFFFFFFFFFFFF70
:1081E000FFFFFFFFFFFFFFFFFFFFFFFFFFFFFFFF9F
:1081F000FFFFFFFFFFFFFFFFFFFFFFFFFFFFFFFF8F
:10820000FFFFFFFFFFFFFF87FFFFFFFFFFFFFFFFF6
:10821000FFFFFFFFFFFFFFFFFFFFFFFFFFFFFFFF6E
:10822000FFFFFFFFFFFFFFFFFFFFFFFFFFFFFFFF5E
:10823000FFFFFFFFFFFFFFFFFFF9E1FFFFFFFFFF72
:10824000FFFFFFFFFFFFFFFFFFFFFFFFFFFFFFFF3E
:10825000FFFFFFFFFFFFFFFFFFFFFFFFFFFFFFFF2E
:10826000FFFFFFFFFFFFFFFFFFFFFFFFE1FFFFFF3C
:10827000FFFFFFFFFFFFFFFFFFFFFFFFFFFFFFFF0E
:10828000FFFFFFFFFFFFFFFFFFFFFFFFFFFFFFFFFE
:10829000FFFFFFFFFFFFFFFFFFFFFFFFFFFFFFFFEE
:1082A000FFFFFFFFFFFFFFFFFFFFFFFFFFFFFFFFDE
:1086D000000000000000000000000003FFFFFFFF9B
:1086E000000000000000000000000000000000008A
:1086F000000000000000000000000000000000007A
:108700000000000000000000000000000007FFFF64
:10871000FFFFF80000000000000000000000000063
:108720000000000000000000000000000000000049
:108730000000000000000000000000000000000732
:10874000FFFFFFFFFF00000000000000000000002E
:108750000000000000000000000000000000000019
:108760000000000000000000000000000000000009
:108770000007FFFFFFFFFFE0000000000000000017
:1087800000000000000000000000000000000000E9
:1087900000000000000000000000000000000000D9
:1087A00000000007FFFFFFFFFFF0000000000000D7
:1087B00000000000000000000000000000000000B9
:1087C00000000000000000000000000000000000A9
:1087D000000000000007FFFFFFFFFFFC000000009B
:1087E0000000000000000000000000000000000089
:1087F0000000000000000000000000000000000079
:108800000000000000000007FFFFFFFFFFFF000067
:108810000F0001E00078007FFE007C000007CFFF22
:10882000FFFF807FFFFE1E00001E003FFF000FFFC6
:10883000FFE01FFFFFFF00000007FFFFFFFFFFFF3C
:1088400080000F0001E0007803FFFF803E00000F72
:108850008FFFFFFF81FFFFFE1E00001E00FFFFC015
:108860000FFFFFF81FFFFFFF00000007FFFFFFFFE4
:10887000FFFFC0000F0001E0007807FFFFE03E00AF
:10888000000F8FFFFFFF83FFFFFE1E00001E03FF90
:10889000FFF00FFFFFFC1FFFFFFF00000007FFFFBF
:1088A000FFFFF9FFE0000F0001E000780FFFFFF08D
:1088B0001F00001F0FFFFFFF87FFFFFE1E00001EAF
:1088C00007FFFFF80FFFFFFE1FFFFFFF000000077D
:1088D000FFFFFFFFF1FFF0000F0001E000781FFF36
:1088E000FFF81F00001F0FFFFFFF87FFFFFE1E00A6
:1088F000001E0FFFFFFC0FFFFFFF1FFFFFFF000029
:108900000007FFFFFFFFE1FFF8000F0001E0007824
:108910001FF00FF80F80003E0F80000007F00000EE
:108920001E00001E0FF807FC0F0001FF1F000000D3
:1089300000000007FFFFFFFFC1FFFC000F0001E088
:1089400000783F8001FC0F80003E0F000000078090
:1089500000001E00001E1FC000FE0F00001F1E00B2
:10896000000000000007FFFFFFFF81FFFC000F0079
:1089700001E000783F00007C07C0007C0F00000091
:10898000078000001E00001E1F80003E0F00000F29
:108990001E00000000000007FFFFFFFF01FFFE00B8
:1089A0000F0001E000783E00007C03C0007C0F0057
:1089B0000000078000001E00001E1F00003E0F0088
:1089C000000F1E00000000000007FFFFFFFE01FF78
:1089D000FF000F0001E000783C00003C03E000F8DD
:1089E0000F80000007C000001F00001E1E00001EB8
:1089F0000F00000F1F00000000000007FFFFFFFC3A
:108A000001FFFF000F0001E000783C00003C01F096
:108A100000F80FFFFFF007FFFFF01FFFFFFE1E0033
:108A2000001E0F00000F1FFFFFE000000007FFFF08
:108A3000FFFC01FFFF800F0001E000783C00003CDC
:108A400001F001F00FFFFFF007FFFFFC1FFFFFFE2B
:108A50001E00001E0F00000F1FFFFFE000000007B8
:108A6000FFFFFFF801FFFF800F0001E000783C00EE
:108A7000003C00F801F00FFFFFF007FFFFFE1FFFB3
:108A8000FFFE1E00001E0F00000F1FFFFFE0000092
:108A90000007FFFFFFF801FFFFC00F0001E00078B3
:108AA0003C00003C00F803E00FFFFFF001FFFFFE79
:108AB0001FFFFFFE1E00001E0F00001F1FFFFFE034
:108AC00000000007C01F01FC01E0FFC00F0001E033
:108AD00000783C00003C007C03C00FFFFFF0007FEB
:108AE000FFFF1FFFFFFE1E00001E0FFFFFFF1FFF07
:108AF000FFE000000007C01F01F801C07FC00F00A9
:108B000001E000783FFFFFFC007C07C00F00000081
:108B10000000003F1E00001E1FFFFFFE0FFFFFFFB3
:108B20001F00000000000007C01F01F801C07FE027
:108B30000F0001E000783FFFFFFC003E07800F00C0
:108B400000000000001F1E00001E1FFFFFFE0FFFA1
:108B5000FFFE1E00000000000007C01E00F807C056
:108B60003FE00F0001E000783FFFFFFC003E0F8078
:108B70000F0000000000000F1E00001E1FFFFFFE80
:108B80000FFFFFFC1E00000000000007C00E00F0F9
:108B90000F803FE00F0001E000783FFFFFFC001F67
:108BA0000F000F0000000000000F1E00001E1FFF3E
:108BB000FFFE0FFFFFF81E00000000000007E00EA0
:108BC00000F00F801FF00F0001E000783FFFFFFC76
:108BD000001F1F000F0000000000000F1E00001EFD
:108BE0001FFFFFFE0FFFF7C01E0000000000000780
:108BF000E00400600F001FF00F0001E000783C006F
:108C0000007C000FBE000F0000000000000F1E00DF
:108C1000001E1F00001E0F0FF0001E0000000000CD
:108C20000007E00400601F000FF00F0001E0007873
:108C30003C00003C000FBE000F0000000000000FD1
:108C40001E00001E1E00001E0F07F8001E00000080
:108C500000000007F00400401E000FF00F0001E0CC
:108C600000783C00003C0007FC000F000000000002
:108C7000000F1E00001E1E00001E0F01FE001E0041
:108C8000000000000007F00000000E0007F00F8059
:108C900001E000F83C00003C0007FC000F00000071
:108CA0000000001F1E00001E1E00001E0F00FF001F
:108CB0001E00000000000007F00000000C0007F09C
:108CC0000FF003E00FF83C00003C0003F8000F80B9
:108CD0000000000001FF1E00001E1E00001E0F000D
:108CE0003FC01F00000000000007F8000000040063
:108CF00003F00FFFFFFFFFF83C00003C0003F8000B
:108D00000FFFFFFF8FFFFFFF1E00001E1E00001E53
:108D10000F001FE01FFFFFFF00000007F80000002A
:108D2000040003F00FFFFFFFFFF83C00003C0001D0
:108D3000F0000FFFFFFF87FFFFFE1E00001E1E005A
:108D4000001E0F0007F01FFFFFFF00000007F800E4
:108D50000000000001F007FFFFFFFFF03C00003CB7
:108D60000001F0000FFFFFFF87FFFFFC1E00001E49
:108D70001E00001E0F0003FC1FFFFFFF000000038A
:108D8000FC000000000401F001FFFFFFFFE03C00D9
:108D9000003C0000E0000FFFFFFF87FFFFF81E0010
:108DA000001E1E00001E0F0001FE1FFFFFFF00003F
:108DB0000003FC002000000600F0003FFFFFFF0062
:108DC0003C00003C0000C0000FFFFFFF87FFFFC01A
:108DD0001E00001E1E00001E0F00007F9FFFFFFFF1
:108DE00000000003FC003000000E00F00000000056
:108DF0000000000000000000000000000000000073
:108E00000000000000000000000000000000000062
:108E1000000000000003FE003000000F00F0000022
:108E20000000000000000000000000000000000042
:108E30000000000000000000000000000000000032
:108E40000000000000000003FE007001000F00F0B1
:108E50000000000000000000000000000000000012
:108E60000000000000000000000000000000000002
:108E700000000000000000000003FE007803001E58
:108E800000F00000000000000000000000000000F2
:108E900000000000000000000000000000000000D2
:108EA000000000000000000000000001FF00780347
:108EB000801E01F000000000000000000000000023
:108EC00000000000000000000000000000000000A2
:108ED0000000000000000000000000000001FF0092
:108EE000F803803E01F000000000000000000000D8
:108EF0000000000000000000000000000000000072
:108F00000000000000000000000000000000000160
:108F1000FF00FC07803C03F00000000000000000A0
:108F20000000000000000000000000000000000041
:108F30000000000000000000000000000000000031
:108F40000000FF80FC07C07C03F00004000000006C
:108F50000000000000000000000000000000000011
:108F600000002000000000001000000000000000D1
:108F700000000000FF81FC0FC07807F00004000033
:108F800000000000000000000000000000000000E1
:108F900000000000200000000000100000000000A1
:108FA0000000000000007F81FE0FFFE007F00004DA
:108FB00000000000000000000000000000000000B1
:108FC0000000000000002000000000001000000071
:108FD00000000000000000007FFFFFFFFFE00FF037
:108FE000000400000000000000000000000000007D
:108FF0000000000000000000200000000000100041
:10900000000000000000000000003FFFFFFFFFE045
:109010001FF00F047801E21303E0000F8880004086
:10902000F807807C04783801F00023C00F10981FE7
:1090300010000081F10183E0000000003FFFFFFF0E
:10904000FFE00FF019858C061A140C300018C88048
:1090500080438E0CC1C6048CC60618002C6030D02C
:10906000A07191010087191E0618000000001FFF63
:10907000FFFFFFE00FF01006060C0618180800208E
:109080003880C082020803010707020C0400303058
:109090006070C0C071018104071C080C0000000052
:1090A0000FFFFFFFFFE01FF0100602180618100464
:1090B00000401841C0840108020086030208020033
:1090C0003010C030808030838108031818040000FD
:1090D00000000FFFFFFFFFE03FF01004021002103E
:1090E000300400C01841618401880600860203181C
:1090F00002002010801081803082C21803181002F4
:109100000000000007FFFFFFFFE07FF00C040210EB
:1091100002103FFE00800821210FFF860400C402D8
:10912000031FFE0020108010810010C6421001189D
:109130001FFE0000000003FFFFFFFFE0FFF006043A
:1091400002100210300000800822330C00030400DB
:10915000C402031800002010801081001044461043
:10916000011810000000000001FFFFFFFFE1FFF009
:109170000184021002102000008008321208000052
:10918000C400C402031000002010801081001044AD
:109190002410011810000000000000FFFFFFFFE393
:1091A000FFF0008402100210300000C018141204F6
:1091B0000000440084020310000020108010818011
:1091C000302824180318100000000000007FFFFF63
:1091D000FFFFFFF000840218061010040040181C66
:1091E0000C04010042008402030802002010C03079
:1091F0008080303818080318180400000000001F91
:10920000FFFFFFFFFFF00084020C0610180800208B
:10921000380C0C02030043010402030C040020106C
:10922000603080C07010180C0718080C0000000097
:10923000000FFFFFFFFFFFF0318402061A100C3011
:109240000038C8080C038E18C186040203061800F3
:10925000201030D0807190101007191806180000E7
:1092600000000003FFFFFFFFFFF00E040201E21009
:1092700003E0000F88000000F807007C04020001F2
:10928000F00020100F10801F10000001F10003E01B
:10929000000000000000FFFFFFFFFFF000000000E3
:1092A00000000000000000000000000000000000BE
:1092B00000000000000000000000000000000000AE
:1092C00000000000000000003FFFFFFFFFF0000073
:1092D000000000000000000000000000000000008E
:1092E000000000000000000000000000000000007E
:1092F0000000000000000000000003FFFFFFFFF07F
:10930000000000000000000000000000000000005D
:10931000000000000000000000000000000000004D
:10932000000000000000000000000000000000003D
:10933000000000000000000000000000000000002D
:1095E00000000000FFFFFFFFFFFFFFFFFFFFFFFF87
:1095F000FFFFFFFFFFFFFFFFFFFFFFFFFFFFFFFF7B
:10960000000FFFFFFFFFFFFFFFFFFFFFFFFFFFFF59
:10961000FFFFFFFFFFFFFFFFFFFFFFFFFFFFFFFF5A
:10962000FFFFFFFFFFFFFFFFC003FFFFFFFFFFFF85
:10963000FFFFFFFFFFFFFFFFFFFFFFFFFFFFFFFF3A
:10964000FFFFFFFFFFFFFFFFFFFFFFFFFFFFFFFF2A
:10965000FFFFFFFFFFFFFFFFFFFFFFFFFFFFFFFF1A
:10966000FFFFFFFF000FFFFFFFFFFFFFFFFFFFFFF9
:10967000FFFFFFFFFFFFFFFFFFFFFFFFFFFFFFFFFA
:10968000FFFFFFFFFFFFFFFFFFFFFFFFC003FFFF25
:10969000FFFFFFFFFFFFFFFFFFFFFFFFFFFFFFFFDA
:1096A000FFFFFFFFFFFFFFFFFFFFFFFFFFFFFFFFCA
:1096B000FFFFFFFFFFFFFFFFFFFFFFFFFFFFFFFFBA
:1096C000FFFFFFFFFFFFFFFF000FFFFFFFFFFFFF99
:1096D000FFFFFFFFFFFFFFFFFFFFFFFFFFFFFFFF9A
:1096E000FFFFFFFFFFFF00000003FFFFFFFFFFFF83
:1096F000C003FFFFFFFFFFFFFFFFFFFFFFFFFFFFB5
:10970000FFFFFFFFFFFFFFFFFFFFFFFFFFFFFFFF69
:10971000FFFFFFFFFFFFFFFFFFFFFFFFFFFFFFFF59
:10972000FFFFFFFFFFFFFFFFFFFFFFFF000FFFFF38
:10973000FFFFFFFFFFFFFFFFFFFFFFFFFFFFFFFF39
:10974000FFFFFFFFFFFFFFFFFC00000000000FFF17
:10975000FFFFFFFFC003FFFFFFFFFFFFFFFFFFFF54
:10976000FFFFFFFFFFFFFFFFFFFFFFFFFFFFFFFF09
:10977000FFFFFFFFFFFFFFFFFFFFFFFFFFFFFFFFF9
:10978000FFFFFFFFFFFFFFFFFFFFFFFFFFFFFFFFE9
:10979000000FFFFFFFFFFFFFFFFFFFFFFFFFFFFFC8
:1097A000FFFFFFFFFFFFFFFFFFFFFFFFFC000000C9
:1097B00000000FFFFFFFFFFFC003FFFFFFFFFFFFE2
:1097C000FFFFFFFFFFFFFFFFFFFFFFFFFFFFFFFFA9
:1097D000FFFFFFFFFFFFFFFFFFFFFFFFFFFFFFFF99
:1097E000FFFFFFFFFFFFFFFFFFFFFFFFFFFFFFFF89
:1097F000FFFFFFFF000FFFFFFFFFFFFFFFFFFFFF68
:10980000FFFFFFFFFFFFFFFFFFFFFFFFFFFFFFFF68
:10981000000000000000003FFFFFFFFFC003FFFF4C
:10982000FFFFFFFFFFFFFFFFFFFFFFFFFFFFFFFF48
:10983000FFFFFFFFFFFFFFFFFFFFFFFFFFFFFFFF38
:10984000FFFFFFFFFFFFFFFFFFFFFFFFFFFFFFFF28
:10985000FFFFFFFFFFFFFFFF000FFFFFFFFFFFFF07
:10986000FFFFFFFFFFFFFFFFFFFFFFFFFFFFFFFF08
:10987000FFFFFFFF000000000000003FFFFFFFFFB1
:10988000C003FFFFFFFFFFFFFFFFFFFFFFFFFFFF23
:10989000FFFFFFFFFFFFFFFFFFFFFFFFFFFFFFFFD8
:1098A000FFFFFFFFFFFFFFFFFFFFFFFFFFFFFFFFC8
:1098B000FFFFFFFFFFFFFFFFFFFFFFFF000FFFFFA7
:1098C000FFFFFFFFFFFFFFFFFFFFFFFFFFFFFFFFA8
:1098D000FFFFFFFFFFFFFFFC000000000000000390
:1098E000FFFFFFFFC003FFFFFFFFFFFFFFFFFFFFC3
:1098F000FFFFFFFFFFFFFFFFFFFFFFFFFFFFFFFF78
:10990000FFFFFFFFFFFFFFFFFFFFFFFFFFFFFFFF67
:10991000FFFFFFFFFFFFFFFFFFFFFFFFFFFFFFFF57
:10992000000FFFFFFFFFFFFFFFFFFFFFFFFFFFFF36
:10993000FFFFFFFFFFFFFFFFFFFFFFFC0000000036
:1099400000000003FFFFFFFFC003FFFFFFFFFFFF5B
:10995000FFFFFFFFFFFFFFFFFFFFFFFFFFFFFFFF17
:10996000FFFFFFFFFFFFFFFFFFFFFFFFFFFFFFFF07
:10997000FFFFFFFFFFFFFFFFFFFFFFFFFFFFFFFFF7
:10998000FFFFFFFF000FFFFFFFFFFFFFFFFFFFFFD6
:10999000FFFFFFFFFFFFFFFFFFFFFFFFFFFFFFC016
:1099A0000000000000000000FFFFFFFFC003FFFFFA
:1099B000FFFFFFFFFFFFFFFFFFFFFFFFFFFFFFFFB7
:1099C000FFFFFFFFFFFFFFFFFFFFFFFFFFFFFFFFA7
:1099D000FFFFFFFFFFFFFFFFFFFFFFFFFFFFFFFF97
:1099E000FFFFFFFFFFFFFFFF000FFFFFFFFFFFFF76
:1099F000FFFFFFFFFFFFFFFFFFFFFFFFFFFFFFFF77
:109A0000FFFFFF0000000000000000000FFFFFFF4D
:109A1000C003FFFFFFFFFFFFFFFFFFFFFFFFFFFF91
:109A2000FFFFFFFFFFFFFFFFFFFFFFFFFFFFFFFF46
:109A3000FFFFFFFFFFFFFFFFFFFFFFFFFFFFFFFF36
:109A4000FFFFFFFFFFFFFFFFFFFFFFFF000FFFFF15
:109A5000FFFFFFFFFFFFFFFFFFFFFFFFFFFFFFFF16
:109A6000FFFFFFFFFFFFFF000000000000000000FD
:109A70000FFFFFFFC003FFFFFFFFFFFFFFFFFFFF21
:109A8000FFFFFFFFFFFFFFFFFFFFFFFFFFFFFFFFE6
:109A9000FFFFFFFFFFFFFFFFFFFFFFFFFFFFFFFFD6
:109AA000FFFFFFFFFFFFFFFFFFFFFFFFFFFFFFFFC6
:109AB000000FFFFFFFFFFFFFFFFFFFFFFFFFFFFFA5
:109AC000FFFFFFFFFFFFFFFFFFFFF00000000000B0
:109AD0000000000003FFFFFFC003FFFFFFFFFFFFC9
:109AE000FFFFFFFFFFFFFFFFFFFFFFFFFFFFFFFF86
:109AF000FFFFFFFFFFFFFFFFFFFFFFFFFFFFFFFF76
:109B0000FFFFFFFFFFFFFFFFFFFFFFFFFFFFFFFF65
:109B1000FFFFFFFF000FFFFFFFFFFFFFFFFFFFFF44
:109B2000FFFFFFFFFFFFFFFFFFFFFFFFFFFFF00053
:109B3000000000000000000003FFFFFFC003FFFF64
:109B4000FFFFFFFFFFFFFFFFFFFFFFFFFFFFFFFF25
:109B5000FFFFFFFFFFFFFFFFFFFFFFFFFFFFFFF024
:109B600000000000000000000000000003FFFFFFF5
:109B7000FFFFFFFFFFFFFFFF000FFFFFFFFFFFFFE4
:109B8000FFFFFFFFFFFFFFFFFFFFFFFFFFFFFFFFE5
:109B9000FFFFC0000000000000000000003FFFFFCA
:109BA000C003FFFFFFFFFFFFFFFFFFFFFFFFFFFF00
:109BB000FFFFFFFFFFFFFFFFFFFFFFFFFFFFFFFFB5
:109BC000FFFFFFF0000000000000000000000000A8
:109BD0000003FFFFFFFFFFFFFFFFFFFF000FFFFF7F
:109BE000FFFFFC000000000000000000000000007B
:109BF00000000000000000000FFF00000000FFFF59
:109C0000003FFFFFC003FFFFFFFFFFFFFFFFFFFF5E
:109C1000FFFFFFFFFFFFFFFFFFFFFFFFFFFFFFFF54
:109C2000FFFFFFFFFFFFFFF000000000000000004B
:109C3000000000000003FFFFFFFFFFFFFFFFFFFF2B
:109C4000000FFFFFFFFFFC0000000000000000000D
:109C50000000000000000000000000000FFF0000F6
:109C60000000FFFF003FFFFFC003FFFFFFFFFFFFFC
:109C7000FFFFFFFFFFFFFFFFFFFFFFFFFFFFFFFFF4
:109C8000FFFFFFFFFFFFFFFFFFFFFFF000000000EF
:109C9000000000000000000000000FFFFFFFFFFFBA
:109CA000FFFFFFFF000FFFFFFFFFFC0000000000B1
:109CB00000000000000000000000000000000003A1
:109CC000FFFFFC00003FFFFFFC0FFFFFC003FFFF93
:109CD000FFFFFFFFFFFFFFFFFFFFFFFFFFFFFFFF94
:109CE000FFFFFFFFFFFFFFFFFFFFFFFFFFFFFFF093
:109CF00000000000000000000000000000000FFF56
:109D0000FFFFFFFFFFFFFFFF000FFFFFFFFFFC0054
:109D10000000000000000000000000000000000043
:109D200000000003FFFFFC00003FFFFFFC0FFFFFF0
:109D3000C003FFFFFFFFFFFFFFFFFFFFFFFFFFFF6E
:109D4000FFFFFFFFFFFFFFFFFFFFFFFFFFFFFFFF23
:109D5000FFFFFFF000000000000000000000000016
:109D60000000003FFFFFFFFFFFFFFFFF000FFFFFAF
:109D7000FFFFFC00000000000000000000000000E9
:109D8000000000000000003FF000FF0000FFF003B3
:109D9000FC0FFFFFC003FFFFFFFFFFFFFFFFFFFF01
:109DA000FFFFFFFFFFFFFFFFFFFFFFFFFFFFFFFFC3
:109DB000FFFFFFFFFFFFFFF00000000000000000BA
:109DC0000000000000000000FFFFFFFFFFFFFFFF9B
:109DD000000FFFFFFFFFFC0000000000000000007C
:109DE0000000000000000000000000FF00003F0035
:109DF00000FC0000FFC0FFFFC003FFFFFFFFFFFFED
:109E0000FFFFFFFFFFFFFFFFFFFFFFFFFFFFFFFF62
:109E1000FFFFFFFFFFFFFFFFFFFFFFF0000000005D
:109E2000000000000000000000000000FFFFFFFF36
:109E3000FFFFFFFF000FFFFFFFFFFC00000000001F
:109E4000000000000000000000000000000000FF13
:109E500000003F0000FC0000FFC0FFFFC003FFFF49
:109E6000FFFFFFFFFFFFFFFFFFFFFFFFFFFFFFFF02
:109E7000FFFFFFFFFFFFFFFFFFFFFFFFFFFFFFF001
:109E800000000000000000000000000000000000D2
:109E90000FFFFFFFFFFFFFFF000FFFFFFFFFFC00B3
:109EA00000000000000000000000000000000000B2
:109EB000000000FC00003FF000FC00000FC03FFF6E
:109EC000C003FFFFFFFFFFFFFFFFFFFFFFFFFFFFDD
:109ED000FFFFFFFFFFFFFFFFFFFFFFFFFFFFFFFF92
:109EE000FFFFFFF000000000000000000000000085
:109EF000000000000FFFFFFFFFFFFFFF000FFFFF4D
:109F0000FFFFFC0000000000000000000000000057
:109F100000000000000000FC00003FF000FC00001A
:109F20000FC03FFFC003FFFFFFFFFFFFFFFFFFFF6B
:109F3000FFFFFFFFFFFFFFFFFFFFFFFFFFFFFFFF31
:109F4000FFFFFFFFFFFFFFF0000000000000000028
:109F5000000000000000000003FFFFFFFFFFFFFF05
:109F6000000FFFFFFFFFFC000000000000000000EA
:109F70000000000000000000000000FC000003F0F2
:109F80000FFC00000FC03FFFC003FFFFFFFFFFFFFC
:109F9000FFFFFFF03FFFFFFFFFFFFFFFFFFFFFFFA0
:109FA000FFFFFFFFFFFFFFFFFFFFFFF000000000CC
:109FB00000000000000000000000000003FFFFFFA1
:109FC000FFFFFFFF000FFFFFFFFFFC00000000008E
:109FD000000000000000000000000000000000FC85
:109FE000000003F00FFC00000FC03FFFC003FFFFA5
:109FF000FFFFFFFFFFFFFFF03FFFFFFFFFFFFFFF40
:10A00000FFFFFFFFFFFFFFFFFFFFFFFFFFFFFFF06F
:10A010000000000000000000000000000000000040
:10A02000003FFFFFFFFFFFFF000FFFFFFFFFFC00F0
:10A03000000002AAAAAAAAAAAAAAAAAAAAAAAAAA7C
:10A04000AAA000FC000003F00FFC00000FF03FFF8F
:10A05000C003FFFFFFFFFFFFFFFFFFF03FFFFFFF1A
:10A06000FFFFFFFFFFFFFFFFFFFFFFFFFFFFFFFF00
:10A07000FFFFFFF0000000000000000000000000F3
:10A0800000000000000FFFFFFFFFFFFF000FFFFFBA
:10A09000FFFFFC00000000AAAAAAAAAAAAAAAAAACC
:10A0A000AAAAAAAAAAA000FF000003F000FC0000D0
:10A0B0000FF03FFFC003FFFFFFFFFFFFFFFFFFF0B9
:10A0C0003FFFF03FFFFFFFFFFFFFFFFFFFFFFFFF2F
:10A0D000FFFFFFFFFFFFFFF0000000000000000097
:10A0E0000000000000000000000FFFFFFFFFFFFF67
:10A0F000000FFFFFFFFFFC00000000AAAAAAAAAA07
:10A10000AAAAAAAAAAAAAAAAAAA000FF000003F0C3
:10A1100000FC00000FF03FFFC003FFFFFFFFFFFF49
:10A12000FFFFFFF03FFFF03FFFFFFFFFFFFFFFFFDD
:10A13000FFFFFFFFFFFFFFFFFFFFFFF0000000003A
:10A140000000000000000000000000000000FFFF11
:10A15000FFFFFFFF000FFFFFFFFFFC000000000AF2
:10A16000AAAAAAAAAAAAAAAAAAAAAAAAAAA0003F6E
:10A17000F0003FF000FF0000FFF03FFFC003FFFFD3
:10A18000FFFFFFFFF03FFFF03FFFC03FFFFFFFFF7C
:10A19000FFFFFFFFFFFFFFFFFFFFFFFFFFFFFFF0DE
:10A1A00000000000000000000000000000000000AF
:10A1B0000000FFFFFFFFFFFF000FFFFFFFFFFC009E
:10A1C0000000000AAAAAAAAAAAAAAAAAAAAAAAAA8D
:10A1D000AAA0003FF0003FF000FF0000FFF03FFFAB
:10A1E000C003FFFFFFFFFFFFF03FFFF03FFFC03F57
:10A1F000FFFFFFFFFFFFFFFFFFFFFFFFFFFFFFFF6F
:10A20000FFFFFFF000000000000000000000000061
:10A210000000000000003FFFFFFFFFFF000FFFFFF7
:10A22000FFFFFC0000000002AAAAAAAAAAAAAAAAE2
:10A23000AAAAAAAAAAA0003FFFFFFFF0003FFFFFC3
:10A24000FFF03FFFC003FFFFFFFFFFFFF003FFF042
:10A250003FFFC0FFFFFFFFFFFFFFFFFFFFFFFFFF0D
:10A26000FFFFFFFFFFFFFFF0000000000000000005
:10A27000000000003C00000000003FFFFFFFFFFF68
:10A28000000FFFFFFFFFFC00000000000AAAAAAABF
:10A29000AAAAAAAAAAAAAAAAAAA00000FFFF03F033
:10A2A0000003FFFF0FC03FFFC003FFFFFFFFFFFFE3
:10A2B000FF03FFF03FFC00FFFFFFFFFFFFFFFFFF7B
:10A2C000FFFFFFFFFFFFFFFFFFFFFFF000000000A9
:10A2D00000000000000000003C00000000003FFF04
:10A2E000FFFFFFFF000FFFFFFFFFFC00000000006B
:10A2F0000AAAAAAAAAAAAAAAAAAAAAAAAAA00000BC
:10A30000FFFF03F00003FFFF0FC03FFFC003FFFF8D
:10A31000FFFFFFFFFF03FFF03FFC00FFFFFFFFFF1A
:10A32000FFFFFFFFFFFFFFFFFFFFFFFFFFFFFFF04C
:10A33000000000000000000000000000FC00000021
:10A34000000003FFFFFFFFFF000FFFFFFFFFFC0008
:10A3500002A0000000AAAAAAAAAAAAAAAAAAAAAA0D
:10A36000AAA00000000003F0000000000FC03FFFA3
:10A37000C003FFFFFFFFFFFFFFC0FFF03FFC0FFF29
:10A38000FFFFFFFFFFFFFFFFFFFFFFFFFFFFFFFFDD
:10A39000FFFFFFF0000000000000000000000000D0
:10A3A000FC000000000003FFFFFFFFFF000FFFFFA6
:10A3B000FFFFFC0002A0000000AAAAAAAAAAAAAA5B
:10A3C000AAAAAAAAAAA00000000003F000000000A8
:10A3D0000FC03FFFC003FFFFFFFFFFFFFFC0FFF005
:10A3E0003FFC0FFFFFFFFFFFFFFFFFFFFFFFFFFF30
:10A3F000FFFFFFFFFFFFFFF0000000000000000074
:10A400000000000FFC000000000000FFFFFFFFFF46
:10A41000000FFFFFFFFFFC0002AA0000002AAAAA0B
:10A42000AAAAAAAAAAAAAAAAAAA0000000003FF063
:10A43000000000000FC03FFFC003FFFFFFFFFFFF52
:10A44000FFC00FF003FC0FFFFFCFFFFFFFFFFFFF79
:10A45000FFFFFFFFFFFFFFFFFFFFFFF00000000017
:10A46000000000000000000FFC000000000000FFE2
:10A47000FFFFFFFF000FFFFFFFFFFC0002AA00002D
:10A48000002AAAAAAAAAAAAAAAAAAAAAAAA00000B4
:10A4900000003FF0000000000FC03FFFC003FFFFBF
:10A4A000FFFFFFFFFFC00FF003FC0FFFFFCFFFFF19
:10A4B000FFFFFFFFFFFFFFFFFFFFFFFFFFFFFFF0BB
:10A4C00000000000000000000000003FFC00000051
:10A4D000000000FFFFFFFFFF000FFFFFFFFFFC007A
:10A4E00002AA80000002AAAAAAAAAAAAAAAAAAAA9A
:10A4F000AAA0000000003F0000000000FFC0FFFF16
:10A50000C003FFFFFFFFFFFFFFFC000000003FFF55
:10A51000F00FFFFFFFFFFFFFFFFFFFFFFFFFFFFF4A
:10A52000FFFFFFF00000000000000000000003FF3C
:10A53000FC0000000000000FFFFFFFFF000FFFFF07
:10A54000FFFFFC0002AAA8000000AAAAAAAAAAAAC1
:10A55000AAAAAAAAAAA800000000FF0000000003FF
:10A56000FC0FFFFFC003FFFFFFFFF0FFFFFC000039
:10A5700000000FFF003FFFFFFFFFFFFFFFFFFFFF98
:10A58000FFFFFFFFFFFFFFF00000000000000000E2
:10A59000000003FFFC0000000000000FFFFFFFFFB2
:10A5A000000FFFFFFFFFFC0002AAA8000000AAAAFC
:10A5B000AAAAAAAAAAAAAAAAAAA800000000FF00FA
:10A5C00000000003FC0FFFFFC003FFFFFFFFF0FFD1
:10A5D000FFFC000000000FFF003FFFFFFFFFFFFF39
:10A5E000FFFFFFFFFFFFFFFFFFFFFFF00000000086
:10A5F00000000000000003FFFC0000000000000F4E
:10A60000FFFFFFFF000FFFFFFFFFFC0002AAAAA051
:10A6100000000AAAAAAAAAAAAAAAAAAAAAA80000E4
:10A62000003FFC000000003FF00FFFFFC003FFFFF2
:10A63000FFFFF003FFFC0000000000FC03FFFFFF32
:10A64000FFFFFFFFFFFFFFFFFFFFFFFFFFFFFFF029
:10A650000000000000000000000003FFFC000000FC
:10A660000000000FFFFFFFFF000FFFFFFFFFFC00D8
:10A6700002AAAAA000000AAAAAAAAAAAAAAAAAAAE0
:10A68000AAA80000003FFC000000003FF00FFFFF01
:10A69000C003FFFFFFFFF003FFFC0000000000FC11
:10A6A00003FFFFFFFFFFFFFFFFFFFFFFFFFFFFFFB6
:10A6B000FFFFFFF00000000000000000000003FFAB
:10A6C000FC00000000000003FFFFFFFF000FFFFF82
:10A6D000FFFFFC0002AAAAA8000002AAAAAAAAAA2E
:10A6E000AAAAAAAAAAAA803FFFFFC000003FFFFFB4
:10A6F000000FFFFFC003FFFFFFFFFF000FC0003F81
:10A70000FF0000000FFF0000000FFFFFFFFFFFFF33
:10A71000FFFFFFFFFFFFFFF0000000000000000050
:10A72000000003FF0000000000000003FFFFFFFF28
:10A73000000FFFFFFFFFFC0002AAAAAA8000002A68
:10A74000AAAAAAAAAAAAAAAAAAAA803FFFC00000E7
:10A75000003FFF00003FFFFFC003FFFFFFFFFFFCC4
:10A76000000003FFFFFC00FFFFC0000000003FFFF0
:10A77000FFFFFFFFFFFFFFFFFFFFFFF000000000F4
:10A7800000000000000003FF0000000000000003C4
:10A79000FFFFFFFF000FFFFFFFFFFC0002AAAAAAB6
:10A7A0008000002AAAAAAAAAAAAAAAAAAAAA803F9C
:10A7B000FFC00000003FFF00003FFFFFC003FFFF9E
:10A7C000FFFFFFFC000003FFFFFC00FFFFC00000D5
:10A7D00000003FFFFFFFFFFFFFFFFFFFFFFFFFF056
:10A7E0000003FFC000003FC000000FFF000000FC9E
:10A7F00000000003FFFFFFFF000FFFFFFFFFFC0053
:10A8000002AAAAAAA0000000AAAAAAAAAAAAAAAA58
:10A81000AAA80000000000000000000003FFFFFFE6
:10A82000C003FFFFFFFFFFFFF0000FFFFFFFCFFFA1
:10A83000FC00000000000FFFFFFFFFFFFFFFFFFF16
:10A84000FFFFFFF00003FFC000003FC000000FFF4C
:10A85000000000FC00000003FFFFFFFF000FFFFFF0
:10A86000FFFFFC0002AAAAAAA0000000AAAAAAAAA6
:10A87000AAAAAAAAAAA800000000000000000000DE
:10A8800003FFFFFFC003FFFFFFFFFFFFF0000FFF0D
:10A89000FFFFCFFFFC00000000000FFFFFFFFFFFE6
:10A8A000FFFFFFFFFFFFFFF00003FFF00003FFC00B
:10A8B00000000FFF00000FFF000000003FFFFFFF40
:10A8C000000FFFFFFFFFFC0002AAAAAAAA000000D7
:10A8D0002AAAAAAAAAAAAAAAAAA00000000000005E
:10A8E0000000000003FFFFFFC003FFFFFFFFFFFFAB
:10A8F000F000FFFFFFFFFFFFF00002AAAA00003FE9
:10A90000FFFFFFFFFFFFFFFFFFFFFFF00003FFF070
:10A910000003FFFC00000FF000000FFF000000002C
:10A920003FFFFFFF000FFFFFFFFFFC0002AAAAAAE4
:10A93000AA80000002AAAAAAAAAAAAAAAA0000009B
:10A9400000000000000000000FFFFFFFC003FFFF3A
:10A95000FFFFFFFFF000FFFFFFFFFFFF0000AAAABD
:10A96000AAA8003FFFFFFFFFFFFFFFFFFFFFFFF071
:10A970000003FFF00003FFFC00000FF000000FFFDA
:10A98000000000003FFFFFFF000FFFFFFFFFFC0084
:10A9900002AAAAAAAA80000002AAAAAAAAAAAAAAE5
:10A9A000AA00000000000000000000000FFFFFFFF1
:10A9B000C003FFFFFFFFFFFFF000FFFFFFFFFFFFF0
:10A9C0000000AAAAAAA8003FFFFFFFFFFFFFFFFFAA
:10A9D000FFFFFFF00000FFFF0003FFFC0000FFF09F
:10A9E00000003FFFF00000003FFFFFFF000FFFFFF0
:10A9F000FFFFFC0002AAAAAAAAA8000000AAAAAA0D
:10AA0000AAAAAAAAA80000000000000000000000F6
:10AA1000FFFFFFFFC003FFFFFFFFFFFFF000FFFF8F
:10AA2000FFFFFFFF000AAAAAAAAA8003FFFFFFFFF9
:10AA3000FFFFFFFFFFFFFFF00000FFFF0003FFFC31
:10AA40000000FFF000003FFFF00000003FFFFFFFAD
:10AA5000000FFFFFFFFFFC0002AAAAAAAAA800009D
:10AA600000AAAAAAAAAAAAAAA80000000000000098
:10AA700000000000FFFFFFFFC003FFFFFFFFFFFF1D
:10AA8000F000FFFFFFFFFFFF000AAAAAAAAA8003A7
:10AA9000FFFFFFFFFFFFFFFFFFFFFFF00000FFFFD3
:10AAA000000FFFFC0000FFC000003FFFF0000000AF
:10AAB0003FFFFFFF000FFFFFFFFFFC0002AAAAAA53
:10AAC000AAAAA000000AAAAAAAAAAAAA0000002A62
:10AAD000000000000000003FFFFFFFFFC003FFFF7A
:10AAE000FFFFFFFFC003FFFFFFFC0000002AAAAA30
:10AAF000AAAA8003FFFFFFFFFFFFFFFFFFFFFFF09A
:10AB00000000FFFF000FFFFC0000FFC000003FFF40
:10AB1000F00000003FFFFFFF000FFFFFFFFFFC0002
:10AB200002AAAAAAAAAAA000000AAAAAAAAAAAAA2B
:10AB30000000002A000000000000003FFFFFFFFFB0
:10AB4000C003FFFFFFFFFFFFC003FFFFFFFC00008C
:10AB5000002AAAAAAAAA8003FFFFFFFFFFFFFFFFA8
:10AB6000FFFFFFF00000FFFF000FFFFF0003FFC02B
:10AB70000003FFFFFC0000003FFFFFFF000FFFFF8F
:10AB8000FFFFFC0002AAAAAAAAAAA8000002AAAA79
:10AB9000AAAAAAA0000000AAA8000000000000FFC6
:10ABA000FFFFFFFFC003FFFFFFFC00000000FFFFEF
:10ABB000FF00000002AAAAAAAAAAA000FFFFFFFFA6
:10ABC000FFFFFFFFFFFFFFF000000FFFC00FFFFFC1
:10ABD0000003FFC00003FFFFFC0000003FFFFFFF7A
:10ABE000000FFFFFFFFFFC0002AAAAAAAAAAAA80E0
:10ABF00000002AAAAAAAAA8000000AAAAAA0000005
:10AC0000000000FFFFFFFFFFC003FFFFFFFC00FF8E
:10AC1000F000FFFFFC00000002AAAAAAAAAAAA004C
:10AC2000FFFFFFFFFFFFFFFFFFFFFFF000000FFF31
:10AC3000C00FFFFF0003FFC00003FFFFFC00000088
:10AC40003FFFFFFF000FFFFFFFFFFC0002AAAAAAC1
:10AC5000AAAAAA8000002AAAAAAAAA8000000AAA70
:10AC6000AAA00000000000FFFFFFFFFFC003FFFFDE
:10AC7000FFFC00FFF000FFFFFC00000002AAAAAAF0
:10AC8000AAAAAA00FFFFFFFFFFFFFFFFFFFFFFF0E1
:10AC900000000FFFFFFFFFFF003FFFF0000FFFFF6F
:10ACA000FFC000003FFFFFFF000FFFFFFFFFFC00A2
:10ACB00002AAAAAAAAAAAA80000000AAAAAAA80070
:10ACC00000002AAAAAAA0000000000FFFFFFFFFF61
:10ACD000C003FFFFFFFFFFFFF000FFFFC000000009
:10ACE00002AAAAAAAAAAAA000FFFFFFFFFFFFFFF5E
:10ACF000FFFFFFF000000FFFFFFFFFFF003FFFF02F
:10AD0000000FFFFFFFC000003FFFFFFF000FFFFF2E
:10AD1000FFFFFC0002AAAAAAAAAAAA80000000AA11
:10AD2000AAAAA80000002AAAAAAA0000000000FF00
:10AD3000FFFFFFFFC003FFFFFFFFFFFFF000FFFF6C
:10AD4000C000000002AAAAAAAAAAAA000FFFFFFF39
:10AD5000FFFFFFFFFFFFFFF000000FFFFFFFFFFF00
:10AD6000FFFFFFFF000FFFFFFFC000003FFFFFFFDF
:10AD7000000FFFFFFFFFFC0002AAAAAAAAAAAA804E
:10AD80000000002AAAAAA00000000AAAAAAAAAAA49
:10AD9000A00000FFFFFFFFFFC003FFFFFFFFFFFF5B
:10ADA000FF00FFFF0002AAAAAAAAAAAAAAAAAA00AA
:10ADB0000FFFFFFFFFFFFFFFFFFFFFF0000003FF9C
:10ADC000FFFC00FFFFFFFFFF000FFF00FFF0000090
:10ADD0003FFFFFFF000FFFFFFFFFFC0002AAAAAA30
:10ADE000AAAAA80000000002AAAA0000000000AA67
:10ADF000AAAAAAAAA00000FFFFFFFFFFC003FFFF4F
:10AE0000FFFFFFFFFF03FFFF000AAAAAAAAAAAAA40
:10AE1000AAAAAA0003FFFFFFFFFFFFFFFFFFFFF04B
:10AE2000000003FFFFFC00FFFFFFFFFF000FFF001C
:10AE3000FFF000003FFFFFFF000FFFFFFFFFFC00E0
:10AE400002AAAAAAAAAAA80000000002AAAA0000B0
:10AE5000000000AAAAAAAAAAA00000FFFFFFFFFF05
:10AE6000C003FFFFFFFFFFFFFF03FFFF000AAAAAC7
:10AE7000AAAAAAAAAAAAAA0003FFFFFFFFFFFFFF30
:10AE8000FFFFFFF0000003FFFFFC00FFFFFFFFFFDD
:10AE900000FFF000FFF000003FFFFFFF000FFFFF8B
:10AEA000FFFFFC0002AAAAAAAAAAA00000000000B4
:10AEB000AAA000000000002AAAAAAAAAA00000FFD7
:10AEC000FFFFFFFFC003FFFFFFFFFFFFF03FFFFF9C
:10AED00000AAAAAAAAAAAAAAAAAAAA00003FFFFF91
:10AEE000FFFFFFFFFFFFFFF0000003FFFFFC00FF7D
:10AEF000FFFFFFFF00FFF000FFF000003FFFFFFF3C
:10AF0000000FFFFFFFFFFC0002AAAAAAAAAAA00046
:10AF100000000000AAA000000000002AAAAAAAAA15
:10AF2000A00000FFFFFFFFFFC003FFFFFFFFFFFFC9
:10AF3000F03FFFFF00AAAAAAAAAAAAAAAAAAAA0040
:10AF4000003FFFFFFFFFFFFFFFFFFFF0000003FFD9
:10AF5000FFFC003FFFFFFFFFFFFFF0000FFF0000BF
:10AF60003FFFFFFF000FFFFFFFFFFC0002AAAAAA9E
:10AF7000AAAA0000000000000A80000000000002F1
:10AF8000AAAAAAAAA00000FFFFFFFFFFC003FFFFBD
:10AF9000FFFFFFFC00FFFFF000AAAAAAAAAAAAAA24
:10AFA000AAAAAA80000FFFFFFFFFFFFFFFFFFFF02D
:10AFB0000000003FFFF0003FFFFF003FFFFFC00029
:10AFC0000FFF00003FFFFFFF000FFFFFFFFFFC0030
:10AFD00002AAAAAAAAA8000002A800000000000075
:10AFE000AA000000AAAAAAAAA00000FFFFFFFFFF74
:10AFF000C003FFFFFFFFFFF00FFFFC0002AAAAAA99
:10B00000AAAAAAAAAAAAAAAA0000FFFFFFFFFFFFF6
:10B01000FFFFFFF00000003FFFF0003FFFFF003F99
:10B02000FFFFC0000FFF00003FFFFFFF000FFFFF0B
:10B03000FFFFFC0002AAAAAAAAA8000002A800001A
:10B0400000000000AA000000AAAAAAAAA00000FF0F
:10B05000FFFFFFFFC003FFFFFFFFFFF00FFFFC003C
:10B0600002AAAAAAAAAAAAAAAAAAAAAA0000FFFF92
:10B07000FFFFFFFFFFFFFFF00000003FFFF00003B6
:10B08000FFFF000FFFFFC0000FFFC0003FFFFFFFEB
:10B09000000FFFFFFFFFFC0002AAAAAAAA8000007F
:10B0A0002AAA80000000000AAAA00000AAAAAAAA50
:10B0B000A00000FFFFFFFFFFC003FFFFFFFFFF0037
:10B0C0003FFF000002AAAAAAAAAAAAAAAAAAAAAAF2
:10B0D000A000FFFFFFFFFFFFFFFFFFF00000003FAA
:10B0E000FFF00003FFFF000FFFFFC0000FFFC000D5
:10B0F0003FFFFFFF000FFFFFFFFFFC0002AAAAAA0D
:10B10000AA8000002AAA80000000000AAAA000006D
:10B11000AAAAAAAAA00000FFFFFFFFFFC003FFFF2B
:10B12000FFFFFF003FFF000002AAAAAAAAAAAAAA3C
:10B13000AAAAAAAAA000FFFFFFFFFFFFFFFFFFF0E0
:10B140000000003FFFF00003FFFC000FFFFC0000C9
:10B150000FFF00003FFFFFFF000FFFFFFFFFFC009E
:10B1600002AAAAAAAA000000AAAAA0000000002A17
:10B17000AAA000000AAAAAAAA00000FFFFFFFFFFE2
:10B18000C003FFFFFFFFF00FFFC0000002AAAAAA42
:10B19000AAAAAAAAAAAAAAAAA8003FFFFFFFFFFF7D
:10B1A000FFFFFFF00000003FFFF00003FFFC000F77
:10B1B000FFFC00000FFF00003FFFFFFF000FFFFF3D
:10B1C000FFFFFC0002AAAAAAAA000000AAAAA000E7
:10B1D0000000002AAAA000000AAAAAAAA00000FF54
:10B1E000FFFFFFFFC003FFFFFFFFF00FFFC00000E6
:10B1F00002AAAAAAAAAAAAAAAAAAAAAAA8003FFF19
:10B20000FFFFFFFFFFFFFFF00000000FFF00000344
:10B21000FFFC000FFFFC00000FFF00003FFFFFFFDF
:10B22000000FFFFFFFFFFC0002AAAAAAA000000A6D
:10B23000AAAAAA00000002AAAAA8000002AAAAAA12
:10B24000A00000FFFFFFFFFFC003FFFFFFFFFFFFA6
:10B25000FF00000002AAAAAAAAAAAAAAAAAAAAAA9F
:10B26000AA803FFFFFFFFFFFFFFFFFFC0000000F72
:10B27000FF000000FFC0000FFFF000000FF0000013
:10B280003FFFFFFF000FFFFFFFFFFC0002AAAAAA7B
:10B290008000002AAAAAAA8000000AAAAAAA8000FE
:10B2A000002AAAAAA00000FFFFFFFFFFC003FFFFC4
:10B2B000FFFFFFFFFF000AAA82AAAAAAAAAAAAAAB7
:10B2C000AAAAAAAAAA8003FFFFFFFFFFFFFFFFFCB5
:10B2D0000000000FFF000000FFC0000FFFF00000A3
:10B2E0000FF000003FFFFFFF000FFFFFFFFFFC001C
:10B2F00002AAAAAA8000002AAAAAAA8000000AAA72
:10B30000AAAA8000002AAAAAA00000FFFFFFFFFF50
:10B31000C003FFFFFFFFFFFFFF000AAA82AAAAAA3D
:10B32000AAAAAAAAAAAAAAAAAA8003FFFFFFFFFFA5
:10B33000FFFFFFFC0000000FFF000000FFC0000047
:10B34000FFF00000FFF000003FFFFFFF000FFFFFD6
:10B35000FFFFFC0002AAAAA8000002AAAAAAAAA8A3
:10B36000000AAAAAAAAAA000000AAAAAA00000FF8E
:10B37000FFFFFFFFC003FFFFFFFFFFFFF000AAAAD0
:10B38000AAAAAAAAAAAAAAAAAAAAAAAAAAA003FF79
:10B39000FFFFFFFFFFFFFFFC0000000FFF000000AA
:10B3A000FFC00000FFF00000FFF000003FFFFFFFC4
:10B3B000000FFFFFFFFFFC0002AAAAA8000002AADC
:10B3C000AAAAAAA8000AAAAAAAAAA000000AAAAA27
:10B3D000A00000FFFFFFFFFFC003FFFFFFFFFFFF15
:10B3E000F000AAAAAAAAAAAAAAAAAAAAAAAAAAAA21
:10B3F000AAA003FFFFFFFFFFFFFFFFFC000000000C
:10B40000FC000000FFC00000FFF00000FFC00000D3
:10B410003FFFFFFF000FFFFFFFFFFC0002AAAAA8EB
:10B4200000000AAAAAAAAAAA002AAAAAAAAAAA0044
:10B430000000AAAAA00000FFFFFFFFFFC003FFFF5C
:10B44000FFFFFFFFF000AAAAAAAAAAAAAAAAAAAA6C
:10B45000AAAAAAAAAAA003FFFFFFFFFFFFFFFFFF00
:10B46000C000000000000000000000000000000319
:10B47000FFC000003FFFFFFF000FFFFFFFFFFC00CA
:10B4800002AAAAA000000AAAAAAAAAAAAAAAAAAAC2
:10B49000AAAAAA8000002AAAA00000FFFFFFFFFFBF
:10B4A000C003FFFFFFFFFFFFC002AAAAAAAAAAAA21
:10B4B000AAAAAAAAAAAAAAAAAAA003FFFFFFFFFFF4
:10B4C000FFFFFFFFC00000000000000000000000C0
:10B4D00000000003FFC000003FFFFFFF000FFFFF61
:10B4E000FFFFFC0002AAAAA000000AAAAAAAAAAA10
:10B4F000AAAAAAAAAAAAAA8000002AAAA00000FFB3
:10B50000FFFFFFFFC003FFFFFFFFFFFFC002AAAA6C
:10B51000AAAAAAAAAAAAAAAAAAAAAAAAAAA003FFE7
:10B52000FFFFFFFFFFFFFFFFC00000000000000063
:10B530000000000000000003FC0000003FFFFFFFD0
:10B54000000FFFFFFFFFFC0002AAAA000000AAAA4A
:10B55000AAAAAAAAAAAAAAAAAAAAAAA8000002AA49
:10B56000A00000FFFFFFFFFFC003FFFFFFFFFFFF83
:10B57000C002AAAAAAAAAAAAAAAAAAAAAAAAAAAABD
:10B58000AA8003FFFFFFFFFFFFFFFFFFC0000000D7
:10B59000000000000000000000000003FC000000AC
:10B5A0003FFFFFFF000FFFFFFFFFFC0002AAAA0002
:10B5B0000000AAAAAAAAAAAAAAAAAAAAAAAAAAA841
:10B5C000000002AAA00000FFFFFFFFFFC003FFFF73
:10B5D000FFFFFFFFC002AAAAAAAAAAAAAAAAAAAA09
:10B5E000AAAAAAAAAA8003FFFFFFFFFFFFFFFFFF8F
:10B5F000F00000000000000000000000000000FF5C
:10B60000FC0000003FFFFFFF000FFFFFFFFFFC00FB
:10B6100002AAA8000002AAAAAAAAAAAAAAAAAAAA30
:10B62000AAAAAAAA000000AAA00000FFFFFFFFFF2D
:10B63000C003FFFFFFFFFFFFC002AAAAAAAAAAAA8F
:10B64000AAAAAAAAAAAAAAAAAA803FFFFFFFFFFF46
:10B65000FFFFFFFFF00000000000000000000000FE
:10B66000000000FFFC0000003FFFFFFF000FFFFF96
:10B67000FFFFFC0002AAA8000002AAAAAAAAAAAA7E
:10B68000AAAAAAAAAAAAAAAA000000AAA00000FF21
:10B69000FFFFFFFFC003FFFFFFFFFFFFC002AAAADB
:10B6A000AAAAAAAAAAAAAAAAAAAAAAAAAA803FFF3A
:10B6B000FFFFFFFFFFFFFFFFF000000000000000A2
:10B6C00000000000000000FFFC0000003FFFFFFF43
:10B6D000000FFFFFFFFFFC0002AA8000002AAAAAB9
:10B6E000AAAAAAAAAAAAAAAAAAAAAAAAA000000AB8
:10B6F000A00000FFFFFFFFFFC003FFFFFFFFFFFFF2
:10B70000F002AAAAAAAAAAAAAAAAAAAAAAAAAAAAFB
:10B71000A8003FFFFFFFFFFFFFFFFFFFFF0000004C
:10B720000000000000000000000000FFFC0000001E
:10B730003FFFFFFF000FFFFFFFFFFC0002AA00001A
:10B7400000AAAAAAAAAAAAAAAAAAAAAAAAAAAAAA03
:10B75000A8000002A00000FFFFFFFFFFC003FFFFE3
:10B76000FFFFFFFFF000AAAAAAAAAAAAAAAAAAAA49
:10B77000AAAAAAAAA8003FFFFFFFFFFFFFFFFFFF43
:10B78000FF0000000000000000000000000000FFBB
:10B79000FC0000003FFFFFFF000FFFFFFFFFFC006A
:10B7A00002AA000000AAAAAAAAAAAAAAAAAAAAAA9F
:10B7B000AAAAAAAAA8000002A00000FFFFFFFFFF9C
:10B7C000C003FFFFFFFFFFFFF000AAAAAAAAAAAAD0
:10B7D000AAAAAAAAAAAAAAAAA8003FFFFFFFFFFF37
:10B7E000FFFFFFFFFFC0000000000000000000009E
:10B7F000000000FFF00000003FFFFFFF000FFFFF11
:10B80000FFFFFC0002A000000AAAAAAAAAAAAAAAEC
:10B81000AAAAAAAAAAAAAAAAAA800000200000FF8F
:10B82000FFFFFFFFC003FFFFFFFFFFFFFF000AAAAC
:10B83000AAAAAAAAAAAAAAAAAAAAAAAAA000FFFF72
:10B84000FFFFFFFFFFFFFFFFFFC000000000000041
:10B8500000000000000000FFF00000003FFFFFFFBD
:10B86000000FFFFFFFFFFC0002A000000AAAAAAA27
:10B87000AAAAAAAAAAAAAAAAAAAAAAAAAA800000A6
:10B88000200000FFFFFFFFFFC003FFFFFFFFFFFFE0
:10B89000FF000AAAAAAAAAAAAAAAAAAAAAAAAAAAFD
:10B8A000A000FFFFFFFFFFFFFFFFFFFFFFC0000043
:10B8B0000000000000000000000000FC000000008C
:10B8C0003FFFFFFF000FFFFFFFFFFC000000000035
:10B8D0002AAAAAAAAAAAAAAAAAAAAAAAAAAAAAAA48
:10B8E000AAA00000000000FFFFFFFFFFC003FFFF52
:10B8F000FFFFFFFFFF00000000000000000000004D
:10B9000000000000000FFFFFFFFFFFFFFFFFFFFF32
:10B91000FFFC00000000000000000000000000C06C
:10B92000000000003FFFFFFF000FFFFFFFFFFC00D4
:10B9300000000002AAAAAAAAAAAAAAAAAAAAAAAA0D
:10B94000AAAAAAAAAAA00000000000FFFFFFFFFF0A
:10B95000C003FFFFFFFFFFFFFFC00000000000006B
:10B960000000000000000000003FFFFFFFFFFFFF9E
:10B97000FFFFFFFFFFFC00000000000000000000D0
:10B98000000000C0000000003FFFFFFF000FFFFFAE
:10B99000FFFFFC0000000002AAAAAAAAAAAAAAAA5B
:10B9A000AAAAAAAAAAAAAAAAAAA00000000000FFFE
:10B9B000FFFFFFFFC003FFFFFFFFFFFFFFC000000F
:10B9C000000000000000000000000000003FFFFF3A
:10B9D000FFFFFFFFFFFFFFFFFFFF00000000000071
:10B9E0000000000000000000000000003FFFFFFF1B
:10B9F000000FFFFFFFFFFC000000000AAAAAAAAA8E
:10BA0000AAAAAAAAAAAAAAAAAAAAAAAAAAAA0000EA
:10BA1000000000FFFFFFFFFFC003FFFFFFFFFFFF6E
:10BA2000FFFC00000000000000000000000000001B
:10BA300003FFFFFFFFFFFFFFFFFFFFFFFFFF000010
:10BA400000000000000000000000000000000000F6
:10BA50003FFFFFFF000FFFFFFFFFFC000000000A99
:10BA6000AAAAAAAAAAAAAAAAAAAAAAAAAAAAAAAA36
:10BA7000AAAA0000000000FFFFFFFFFFC003FFFFB6
:10BA8000FFFFFFFFFFFC00000000000000000000BF
:10BA90000000000003FFFFFFFFFFFFFFFFFFFFFFAE
:10BAA000FFFFF000000000000000000000000000A8
:10BAB000000000003FFFFFFF000FFFFFFFFFFC0043
:10BAC000000000AAAAAAAAAAAAAAAAAAAAAAAAAAD4
:10BAD000AAAAAAAAAAAA8000000000FFFFFFFFFFEF
:10BAE000C003FFFFFFFFFFFFFFFFFC00000000009F
:10BAF0000000000000000003FFFFFFFFFFFFFFFF4B
:10BB0000FFFFFFFFFFFFFC0000000000000000003F
:10BB100000000000000000003FFFFFFF000FFFFFDC
:10BB2000FFFFFC00000002AAAAAAAAAAAAAAAAAA1F
:10BB3000AAAAAAAAAAAAAAAAAAAAA800000000FFBA
:10BB4000FFFFFFFFC003FFFFFFFFFFFFFFFFFFFF40
:10BB5000FFFFFFFFFFFFFFFFFFFFFFFFFFFFFFFFF5
:10BB6000FFFFFFFFFFFFFFFFFFFFFC0000000000E3
:10BB70000000000000000000000000003FFFFFFF89
:10BB8000000FFFFFFFFFFC00000002AAAAAAAAAA5A
:10BB9000AAAAAAAAAAAAAAAAAAAAAAAAAAAAA800B1
:10BBA000000000FFFFFFFFFFC003FFFFFFFFFFFFDD
:10BBB000FFFFFFFFFFFFFFFFFFFFFFFFFFFFFFFF95
:10BBC000FFFFFFFFFFFFFFFFFFFFFFFFFFFFFFC0C4
:10BBD0000000000000000000000000000000000065
:10BBE0003FFFFFFF000FFFFFFFFFFC000000000012
:10BBF0000000000000000000000000000000000045
:10BC000000000000000000FFFFFFFFFFC003FFFF78
:10BC1000FFFFFFFFFFFFFFFFFFFFFFFFFFFFFFFF34
:10BC2000FFFFFFFFFFFFFFFFFFFFFFFFFFFFFFFF24
:10BC3000FFFFFFC000000000000000000000000047
:10BC4000000000003FFFFFFF000FFFFFFFFFFC00B1
:10BC500000000000000000000000000000000000E4
:10BC60000000000000000000000000FFFFFFFFFFD9
:10BC7000C003FFFFFFFFFFFFFFFFFFFFFFFFFFFF0F
:10BC8000FFFFFFFFFFFFFFFFFFFFFFFFFFFFFFFFC4
:10BC9000FFFFFFFFFFFFFFFF0000000000000000AC
:10BCA00000000000000000003FFFFFFF000FFFFF4B
:10BCB000FFFFFC000000000000000000000000008A
:10BCC000000000000000000000000000000000FF75
:10BCD000FFFFFFFFC003FFFFFFFFFFFFFFFFFFFFAF
:10BCE000FFFFFFFFFFFFFFFFFFFFFFFFFFFFFFFF64
:10BCF000FFFFFFFFFFFFFFFFFFFFFFFF0000000050
:10BD00000000000000000000000000003FFFFFFFF7
:10BD1000000FFFFFFFFFFC0000000000000000001C
:10BD20000000000000000000000000000000000013
:10BD3000000000FFFFFFFFFFC003FFFFFFFFFFFF4B
:10BD4000FFFFFFFFFFFFFFFFFFFFFFFFFFFFFFFF03
:10BD5000FFFFFFFFFFFFFFFFFFFFFFFFFFFFFFFFF3
:10BD6000C000000000000000000000000000000013
:10BD70003FFFFFFF000FFFFFFFFFFC000000000080
:10BD800000000000000000000000000000000000B3
:10BD900000000000000000FFFFFFFFFFC003FFFFE7
:10BDA000FFFFFFFFFFFFFFFFFFFFFFFFFFFFFFFFA3
:10BDB000FFFFFFFFFFFFFFFFFFFFFFFFFFFFFFFF93
:10BDC000FFFFFFFFFF000000000000000000000078
:10BDD000000000003FFFFFFF000FFFFFFFFFFC0020
:10BDE0000000000000000000000000000000000053
:10BDF0000000000000000000000000FFFFFFFFFF48
:10BE0000C003FFFFFFFFFFFFFFFFFFFFFFFFFFFF7D
:10BE1000FFFFFFFFFFFFFFFFFFFFFFFFFFFFFFFF32
:10BE2000FFFFFFFFFFFFFFFFFF000000000000001B
:10BE300000000000000000003FFFFFFF000FFFFFB9
:10BE4000FFFFFC00000000000000000000000000F8
:10BE5000000000000000000000000000000000FFE3
:10BE6000FFFFFFFFC003FFFFFFFFFFFFFFFFFFFF1D
:10BE7000FFFFFFFFFFFFFFFFFFFFFFFFFFFFFFFFD2
:10BE8000FFFFFFFFFFFFFFFFFFFFFFFFFFFC0000C3
:10BE90000000000000000000000000003FFFFFFF66
:10BEA000000FFFFFFFFFFC0000000000000000008B
:10BEB0000000000000000000000000000000000082
:10BEC000000000FFFFFFFFFFC003FFFFFFFFFFFFBA
:10BED000FFFFFFFFFFFFFFFFFFFFFFFFFFFFFFFF72
:10BEE000FFFFFFFFFFFFFFFFFFFFFFFFFFFFFFFF62
:10BEF000FFFC000000000000000000000000000047
:10BF00003FFFFFFF000FFFFFFFFFFC0000000000EE
:10BF10000000000000000000000000000000000021
:10BF200000000000000000FFFFFFFFFFC003FFFF55
:10BF3000FFFFFFFFFFFFFFFFFFFFFFFFFFFFFFFF11
:10BF4000FFFFFFFFFFFFFFFFFFFFFFFFFFFFFFFF01
:10BF5000FFFFFFFFFFFFFF000000000000000000E8
:10BF6000000000003FFFFFFF000FFFFFFFFFFC008E
:10BF700000000000000000000000000000000000C1
:10BF80000000000000000000000000FFFFFFFFFFB6
:10BF9000C003FFFFFFFFFFFFFFFFFFFFFFFFFFFFEC
:10BFA000FFFFFFFFFFFFFFFFFFFFFFFFFFFFFFFFA1
:10BFB000FFFFFFFFFFFFFFFFFFFFFFFFFFFFFFFF91
:10BFC000FFFFFFFFFFFFFFFFFFFFFFFF000FFFFF70
:10BFD000FFFFFFFFFFFFFFFFFFFFFFFFFFFFFFFF71
:10BFE000FFFFFFFFFFFFFFFFFFFFFFFFFFFFFFFF61
:10BFF000FFFFFFFFC003FFFFFFFFFFFFFFFFFFFF8C
:10C00000FFFFFFFFFFFFFFFFFFFFFFFFFFFFFFFF40
:10C01000FFFFFFFFFFFFFFFFFFFFFFFFFFFFFFFF30
:10C02000FFFFFFFFFFFFFFFFFFFFFFFFFFFFFFFF20
:10C03000000FFFFFFFFFFFFFFFFFFFFFFFFFFFFFFF
:10C04000FFFFFFFFFFFFFFFFFFFFFFFFFFFFFFFF00
:10C05000FFFFFFFFFFFFFFFFC003FFFFFFFFFFFF2B
:10C06000FFFFFFFFFFFFFFFFFFFFFFFFFFFFFFFFE0
:10C07000FFFFFFFFFFFFFFFFFFFFFFFFFFFFFFFFD0
:10C08000FFFFFFFFFFFFFFFFFFFFFFFFFFFFFFFFC0
:10C09000FFFFFFFF000FFFFFFFFFFFFFFFFFFFFF9F
:10C0A000FFFFFFFFFFFFFFFFFFFFFFFFFFFFFFFFA0
:10C0B000FFFFFFFFFFFFFFFFFFFFFFFFC003FFFFCB
:10C0C000FFFFFFFFFFFFFFFFFFFFFFFFFFFFFFFF80
:10C0D000FFFFFFFFFFFFFFFFFFFFFFFFFFFFFFFF70
:10C0E000FFFFFFFFFFFFFFFFFFFFFFFFFFFFFFFF60
:10C0F000FFFFFFFFFFFFFFFF000FFFFFFFFFFFFF3F
:10C10000FFFFFFFFFFFFFFFFFFFFFFFFFFFFFFFF3F
:10C11000FFFFFFFFFFFFFFFFFFFFFFFFFFFFFFFF2F
:10C12000C003FFFFFFFFFFFFFFFFFFFFFFFFFFFF5A
:10C13000FFFFFFFFFFFFFFFFFFFFFFFFFFFFFFFF0F
:10C14000FFFFFFFFFFFFFFFFFFFFFFFFFFFFFFFFFF
:10C15000FFFFFFFFFFFFFFFFFFFFFFFF000FFFFFDE
:10C16000FFFFFFFFFFFFFFFFFFFFFFFFFFFFFFFFDF
:10C17000FFFFFFFFFFFFFFFFFFFFFFFFFFFFFFFFCF
:10C18000FFFFFFFFC003FFFFFFFFFFFFFFFFFFFFFA
:10C19000FFFFFFFFFFFFFFFFFFFFFFFFFFFFFFFFAF
:10C1A000FFFFFFFFFFFFFFFFFFFFFFFFFFFFFFFF9F
:10C1B000FFFFFFFFFFFFFFFFFFFFFFFFFFFFFFFF8F
:10C1C000000FFFFFFFFFFFFFFFFFFFFFFFFFFFFF6E
:10C1D000FFFFFFFFFFFFFFFFFFFFFFFFFFFFFFFF6F
:10C1E000FFFFFFFFFFFFFFFFC003FFFFFFFFFFFF9A
:10C1F000FFFFFFFFFFFFFFFFFFFFFFFFFFFFFFFF4F
:10C20000FFFFFFFFFFFFFFFFFFFFFFFFFFFFFFFF3E
:10C21000FFFFFFFFFFFFFFFFFFFFFFFFFFFFFFFF2E
:10C22000FFFFFFFF000FFFFFFFFFFFFFFFFFFFFF0D
:10C23000FFFFFFFFFFFFFFFFFFFFFFFFFFFFFFFF0E
:10C24000FFFFFFFFFFFFFFFFFFFFFFFFC003FFFF39
:10C25000FFFFFFFFFFFFFFFFFFFFFFFFFFFFFFFFEE
:10C26000FFFFFFFFFFFFFFFFFFFFFFFFFFFFFFFFDE
:10C27000FFFFFFFFFFFFFFFFFFFFFFFFFFFFFFFFCE
:10C28000FFFFFFFFFFFFFFFF000FFFFFFFFFFFFFAD
:10C29000FFFFFFFFFFFFFFFFFFFFFFFFFFFFFFFFAE
:10C2A000FFFFFFFFFFFFFFFFFFFFFFFFFFFFFFFF9E
:10C2B000C003FFFFFFFFFFFFFFFFFFFFFFFFFFFFC9
:10C2C000FFFFFFFFFFFFFFFFFFFFFFFFFFFFFFFF7E
:10C2D000FFFFFFFFFFFFFFFFFFFFFFFFFFFFFFFF6E
:10C2E000FFFFFFFFFFFFFFFFFFFFFFFF000FFFFF4D
:10C2F000FFFFFFFFFFFFFFFFFFFFFFFFFFFFFFFF4E
:10C30000FFFFFFFFFFFFFFFFFFFFFFFFFFFFFFFF3D
:10C31000FFFFFFFFC003FFFFFFFFFFFFFFFFFFFF68
:10C32000FFFFFFFFFFFFFFFFFFFFFFFFFFFFFFFF1D
:10C33000FFFFFFFFFFFFFFFFFFFFFFFFFFFFFFFF0D
:10C34000FFFFFFFFFFFFFFFFFFFFFFFFFFFFFFFFFD
:10C35000000FFFFFFFFFFFFFFFFFFFFFFFFFFFFFDC
:10C36000FFFFFFFFFFFFFFFFFFFFFFFFFFFFFFFFDD
:10C37000FFFFFFFFFFFFFFFFC003FFFFFFFFFFFF08
:10C38000FFFFFFFFFFFFFFFFFFFFFFFFFFFFFFFFBD
:10C39000FFFFFFFFFFFFFFFFFFFFFFFFFFFFFFFFAD
:10C3A000FFFFFFFFFFFFFFFFFFFFFFFFFFFFFFFF9D
:10C3B000FFFFFFFF000FFFFFFFFFFFFFFFFFFFFF7C
:10C3C000FFFFFFFFFFFFFFFFFFFFFFFFFFFFFFFF7D
:10C3D000FFFFFFFFFFFFFFFFFFFFFFFFC003FFFFA8
:10C3E000FFFFFFFFFFFFFFFFFFFFFFFFFFFFFFFF5D
:10C3F000FFFFFFFFFFFFFFFFFFFFFFFFFFFFFFFF4D
:10C40000FFFFFFFFFFFFFFFFFFFFFFFFFFFFFFFF3C
:10C41000FFFFFFFFFFFFFFFF000FFFFFFFFFFFFF1B
:10C42000FFFFFFFFFFFFFFFFFFFFFFFFFFFFFFFF1C
:10C43000FFFFFFFFFFFFFFFFFFFFFFFFFFFFFFFF0C
:10C44000C003FFFFFFFFFFFFFFFFFFFFFFFFFFFF37
:10C45000FFFFFFFFFFFFFFFFFFFFFFFFFFFFFFFFEC
:10C46000FFFFFFFFFFFFFFFFFFFFFFFFFFFFFFFFDC
:10C47000FFFFFFFFFFFFFFFFFFFFFFFF000FFFFFBB
:10C48000FFFFFFFFFFFFFFFFFFFFFFFFFFFFFFFFBC
:10C49000FFFFFFFFFFFFFFFFFFFFFFFFFFFFFFFFAC
:10C4A000FFFFFFFFC003FFFFFFFFFFFFFFFFFFFFD7
:10C4B000FFFFFFFFFFFFFFFFFFFFFFFFFFFFFFFF8C
:10C4C000FFFFFFFFFFFFFFFFFFFFFFFFFFFFFFFF7C
:10C4D000FFFFFFFFFFFFFFFFFFFFFFFFFFFFFFFF6C
:10C4E000000FFFFFFFFFFFFFFFFFFFFFFFFFFFFF4B
:10C4F000FFFFFFFFFFFFFFFFFFFFFFFFFFFFFFFF4C
:10C50000FFFFFFFFFFFFFFFFC003FFFFFFFFFFFF76
:10C51000FFFFFFFFFFFFFFFFFFFFFFFFFFFFFFFF2B
:10C52000FFFFFFFFFFFFFFFF000000000000000013
:10C5300000000000000000000000000000000000FB
:10C5400000000000000000000000000000000000EB
:10C5500000000000000000000000000000000000DB
:10C5600000000000000000000000000000000000CB
:10C7E00000000000FFFFFFFFFFFFFFFFFFFFFFFF55
:10C7F000FFFFFFFFFFFFFFFFFFFFFFFFFFFFFFFF49
:10C80000FFFFFFFFFFFFFFFFFFFFFFFFFFFFFFFF38
:10C81000FFFFFFFFFFFFFFFFFFFFFFFFFFFFFFFF28
:10C82000FFFFFFFFFFFFFFFFFFFFFFFFFFFFFFFF18
:10CC1000FFFFAAAAAAAAAAAAAAAAAAAAAAAAAAAACA
:10CC2000AAAAAAAAAAAAAAAAAAAAAAAABFFFFFFF50
:10CC3000FFFFFFFFFFFFFFFFFFFFFFFFFFFFFFFF04
:10CC4000FFFFFFFFFFFFFFFFFFFFFFFFFFFFFFFFF4
:10CC5000FFFFFFFFFFFFFFFFFFFFFFFFFFFFFFFFE4
:10CC6000FFFFFFFFFFFFFFFFFFFFFFFFFFFFFFFFD4
:10CC7000FFFFFFFFFFFFAAAAAAAAAAAAAAAAAAAA16
:10CC8000AAAAAAAAAAAAAAAAAAAAAAAAAAAAAAAA04
:10CC9000BFFFFFFFFFFFFFFFFFFFFFFFFFFFFFFFE4
:10CCA000FFFFFFFFFFFFFFFF00003FFFFFFFFFFF52
:10CCB000FFFFFFFFFFFFFFFFFFFFFFFFFFFFFFFF84
:10CCC000FF00003FFFFFFFFFFFFFFFFFFFF000033C
:10CCD000FFFFFFFFFFFFFFFFFFFFAAAAAAAAAAAA62
:10CCE000AAAAAAAAAAAAAAAAAAAAAAAAAAAAAAAAA4
:10CCF000AAAAAAAABFFFFFFFFFFFFFFFFFFFFFFFD8
:10CD0000C0000FFFFFFFFFFFFFFFFF000000000F4D
:10CD1000FFFFFFFFFFFFFFFFFFFFFFFFFFFFFFFF23
:10CD2000FFFFFFFF000000000FFFFFFFFFFFFFFFFF
:10CD3000F000000000FFFFFFFFFFFFFFFFFFAAAAB8
:10CD4000AAAAAAAAAAAAAAAAAAAAAAAAAAAAAAAA43
:10CD5000AAAAAAAAAAAAAAAABFFFFFFFFFFFFFFFCB
:10CD6000FFFFFFFFC0000FFFFFFFFFFFFFFFFF0000
:10CD70000000000FFFFFFFFFFFFFFFFFFFFFFFFFB0
:10CD8000FFFFFFFFFFFFFFFF000000000FFFFFFF9F
:10CD9000FFFFFFFFF000000000FFFFFFFFFFFFFFAE
:10CDA000FFFFAAAAAAAAAAAAAAAAAAAAAAAAAAAA39
:10CDB000AAAAAAAAAAAAAAAAAAAAAAAABFFFFFFFBF
:10CDC000FFFFFFFFFFFFFFFF00000FFFFFFFFFFF61
:10CDD000FFFFC00000000003FFFFFFFFFFFFFFFF9A
:10CDE000FFFFFFFFFFFFFFFFFFFFFFC0000000008E
:10CDF00003FFFFFFFFFFFFFC00000000003FFFFFFD
:10CE0000FFFFFFFFFFFFAAAAAAAAAAAAAAAAAAAA84
:10CE1000AAAAAAAAAAAAAAAAAAAAAAAAAAAAAAAA72
:10CE2000BFFFFFFFFFFFFFFFFFFFFFFF00000FFF40
:10CE3000FFFFFFFFFFFFC00000000003FFFFFFFF39
:10CE4000FFFFFFFFFFFFFFFFFFFFFFFFFFFFFFC031
:10CE50000000000003FFFFFFFFFFFFFC00000000D9
:10CE6000003FFFFFFFFFFFFFFFFFAAAAAAAAAAAA8F
:10CE7000AAAAAAAAAAAAAAAAAAAAAAAAAAAAAAAA12
:10CE8000AAAAAAAABFFFFFFFFFFFFFFFFFFFFFC085
:10CE900000000FFFFFFFFFFFFFFC0000000000008D
:10CEA0003FFFFFFFFFFFFFFFFFFFFFFFFFFFFFFF52
:10CEB000FFFFFC0000000000003FFFFFFFFFFFC07E
:10CEC000000000000003FFFFFFFFFFFFFFFFAAAA13
:10CED000AAAAAAAAAAAAAAAAAAAAAAAAAAAAAAAAB2
:10CEE000AAAAAAAAAAAAAAAABFFFFFFFFFFFFFFF3A
:10CEF000FFFFFFC000000FFFFFFFFFFFFFFC000070
:10CF0000000000003FFFFFFFFFFFFFFFFFFFFFFFED
:10CF1000FFFFFFFFFFFFFC0000000000003FFFFFDE
:10CF2000FFFFFFC0000000000003FFFFFFFFFFFF47
:10CF3000FFFFAAAAAAAAAAAAAAAAAAAAAAAAAAAAA7
:10CF4000AAAAAAAAAAAAAAAAAAAAAAAABFFFFFFF2D
:10CF5000FFFFFFFFFFFFF00000000FFFFFFFFFFFDD
:10CF6000FFF00000FFFF00000FFFFFFFFFFFFFFFCC
:10CF7000FFFFFFFFFFFFFFFFFFFFF00000FFFF00CD
:10CF8000000FFFFFFFFFFF00000FFFF00000FFFF9B
:10CF9000FFFFFFFFFFFFAAAAFFFFFFFFFFFFFFFF4B
:10CFA000FFFFFFFFFFFFFFFFFFFFFFFFFFFFEAAAFB
:10CFB000BFFFFFFFFFFFFFFFFFFC000000000FFFB0
:10CFC000FFFFFFFFFF00003FFFFFFC0000FFFFFF30
:10CFD000FFFFFFFFFFFFFFFFFFFFFFFFFFFF00005F
:10CFE0003FFFFFFC0000FFFFFFFFF00003FFFFFF1C
:10CFF000C0000FFFFFFFFFFFFFFFAAAAFFFFFFFF19
:10D00000FFFFFFFFFFFFFFFFFFFFFFFFFFFFFFFF30
:10D01000FFFFEAAABFFFFFFFFFFFFFFFFFFC0000CB
:10D0200000000FFFFFFFFFFFFF00003FFFFFFC00BE
:10D0300000FFFFFFFFFFFFFFFFFFFFFFFFFFFFFFFF
:10D04000FFFF00003FFFFFFC0000FFFFFFFFF000BD
:10D0500003FFFFFFC0000FFFFFFFFFFFFFFFAAAAB4
:10D06000FFFFFFFFFFFFFFFFFFFFFFFFFFFFFFFFD0
:10D07000FFFFFFFFFFFFEAAABFFFFFFFFFFFFFFF6A
:10D08000FFC00000C0000FFFFFFFFFFFFF0000FF19
:10D09000FFFFFF00000FFFFFFFFFFFFFFFFFFFFF8E
:10D0A000FFFFFFFFFFFF0000FFFFFFFF00000FFF7C
:10D0B000FFFFF0000FFFFFFFF00000FFFFFFFFFF8B
:10D0C000FFFFAAAAFFFFFFFFFFAAAAAAFFFFFFFF19
:10D0D000AAAAABFFFFFAAAAAFFFFEAAABFFFFFFFB7
:10D0E000FFFFFFFFFFC00000C0000FFFFFFFFFFFBB
:10D0F000FF0000FFFFFFFF00000FFFFFFFFFFFFF2C
:10D10000FFFFFFFFFFFFFFFFFFFF0000FFFFFFFF2D
:10D1100000000FFFFFFFF0000FFFFFFFF00000FF18
:10D12000FFFFFFFFFFFFAAAAFFFFFFFFFFAAAAAAB8
:10D13000FFFFFFFFAAAAABFFFFFAAAAAFFFFEAAA16
:10D14000BFFFFFFFFFFFFFFFF000000FC0000FFF5A
:10D15000FFFFFFFFFC000FFFFFFFFFF0000FFFFFCF
:10D16000FFFFFFFFFFFFFFFFFFFFFFFFFFFC000FC1
:10D17000FFFFFFFFF0000FFFFFFFC000FFFFFFFFFB
:10D18000FF0000FFFFFFFFFFFFFFAAAAFFFFFFFF57
:10D19000FAAAAAAAFFFFFFFFAAAAABFFFFFAAAAA50
:10D1A000FFFFEAAABFFFFFFFFFFFFFFFC00003FF73
:10D1B000C0000FFFFFFFFFFFFC000FFFFFFFFFF0AE
:10D1C0000003FFFFFFFFFFFFFFFFFFFFFFFFFFFF6A
:10D1D000FFFC000FFFFFFFFFF00003FFFFFFC00099
:10D1E000FFFFFFFFFF00003FFFFFFFFFFFFFAAAAB7
:10D1F000FFFFFFFFFAAAAAAAFFFFFFFFAAAAABFF41
:10D20000FFFAAAAAFFFFEAAABFFFFFFFFFFFFFFF87
:10D21000C00003FFC0000FFFFFFFFFFFFC000FFF78
:10D22000FFFFFFF00003FFFFFFFFFFFFFFFFFFFF18
:10D23000FFFFFFFFFFFC000FFFFFFFFFF00003FFFA
:10D24000FFFFC000FFFFFFFFFF00003FFFFFFFFFEA
:10D25000FFFFAAAAFFFFFFFFFAAAAAAAFFFFFFFF8C
:10D26000AAAAABFFFFFAAAAAFFFFEAAABFFFFFFF25
:10D27000FFFFFFFFF0000FFFC0000FFFFFFFFFFFEA
:10D28000C0003FFFFFFFFFFC0003FFFFFFFFFFFFAA
:10D29000FF00FFFFFFFFFFFFFFC0003FFFFFFFFF9B
:10D2A000FC0003FFFFFC0003FFFFFFFFFFC0003F88
:10D2B000FFFFFFFFFFFFAAAAFFFFFFFFFAAAAAAA2C
:10D2C000BFFFFFFFAAAAAAFFFFAAAAAAFFFFEAAA16
:10D2D000BFFFFFFFFFFFFFFFF0000FFFC0000FFFCA
:10D2E000FFFFFFFFC0003FFFFFFFFFFC0003FFFF4A
:10D2F000FFFFFFFFFF00FFFFFFFFFFFFFFC0003F3B
:10D30000FFFFFFFFFC0003FFFFFC0003FFFFFFFF29
:10D31000FFC0003FFFFFFFFFFFFFAAAAFFFFFFFFC5
:10D32000FAAAAAAABFFFFFFFAAAAAAFFFFAAAAAA4F
:10D33000FFFFEAAABFFFFFFFFFFFFFFFF003FFFFB2
:10D34000C0000FFFFFFFFFFFC0003FFFFFFFFFFC1C
:10D350000003FFFFFFFFFFFFC00003FFFFFFFFFF12
:10D36000FFC0003FFFFFFFFFFC0003FFFFFC0003C7
:10D37000FFFFFFFFFFC0003FFFFFFFFFFFFFAAAA65
:10D38000FFFFFFFFEAAAAAAABFFFFFFFAAAAAAFF00
:10D39000FFAAAAAAFFFFEAAABFFFFFFFFFFFFFFF46
:10D3A000F003FFFFC0000FFFFFFFFFFFC0003FFFC4
:10D3B000FFFFFFFC0003FFFFFFFFFFFFC00003FFB5
:10D3C000FFFFFFFFFFC0003FFFFFFFFFFC0003FF69
:10D3D000FFFC0003FFFFFFFFFFC0003FFFFFFFFF59
:10D3E000FFFFAAAAFFFFFFFFEAAAAAAABFFFFFFF4B
:10D3F000AAAAAAFFFFAAAAAAFFFFEAAABFFFFFFFE5
:10D40000FFFFFFFFFF3FFFFFC0000FFFFFFFFFFF1A
:10D41000C0003FFFFFFFFFF00003FFFFFFFFFFFF24
:10D42000C00003FFFFFFFFFFFFC0003FFFFFFFFF44
:10D43000F00003FFFFFC0003FFFFFFFFFF00003FC2
:10D44000FFFFFFFFFFFFAAAAFFFFFFFFEAAAFAAA5A
:10D45000BFFFFFFFAAAAAAFFFFAAAAAAFFFFEAAA84
:10D46000BFFFFFFFFFFFFFFFFFFFFFFFC0000FFF3A
:10D47000FFFFFFFF0003FFFFFFFFFF0000003FFF74
:10D48000FFFFFFFC0000003FFFFFFFFFFF0003FF67
:10D49000FFFFFFFF0000003FFFF0003FFFFFFFFF27
:10D4A000F0000003FFFFFFFFFFFFAAAAFFFFFFFF3F
:10D4B000EAAAFAAAABFFFFFFAAAAAAFFFFAAAAAA92
:10D4C000FFFFEAAABFFFFFFFFFFFFFFFFFFFFFFF16
:10D4D000C0000FFFFFFFFFFF0003FFFFFFFFFF0084
:10D4E00000003FFFFFFFFFFC0000003FFFFFFFFFCA
:10D4F000FF0003FFFFFFFFFF0000003FFFF0003FC2
:10D50000FFFFFFFFF0000003FFFFFFFFFFFFAAAADE
:10D51000FFFFFFFFEAAAFAAAABFFFFFFAAAAAAFF32
:10D52000FFAAAAAAFFFFEAAABFFFFFFFFFFFFFFFB4
:10D53000FFFFFFFFC0000FFFFFFFFFFF0003FFFF24
:10D54000FFFFFC0000003FFFFFFFFFFC0000003F6B
:10D55000FFFFFFFFFF0003FFFFFFFFFC0000003F96
:10D56000FFF0003FFFFFFFFFC0000003FFFFFFFFD2
:10D57000FFFFAAAAFFFFFFFEAAAAFAAAABFFFFFFBE
:10D58000AAAAAAAFFEAABAAAFFFFEAAABFFFFFFF94
:10D59000FFFFFFFFFFFFFFFFC0000FFFFFFFFFFFC9
:10D5A0000003FFFFFFFFFC0000003FFFFFFFFFFC49
:10D5B0000000003FFFFFFFFFFF0003FFFFFFFFFC36
:10D5C0000000003FFFF0003FFFFFFFFFC00000032F
:10D5D000FFFFFFFFFFFFAAAAFFFFFFFEAAAAFAAA0A
:10D5E000ABFFFFFFAAAAAAAFFEAABAAAFFFFEAAA48
:10D5F000BFFFFFFFFFFFFFFFFFFFFFFFC0000FFFA9
:10D60000FFFFFFFF0003FFFFFFFF000000003FFFE1
:10D61000FFFFFFFC0000003FFFFFFFFFFF0003FFD5
:10D62000FFFFFF000000003FFFF0003FFFFFFFF0A3
:10D6300000000003FFFFFFFFFFFFAAAAFFFFFFFE9E
:10D64000AAAAFAAAABFFFFFFAAAFAAAFFEAABAAA7C
:10D65000FFFFEAAABFFFFFFFFFFFFFFFFFFFFFFF84
:10D66000C0000FFFFFFFFFFF0003FFFFFFF0000000
:10D6700000003FFFFFFFFFFFC00003FFFFFFFFFFB2
:10D68000FF0003FFFFFFF0000000003FFFF0003F3E
:10D69000FFFFFF0000000003FFFFFFFFFFFFAAAA3C
:10D6A000FFFFFFFEAAABFEAAABFFFFFFAAAFAAAF28
:10D6B000FEAABAAAFFFFEAAABFFFFFFFFFFFFFFF14
:10D6C000FFFFFFFFC0000FFFFFFFFFFF0003FFFF93
:10D6D000FFF0000000003FFFFFFFFFFFC00003FF5F
:10D6E000FFFFFFFFFF0003FFFFFFF0000000003F10
:10D6F000FFF0003FFFFFFF0000000003FFFFFFFF00
:10D70000FFFFAAAAFFFFFFFEAAABFEAAABFFFFFF27
:10D71000AAAFAAAFFEAABAAAFFFFEAAABFFFFFFFFD
:10D72000FFFFFFFFFFFFFFFFC0000FFFFFFFFFFF37
:10D730000003FFFFFFC00003C0003FFFFFFFFFFF2C
:10D74000C00003FFFFFFFFFFFF0003FFFFFFC0005C
:10D7500003C0003FFFF0003FFFFFFC00003C000360
:10D76000FFFFFFFFFFFFAAAAFFFFFFFEAAABFEAA73
:10D77000AAFFFFFEAAAFAAAFFEABFAAAAFFFEAAAC2
:10D78000BFFFFFFFFFFFFFFFFFFFFFFFC0000FFF17
:10D79000FFFFFFFF0003FFFFFFC00003C0003FFFCC
:10D7A000FFFFFFFFC00003FFFFFFFFFFFF0003FFBE
:10D7B000FFFFC00003C0003FFFF0003FFFFFFC0081
:10D7C000003C0003FFFFFFFFFFFFAAAAFFFFFFFED1
:10D7D000AAABFEAAAAFFFFFEAAAFAAAFFEABFAAAA7
:10D7E000AFFFEAAABFFFFFFFFFFFFFFFFFFFFFFF43
:10D7F000C0000FFFFFFFFFFF0003FFFFF000000F5F
:10D80000C0003FFFFFFFFFFFFF00FFFFFFFFFFFF25
:10D81000FF0003FFFFF000000FC0003FFFF0003FDC
:10D82000FFFF000000FC0003FFFFFFFFFFFFAAAAAD
:10D83000FFFFFFFAAAABFEAAAAFFFFFEAAAFEAAA61
:10D84000EAABFAAAAFFFEAAABFFFFFFFFFFFFFFFA5
:10D85000FFFFFFFFC0000FFFFFFFFFFF0003FFFF01
:10D86000000000FFC0003FFFFFFFFFFFFFFFFFFFC3
:10D87000FFFFFFFFFF0003FFFF000000FFC0003FAE
:10D88000FFF0003FFFF000000FFC0003FFFFFFFF71
:10D89000FFFFAAAAFFFFFFFAAABFFEAAAAFFFFFE88
:10D8A000AAAFEAAAEAABFAAAAFFFEAAABFFFFFFF54
:10D8B000FFFFFFFFFFFFFFFFC0000FFFFFFFFFFFA6
:10D8C0000003FFFF000000FFC0003FFFFFFFFFFF5E
:10D8D000FFFFFFFFFFFFFFFFFF0003FFFF00000050
:10D8E000FFC0003FFFF0003FFFF000000FFC00030F
:10D8F000FFFFFFFFFFFFAAAAFFFFFFFAAABFFEAAD2
:10D90000AAFFFFFEAAAFEAAAEAABFAAAAFFFEAAA09
:10D91000BFFFFFFFFFFFFFFFFFFFFFFFC0000FFF85
:10D92000FFFFFFFF0003FFFC00003FFFC0003FFFC1
:10D93000FFFFFFFFFFFFFFFFFFFFFFFFFF0003FFF2
:10D94000FC00003FFFC0003FFFF0003FFFC00003AE
:10D95000FFFC0003FFFFFFFFFFFFAAAAFFFFFFFA84
:10D96000AABFFFEAAAAFFFFEAAAFEAAAEAAFFAAAE5
:10D97000AFFFEAAABFFFFFFFFFFFFFFFFFFFFFFFB1
:10D98000C0000FFFFFFFFFFF0003FFFC00003FFF91
:10D99000C0003FFFFFFFFFFFFFFFFFFFFFFFFFFF95
:10D9A000FF0003FFFC00003FFFC0003FFFF0003F0F
:10D9B000FFC00003FFFC0003FFFFFFFFFFFFAAAA59
:10D9C000FFFFFFFAAABFFFEAAAAFFFFEAAAFEAAACB
:10D9D000EAAFFAAAAFFFEAAABFFFFFFFFFFFFFFF10
:10D9E000FFFFFFFFC0000FFFFFFFFFFF0003FF006F
:10D9F0000000FFFFC0003FFFFFFFFFFFFFFFFFFF33
:10DA0000FFFFFFFFFF0003FF000000FFFFC0003F1C
:10DA1000FFF0003FF000000FFFFC0003FFFFFFFFDF
:10DA2000FFFFAAAAFFFFFFAAAABFFFEAAAAFFFFE55
:10DA3000AAAFEAAAEAAFFAAAAFFFEAAABFFFFFFFBE
:10DA4000FFFFFFFFFFFFFFFFC0000FFFFFFFFFFF14
:10DA50000003FF000000FFFFC0003FFFFFFFFFFFCC
:10DA6000FFFFFFFFFFFFFFFFFF0003FF000000FFBE
:10DA7000FFC0003FFFF0003FF000000FFFFC00037D
:10DA8000FFFFFFFFFFFFAAAAFFFFFFAAAABFFFEA4F
:10DA9000AAAFFFFEAAAFEAAAEAAFFAAAAFFFEAAAC4
:10DAA000BFFFFFFFFFFFFFFFFFFFFFFFC0000FFFF4
:10DAB000FFFFFFFF0003F000000FFFFFC0003FFF6C
:10DAC000FFFFFFFFFFFFFFFFFFFFFFFFFF0003F070
:10DAD00000000FFFFFC0003FFFF0003F000000FF0D
:10DAE000FFFC0003FFFFFFFFFFFFAAAAFFFFFFAA43
:10DAF000AABFFFEAAAAFFFFEAAAFFEAAAAAFFAAA80
:10DB0000AFFFEAAABFFFFFFFFFFFFFFFFFFFFFFF1F
:10DB1000C0000FFFFFFFFFFF0000000003FFFFFF3B
:10DB2000C0003FFFFFFFFFFFFFFFFFFFFFFFFFFF03
:10DB3000FF0000000003FFFFFFC0003FFFF00000F8
:10DB400000003FFFFFFC0003FFFFFFFFFFFFAAAA4B
:10DB5000FFFFFFAAAAFFFFEAAAAFFFFEAAAFFEAA35
:10DB6000AAAFFAAAAFFFEAAABFFFFFFFFFFFFFFFBE
:10DB7000FFFFFFFFC0000FFFFFFFFFFF00000000DF
:10DB800003FFFFFFC0003FFFFFFFFFFFFFFFFFFF9F
:10DB9000FFFFFFFFFF0000000003FFFFFFC0003F8B
:10DBA000FFF0000000003FFFFFFC0003FFFFFFFF4E
:10DBB000FFFFAAAAFFFFFFAAAAFFFFEAAAAFFFFE84
:10DBC000AAAFFEAAAAAFFAAAAFFFEAAABFFFFFFF59
:10DBD000FFFFFFFFFFFFFFFFC0000FFFFFFFFFFF83
:10DBE000000000000FFFFFFFC0003FFFFFFFFFFF2F
:10DBF000FFFFFFFFFFFFFFFFFF000000000FFFFF21
:10DC0000FFC0003FFFF000000000FFFFFFFC00032B
:10DC1000FFFFFFFFFFFFAAAAFFFFFFAAAAFFFFFA6D
:10DC2000AAABFFFEAAAFFEAAAAFFFAAAAFFFEAAA12
:10DC3000BFFFFFFFFFFFFFFFFFFFFFFFC0000FFF62
:10DC4000FFFFFFFF000000000FFFFFFFC0003FFFCE
:10DC5000FFFFFFFFFFFFFFFFFFFFFFFFFF000000D1
:10DC6000000FFFFFFFC0003FFFF000000000FFFFBC
:10DC7000FFFC0003FFFFFFFFFFFFAAAAFFFFFFAAB1
:10DC8000AAFFFFFAAAABFFFEAAAFFEAAAAFFFAAA52
:10DC9000AFFFEAAABFFFFFFFFFFFFFFFFFFFFFFF8E
:10DCA000C0000FFFFFFFFFFF00000003FFFFFFFFAB
:10DCB000C0003FFFFFFFFFFFFFFFFFFFFFFFFFFF72
:10DCC000FF00000003FFFFFFFFC0003FFFF0000068
:10DCD000003FFFFFFFFC0003FFFFFFFFFFFFAAAABB
:10DCE000FFFFFAAAAAFFFFFAAAABFFFEAAAFFEAA9D
:10DCF000AAFFFAAAAFFFEAAABFFFFFFFFFFFFFFFDD
:10DD0000FFFFFFFFC0000FFFFFFFFFFF0000003F0E
:10DD1000FFFFFFFFC0003FFFFFFFFFFFFFFFFFFF11
:10DD2000FFFFFFFFFF0000003FFFFFFFFFC0003FBE
:10DD3000FFF0000003FFFFFFFFFC0003FFFFFFFFFA
:10DD4000FFFFAAAAFFFFFAAAAFFFFFFAAAABFFFEE6
:10DD5000AAAFFFAAAAFFFAAAAFFFEAAABFFFFFFF76
:10DD6000FFFFFFFFFFFFFFFFC0000FFFFFFFFFFFF1
:10DD70000000003FFFFFFFFFC0003FFFFFFFFFFF6E
:10DD8000FFFFFFFFFFFFFFFFFF0000003FFFFFFF60
:10DD9000FFC0003FFFF0000003FFFFFFFFFC000398
:10DDA000FFFFFFFFFFFFAAAAFFFFFAAAAFFFFFFADC
:10DDB000AAABFFFEAAAFFFAAAAFFFAAAAFFFEAAA80
:10DDC000BFFFFFFFFFFFFFFFFFFFFFFFC0000FFFD1
:10DDD000FFFFFFFF000000FFFFFFFFFFC0003FFF4E
:10DDE000FFFFFFFFFFFFFFFFFFFFFFFFFF00000040
:10DDF000FFFFFFFFFFC0003FFFF000000FFFFFFF2E
:10DE0000FFFC0003FFFFFFFFFFFFAAAAFFFFFAAA24
:10DE1000AAAAAAAAAAAABFFEAAAFFFAAABFFFAAAF9
:10DE2000AFFFEAAABFFFFFFFFFFFFFFFFFFFFFFFFC
:10DE3000C0000FFFFFFFFFFF000000FFFFFFFFFF1D
:10DE4000C0003FFFFFFFFFFFFFFFFFFFFFFFFFFFE0
:10DE5000FF000000FFFFFFFFFFC0003FFFF00000DA
:10DE60000FFFFFFFFFFC0003FFFFFFFFFFFFAAAA5A
:10DE7000FFFFFAAAAAAAAAAAAAAABFFEAAAFFFAA45
:10DE8000ABFFFAAAAFFFEAAABFFFFFFFFFFFFFFF4A
:10DE9000FFFFFFFFC0000FFFFFFFFFFF00003FFF7E
:10DEA000FFFFFFFFC0003FFFFFFFFFFFFFFFFFFF80
:10DEB000FFFFFFFFFF00003FFFFFFFFFFFC0003F2E
:10DEC000FFF00003FFFFFFFFFFFC0003FFFFFFFF6A
:10DED000FFFFAAAAFFFFEAAAAAAAAAAAAAAABFFEA5
:10DEE000AAAFFFAAABFFFAAAAFFFEAAABFFFFFFFE4
:10DEF000FFFFFFFFFFFFFFFFC0000FFFFFFFFFFF60
:10DF000000003FFFFFFFFFFFC0003FFFFFFFFFFFDD
:10DF1000FFFFFFFFFFFFFFFFFF00003FFFFFFFFFCF
:10DF2000FFC0003FFFF00003FFFFFFFFFFFC000307
:10DF3000FFFFFFFFFFFFAAAAFFFFEAAAAAAAAAAA59
:10DF4000AAAABFFEAAAFFFAAABFFFAAAAFFFEAAA2E
:10DF5000BFFFFFFFFFFFFFFFFFFFFFFFC0000FFF3F
:10DF6000FFFFFFFFC0003FFFFFFFFFFC0003FFFFBD
:10DF7000FFFFFFFFFFFFFFFFFFFFFFFFFFC0003FAF
:10DF8000FFFFFFFFFC0003FFFFFC0003FFFFFFFF9D
:10DF9000FFC0003FFFFFFFFFFFFFAAAAFFFFEAAAA3
:10DFA000AAAAAAAAAAAABFFEAAAFFFFFFFFFFAAABF
:10DFB000AFFFEAAABFFFFFFFFFFFFFFFFFFFFFFF6B
:10DFC000C0000FFFFFFFFFFFC0003FFFFFFFFFFC90
:10DFD0000003FFFFFFFFFFFFFFFFFFFFFFFFFFFF4C
:10DFE000FFC0003FFFFFFFFFFC0003FFFFFC00033B
:10DFF000FFFFFFFFFFC0003FFFFFFFFFFFFFAAAAD9
:10E00000FFFFEAAAAAAAAAAAAAAABFFEAAAFFFFF6E
:10E01000FFFFFAAAAFFFEAAABFFFFFFFFFFFFFFF64
:10E02000FFFFFFFFC0000FFFFFFFFFFFC0003FFF2C
:10E03000FFFFFFFC0003FFFFFFFFFFFFFFFFFFFFEE
:10E04000FFFFFFFFFFC0003FFFFFFFFFFC0003FFDC
:10E05000FFFC0003FFFFFFFFFFC0003FFFFFFFFFCC
:10E06000FFFFAAAAFFFFEAAAAAAAAAAAAAAABFFE13
:10E07000AAAFFFFFFFFFFAAAAFFFEAAABFFFFFFFA9
:10E08000FFFFFFFFFFFFFFFFC0000FFFFFFFFFFFCE
:10E09000C0003FFFFFFFFFFC0003FFFFFFFFFFFF8C
:10E0A000FFFFFFFFFFFFFFFFFFC0003FFFFFFFFF7E
:10E0B000FC0003FFFFFC0003FFFFFFFFFFC0003F6A
:10E0C000FFFFFFFFFFFFAAAAFFFEAAAAAAAAAAAA09
:10E0D000AAAAAFFEAAAFFFFFFFFFFAAAAFFFEAAA04
:10E0E000BFFFFFFFFFFFFFFFFFFFFFFFC0000FFFAE
:10E0F000FFFFFFFFC0003FFFFFFFFFFC0003FFFF2C
:10E10000FFFFFFFFFFFFFFFFFFFFFFFFFFC0003F1D
:10E11000FFFFFFFFFC0003FFFFFC0003FFFFFFFF0B
:10E12000FFC0003FFFFFFFFFFFFFAAAAFFFEAAAA52
:10E13000AAAAAAAAAAAAAFFEAAAFFFFFFFFFFAAA3D
:10E14000AFFFEAAABFFFFFFFFFFFFFFFFFFFFFFFD9
:10E15000C0000FFFFFFFFFFFC0000FFFFFFFFFF03A
:10E16000000FFFFFFFFFFFFFFF00FFFFFFFFFFFFAD
:10E17000FFC0000FFFFFFFFFF0000FFFFFFC0000DC
:10E18000FFFFFFFFFF0000FFFFFFFFFFFFFFAAAA47
:10E19000FFFEAAAABFFFFFFFEAAAAFFEAAAFFFFFDA
:10E1A000FFFFFAAAAFFFEAAABFFFFFFFFFFFFFFFD3
:10E1B000FFFFFFFFC0000FFFFFFFFFFFFC0000FF9E
:10E1C000FFFFFFF0000FFFFFFFFFFFFFC00003FF97
:10E1D000FFFFFFFFFFFC0000FFFFFFFFF0000FFF4E
:10E1E000FFFFC0000FFFFFFFFF0000FFFFFFFFFF6B
:10E1F000FFFFAAAAFFFEAAABFFFFFFFFEAAAAFFE3E
:10E20000AAAFFFFFFFFFFAAAAFFFEAAABFFFFFFF17
:10E21000FFFFFFFFFFFFFFFFC0000FFFFFFFFFFF3C
:10E22000FC0000FFFFFFFFF0000FFFFFFFFFFFFFFD
:10E23000C00003FFFFFFFFFFFFFC0000FFFFFFFF29
:10E24000F0000FFFFFFFC0000FFFFFFFFF0000FF08
:10E25000FFFFFFFFFFFFAAAAFFFEAAABFFFFFFFF22
:10E26000EAAAAFFEAAAFFFFFFFFFFAAAAFFFEAAA32
:10E27000BFFFFFFFFFFFFFFFFFFFFFFFC0000FFF1C
:10E28000FFFFFFFFFC0000FFFFFFFF0000FFFFFF9D
:10E29000FFFFFFFFC00003FFFFFFFFFFFFFC0000C9
:10E2A000FFFFFFFF0000FFFFFFFFC0000FFFFFFFAA
:10E2B000F0000FFFFFFFFFFFFFFFAAAAFFFEAAABC0
:10E2C000FFFFFFFFEAAAAAFEAABFFFFFFFFFFAAA0D
:10E2D000AFFFEAAABFFFFFFFFFFFFFFFFFFFFFFF48
:10E2E000C0000FFFFFFFFFFFFC0000FFFFFFFF006C
:10E2F00000FFFFFFFFFFFFFFC00003FFFFFFFFFF67
:10E30000FFFC0000FFFFFFFF0000FFFFFFFFC0005A
:10E310000FFFFFFFF0000FFFFFFFFFFFFFFFAAAAA5
:10E32000FFFEAAABFFFFFFFFEAAAAAFEAABFFFFFFC
:10E33000FFFFFAAAAFFFEAAABFFFFFFFFFFFFFFF41
:10E34000F0000000000000000003FFFFFF00003F9E
:10E35000FFFFFC0000FFFFFFFFFFFFFC0000003F8E
:10E36000FFFFFFFFFFFF00003FFFFFFC0000FFFF7C
:10E37000FFFFF00003FFFFFFC0000FFFFFFFFFFFE5
:10E38000FFFFAAAAFFFAAAABFFFFFFFFEAAAAAFEB5
:10E39000AABFFFFFFFFFFAAAAFFFEAAABFFFFFFF76
:10E3A000FFFFFFFFF0000000000000000003FFFF80
:10E3B000FFF00000FFFF00000FFFFFFFFFFFFFFC6B
:10E3C0000000003FFFFFFFFFFFFFF00000FFFF0026
:10E3D000000FFFFFFFFFFF00000FFFF00000FFFF37
:10E3E000FFFFFFFFFFFFAAAAFFFAAAABFFFFFFFF95
:10E3F000FEAAAAFEAABFFFFFFFFFFAAAAFFFEAAA82
:10E40000BFFFFFFFFFFFFFFFF00000000000000064
:10E410000003FFFFFFF00000FFFF00000FFFFFFF02
:10E42000FFFFFFFC0000003FFFFFFFFFFFFFF000CA
:10E4300000FFFF00000FFFFFFFFFFF00000FFFF0D6
:10E440000000FFFFFFFFFFFFFFFFAAAAFFFAAAAB32
:10E45000FFFFFFFFFEAAAAFEAABFFFFFFFFFFAAA67
:10E46000AFFFEAAABFFFFFFFFFFFFFFFF0000000C2
:10E47000000000000003FFFFFFF0000000000000AC
:10E480003FFFFFFFFFFFFFFC0000003FFFFFFFFF1C
:10E49000FFFFF00000000000003FFFFFFFFFFF0054
:10E4A000000000000003FFFFFFFFFFFFFFFFAAAA1D
:10E4B000FFFAAAAFFFFFFFFFFEAAAAFEAABFFFFF57
:10E4C000FFFFFAAAAFFFEAAABFFFFFFFFFFFFFFFB0
:10E4D000F0000000000000000003FFFFFFF000005C
:10E4E000000000003FFFFFFFFFFFFFFC0000003FB8
:10E4F000FFFFFFFFFFFFF00000000000003FFFFFF5
:10E50000FFFFFF00000000000003FFFFFFFFFFFF11
:10E51000FFFFAAAAFFFAAAAFFFFFFFFFFEAAAAFE0B
:10E52000AABFFFFFFFFFFAAAAFFFEAAABFFFFFFFE4
:10E53000FFFFFFFFF0000000000000000003FFFFEE
:10E54000FFFFC00000000003FFFFFFFFFFFFFFFF12
:10E55000C00003FFFFFFFFFFFFFFFFC00000000040
:10E5600003FFFFFFFFFFFFFC00000000003FFFFF75
:10E57000FFFFFFFFFFFFAAAAFFFFFFFFFFFFFFFF55
:10E58000FFFFFFFFFFFFFFFFFFFFFFFFFFFFEAAA05
:10E59000BFFFFFFFFFFFFFFFF000000000000000D3
:10E5A0000003FFFFFFFFC00000000003FFFFFFFFAD
:10E5B000FFFFFFFFC00003FFFFFFFFFFFFFFFFC0E4
:10E5C0000000000003FFFFFFFFFFFFFC0000000052
:10E5D000003FFFFFFFFFFFFFFFFFAAAAFFFFFFFFB4
:10E5E000FFFFFFFFFFFFFFFFFFFFFFFFFFFFFFFF3B
:10E5F000FFFFEAAABFFFFFFFFFFFFFFFF0000000E1
:10E60000000000000003FFFFFFFFF000000000FF1C
:10E61000FFFFFFFFFFFFFFFFC00003FFFFFFFFFF44
:10E62000FFFFFFF000000000FFFFFFFFFFFFFFFF05
:10E63000000000000FFFFFFFFFFFFFFFFFFFAAAA80
:10E64000FFFFFFFFFFFFFFFFFFFFFFFFFFFFFFFFDA
:10E65000FFFFFFFFFFFFEAAABFFFFFFFFFFFFFFF74
:10E66000FFFFFFFFFFFFFFFFFFFFFFFFFFFFFFFCBD
:10E670000000FFFFFFFFFFFFFFFFFFFFFF00FFFFA7
:10E68000FFFFFFFFFFFFFFFFFC0000FFFFFFFFFF9B
:10E69000FFFFFFFFFFC0000FFFFFFFFFFFFFFFFFB8
:10E6A000FFFFAAAAAAAAAAAAAAAAAAAAAAAAAAAA20
:10E6B000AAAAAAAAAAAAAAAAAAAAAAAABFFFFFFFA6
:10E6C000FFFFFFFFFFFFFFFFFFFFFFFFFFFFFFFF5A
:10E6D000FFFFFFFC0000FFFFFFFFFFFFFFFFFFFF4B
:10E6E000FF00FFFFFFFFFFFFFFFFFFFFFC0000FF3A
:10E6F000FFFFFFFFFFFFFFFFFFC0000FFFFFFFFF58
:10E70000FFFFFFFFFFFFAAAAAAAAAAAAAAAAAAAA6B
:10E71000AAAAAAAAAAAAAAAAAAAAAAAAAAAAAAAA59
:10E72000BFFFFFFFFFFFFFFFFFFFFFFFFFFFFFFF39
:10E73000FFFFFFFFFFFFFFFFFFFFFFFFFFFFFFFFE9
:10E74000FFFFFFFFFFFFFFFFFFFFFFFFFFFFFFFFD9
:10E75000FFFFFFFFFFFFFFFFFFFFFFFFFFFFFFFFC9
:10E76000FFFFFFFFFFFFFFFFFFFFAAAAAAAAAAAAB7
:10E77000AAAAAAAAAAAAAAAAAAAAAAAAAAAAAAAAF9
:10E78000AAAAAAAABFFFFFFFFFFFFFFFFFFFFFFF2D
:10E79000FFFFFFFFFFFFFFFFFFFFFFFFFFFFFFFF89
:10E7A000FFFFFFFFFFFFFFFFFFFFFFFFFFFFFFFF79
:10E7B000FFFFFFFFFFFFFFFFFFFFFFFFFFFFFFFF69
:10E7C000FFFFFFFFFFFFFFFFFFFFFFFFFFFFAAAA03
:10E7D000AAAAAAAAAAAAAAAAAAAAAAAAAAAAAAAA99
:10E7E000AAAAAAAAAAAAAAAABFFFFFFFFFFFFFFF21
:10E7F000FFFFFFFFFFFFFFFFFFFFFFFFFFFFFFFF29
:10E80000FFFFFFFFFFFFFFFFFFFFFFFFFFFFFFFF18
:10E81000FFFFFFFFFFFFFFFFFFFFFFFFFFFFFFFF08
:10E82000FFFFFFFFFFFFFFFFFFFFFFFFFFFFFFFFF8
:10E83000FFFFAAAAAAAAAAAAAAAAAAAAAAAAAAAA8E
:10E84000AAAAAAAAAAAAAAAAAAAAAAAABFFFFFFF14
:10E85000FFFFFFFFFFFFFFFFFFFFFFFFFFFFFFFFC8
:10E86000FFFFFFFFFFFFFFFFFFFFFFFFFFFFFFFFB8
:10E87000FFFFFFFFFFFFFFFFFFFFFFFFFFFFFFFFA8
:10E88000FFFFFFFFFFFFFFFFFFFFFFFFFFFFFFFF98
:10E89000FFFFFFFFFFFFAAAAAAAAAAAAAAAAAAAADA
:10E8A000AAAAAAAAAAAAAAAAAAAAAAAAAAAAAAAAC8
:10E8B000BFFFFFFFFFFFFFFFFFFFFFFFFFFFFFFFA8
:10E8C000FFFFFFFFFFFFFFFFFFFFFFFFFFFFFFFF58
:10E8D000FFFFFFFFFFFFFFFFFFFFFFFFFFFFFFFF48
:10E8E000FFFFFFFFFFFFFFFFFFFFFFFFFFFFFFFF38
:10E8F000FFFFFFFFFFFFFFFFFFFFAAAAAAAAAAAA26
:10E90000AAAAAAAAAAAAAAAAAAAAAAAAAAAAAAAA67
:10E91000AAAAAAAABFFFFFFFFFFFFFFFFFFFFFFF9B
:10E92000FFFFFFFFFFFFFFFFFFFFFFFFFFFFFFFFF7
:10E93000FFFFFFFFFFFFFFFFFFFFFFFFFFFFFFFFE7
:10E94000FFFFFFFFFFFFFFFFFFFFFFFFFFFFFFFFD7
:10E95000FFFFFFFFFFFFFFFFFFFFFFFFFFFFAAAA71
:10E96000AAAAAAAAAAAAAAAAAAAAAAAAAAAAAAAA07
:10E97000AAAAAAAAAAAAAAAABFFFFFFFFFFFFFFF8F
:10E98000FFFFFFFFFFFFFFFFFFFFFFFFFFFFFFFF97
:10E99000FFFFFFFFFFFFFFFFFFFFFFFFFFFFFFFF87
:10E9A000FFFFFFFFFFFFFFFFFFFFFFFFFFFFFFFF77
:10E9B000FFFFFFFFFFFFFFFFFFFFFFFFFFFFFFFF67
:10E9C000FFFFAAAAAAAAAAAAAAAAAAAAAAAAAAAAFD
:10E9D000AAAAAAAAAAAAAAAAAAAAAAAABFFFFFFF83
:10E9E000FFFFFFFFFFFFFFFFFFFFFFFFFFFFFFFF37
:10E9F000FFFFFFFFFFFFFFFFFFFFFFFFFFFFFFFF27
:10EA0000FFFFFFFFFFFFFFFFFFFFFFFFFFFFFFFF16
:10EA1000FFFFFFFFFFFFFFFFFFFFFFFFFFFFFFFF06
:10EFB000000000000000000000000000AAAAAAAAA9
:10EFC000AAAAAAAAAAAAAAAAAAAAAAAAAAAAAAAAA1
:10EFD000AAAAAAAAAAAAAAAAAAAAAAAAAAAAAAAA91
:10EFE000AAAAAAAAAAAAAAAAAAAAAAAAAAAAAAAA81
:10EFF000AAAAAAAAAAAAAAAAAAAAAAAAAAAAAAAA71
:10F5E000AAAAA00AAAAAAAAAAAAAAAAAAAAAAAAA25
:10F5F000AAAAAAAAAAAAAAAAAAAAAAAAAAAAAAAA6B
:10F60000AAAAAAAAAAAAAAAAAAAAAAAAAAAAAAAA5A
:10F61000AAAAAAAAAAAAAAAAAAAAAAAAAAAAAAAA4A
:10F62000AAAAAAAAAAAAAAAAAAAAAAAAAAAAAAAA3A
:10F63000AAAAAAAAAAAAAAAAAAAAAAAAAAAAAAAA2A
:10F64000AAAAAAAAAAAAA00AAAAAAAAAAAAAAAAAC4
:10F65000AAAAAAAAAAAAAAAAAAAAAAAAAAAAAAAA0A
:10F66000AAAAAAAAAAAAAAAAAAAAAAAAAAAAAAAAFA
:10F67000AAAAAAAA000AAAAAAAAAAAAAAAAAAAAA34
:10F68000AAAAAAAAAAAAAAAAAAAAAAAA00AAAAAA84
:10F69000AAAA0000AAAAAAAAAAAAAA02AAAAAAA8C8
:10F6A0000AAAAAAAAAAAAAAAAAAAA00AAAAAAAAA04
:10F6B000AAAAAAAAAAAAAAAAAAAAAAAAAAAAAAAAAA
:10F6C000AAAAAAAAAAAAAAAAAAAAAAAAAAAAAAAA9A
:10F6D000AAAAAAAAAAAAAAAA000AAAAAAAAAAAAAD4
:10F6E000AAAAAAAAAAAAAAAAAAAAAAAAAAAAAAAA7A
:10F6F00000AAAAAAAAAA0000AAAAAAAAAAAAAA0210
:10F70000AAAAAAA80AAAAAAAAAAAAAAAAAAAA00AA5
:10F71000AAAAAAAAAAAAAAAAAAAAAAAAAAAAAAAA49
:10F72000AAAAAAAAAAAAAAAAAAAAAAAAAAAAAAAA39
:10F73000AAAAAAAAAAAAAAAAAAAAAAAA000AAAAA73
:10F74000AAAAAAAAAAAAAAAAAAAAAAAAAAAAAAAA19
:10F75000AAAAAA8000AAAAAAAA800000AAAAAAAA5B
:10F76000AAAAAA02AAAAAAA80AAAAAAAAAAAAAAA43
:10F77000AAAAA00AAAAAAAAAAAAAAAAAAAAAAAAA93
:10F78000AAAAAAAAAAAAAAAAAAAAAAAAAAAAAAAAD9
:10F79000AAAAAAAAAAAAAAAAAAAAAAAAAAAAAAAAC9
:10F7A000000AAAAAAAAAAAAAAAAAAAAAAAAAAAAA03
:10F7B000AAAAAAAAAAAAAA8000AAAAAAAA800000FB
:10F7C000AAAAAAAAAAAAAA02AAAAAAA80AAAAAAAE3
:10F7D000AAAAAAAAAAAAA00AAAAAAAAAAAAAAAAA33
:10F7E000AAAAAAAAAAAAAAAAAAAAAAAAAAAAAAAA79
:10F7F000AAAAAAAAAAAAAAAAAAAAAAAAAAAAAAAA69
:10F80000AAAAAAAA0000AAAAAAAAAAAAAAAAAAAAAC
:10F81000AAAAAAAAAAAAAAAAAAAAA00A00AAAAAA9C
:10F82000A800AAAAAAAAAAAAAAAAAA002AAAAAA810
:10F830000AAAAAAAAAAAAAAAAAAAA00AAAAAAAAA72
:10F84000AAAAAAAAAAAAAAAAAAAAAAAAAAAAAAAA18
:10F85000AAAAAAAAAAAAAAAAAAAAAAAAAAAAAAAA08
:10F86000AAAAAAAAAAAAAAA80280AAAAAAAAAAAACC
:10F87000AAAAAAAAAAAAAAAAAAAAAAAAAAAA002A12
:10F8800000AAAAAAA02AAAAAAAAAAAAAAAAAAA00B6
:10F890002AAAAAA80AAAAAAAAAAAAAAAAAAAA00A94
:10F8A000AAAAAAAAAAAAAAAAAAAAAAAAAAAAAAAAB8
:10F8B000AAAAAAAAAAAAAAAAAAAAAAAAAAAAAAAAA8
:10F8C000AAAAAAAAAAAAAAAAAAAAAAA80280AAAA6C
:10F8D000AAAAAAAAAAAAAAAAAAAAAAAAAAAAAAAA88
:10F8E000AAAA002A00AAAAAAA02AAAAAAAAAAAAAD6
:10F8F000AAAAAA002AAAAAA80AAAAAAAAAAAAAAA34
:10F90000AAAAA00AAAAAAAAAAAAAAAAAAAAAAAAA01
:10F91000AAAAAAAAAAAAAAAAAAAAAAAAAAAAAAAA47
:10F92000AAAAAAAAAAAAAAAAAAAAAAAAAAAAAAA839
:10F930000A80AAAAA00AAAAA02AAAAA80000002AC3
:10F94000AAAAAAAAAAAAAAAA00AAAAAA002AAAAAEB
:10F95000AAAAAAAAAAAAAA002AAAAAA80AAAA8007F
:10F960000AAAAAAAA800000AAAAAAAAAAAAAAAAA8D
:10F97000AAAAAAAAAAAAAAAAAAAAAAAAAAAAAAAAE7
:10F98000AAAAAAAAAAAAAAAAAAAAAAAAAAAAAAAAD7
:10F99000AAAAAAA80A80AAAAA00AAAAA02AAAAA8E7
:10F9A0000000002AAAAAAAAAAAAAAAAA00AAAAAADF
:10F9B000002AAAAAAAAAAAAAAAAAAA002AAAAAA8FD
:10F9C0000AAAA8000AAAAAAAA800000AAAAAAAAA79
:10F9D000AAAAAAAAAAAAAAAAAAAAAAAAAAAAAAAA87
:10F9E000AAAAAAAAAAAAAAAAAAAAAAAAAAAAAAAA77
:10F9F000AAAAAAAAAAAAAAA80A802AAAA00AAAAA5D
:10FA000002AAAA000000002AAAAAAAAAAAAAAAAA26
:10FA100000AAAAAA02AAAAAAAAAAAAAAAAAAAAA0A2
:10FA20002AAAAAA80AAA000000AAAAAA0000000AF4
:10FA3000AAAAAAAAAAAAAAAAAAAAAAAAAAAAAAAA26
:10FA4000AAAAAAAAAAAAAAAAAAAAAAAAAAAAAAAA16
:10FA5000AAAAAAAAAAAAAAAAAAAAAA800AA02AAA5A
:10FA6000A00AAAAA02AAA802AA800AAAAAAAAAAABC
:10FA7000AAAAAAAA00AAAAAA02AAAAAAAAAAAAAA38
:10FA8000AAAAAAA02A80AAA80AA002AA802AAAA092
:10FA900002AA800AAAAAAAAAAAAAAAAAAAAAAAAA38
:10FAA000AAAAAAAAAAAAAAAAAAAAAAAAAAAAAAAAB6
:10FAB000AAAAAAAAAAAAAAAAAAAAAAAAAAAAAA80D0
:10FAC0000AA02AAAA00AAAAA02AAA802AA800AAA86
:10FAD000AAAAAAAAAAAAAAAA00AAAAAA02AAAAAAD8
:10FAE000AAAAAAAAAAAAAAA02A80AAA80AA002AA7E
:10FAF000802AAAA002AA800AAAAAAAAAAAAAAAAA8C
:10FB0000AAAAAAAAAAAAAAAAAAAAAAAAAAAAAAAA55
:10FB1000AAAAAAAAAAAAAAAAAAAAAAAAAAAAAAAA45
:10FB2000AAAAAA80AAA02AAAA00AAAAA02AAA80ADD
:10FB3000AAA80AAAAAAAAAAAAAAAAAAA00AAAAA873
:10FB40000280002AAAAAAAAAAAAAAAA02A80AAA8C7
:10FB50000AA02AAAA002AA802AAAA00AAAAAAAAA35
:10FB6000AAAAAAAAAAAAAAAAAAAAAAAAAAAAAAAAF5
:10FB7000AAAAAAAAAAAAAAAAAAAAAAAAAAAAAAAAE5
:10FB8000AAAAAAAAAAAAAA80AAA02AAAA00AAAAA33
:10FB900002AAA80AAAA80AAAAAAAAAAAAAAAAAAAB1
:10FBA00000AAAAA80280002AAAAAAAAAAAAAAAA067
:10FBB0002A80AAA80AA02AAAA002AA802AAAA00A81
:10FBC000AAAAAAAAAAAAAAAAAAAAAAAAAAAAAAAA95
:10FBD000AAAAAAAAAAAAAAAAAAAAAAAAAAAAAAAA85
:10FBE000AAAAAAAAAAAAAAAAAAAAAA80AAA002AA51
:10FBF000A00AAAAA02AAA80AAAA80AAAAAAAAAAAFB
:10FC0000AAAAAAAA00AAAAA800000000AAAAAAAAA8
:10FC1000AAAAAAA02A800AA80A802AAAAA02AA80B6
:10FC2000AAAAA00AAAAAAAAAAAAAAAAAAAAAAAAADE
:10FC3000AAAAAAAAAAAAAAAAAAAAAAAAAAAAAAAA24
:10FC4000AAAAAAAAAAAAAAAAAAAAAAAAAAAAAA803E
:10FC5000AAA002AAA00AAAAA02AAA80AAAA80AAA4C
:10FC6000AAAAAAAAAAAAAAAA00AAAAA80000000048
:10FC7000AAAAAAAAAAAAAAA02A800AA80A802AAA84
:10FC8000AA02AA80AAAAA00AAAAAAAAAAAAAAAAA50
:10FC9000AAAAAAAAAAAAAAAAAAAAAAAAAAAAAAAAC4
:10FCA000AAAAAAAAAAAAAAAAAAAAAAAAAAAAAAAAB4
:10FCB000AAAAAA00AAAA02AAA00AAAAA02AAA80AEA
:10FCC000AAA80AAAAAAAAAAAAAAAAAAA00AAAAA8E2
:10FCD000002AAA802AAAAAAAAAAAAAA02A000AA82E
:10FCE0000A802AAAAA02AA80AAAAA00AAAAAAAAA3A
:10FCF000AAAAAAAAAAAAAAAAAAAAAAAAAAAAAAAA64
:10FD0000AAAAAAAAAAAAAAAAAAAAAAAAAAAAAAAA53
:10FD1000AAAAAAAAAAAAAA02AAAA02AAA00AAAAA3D
:10FD200002AAA802AA800AAAAAAAAAAAAAAAAAAA4F
:10FD300000AAAAA802AAAAA02AAAAAAAAAAAAAA00B
:10FD40002A020AA8AA8000000002AA80AAAAA00A81
:10FD5000AAAAAAAAAAAAAAAAAAAAAAAAAAAAAAAA03
:10FD6000AAAAAAAAAAAAAAAAAAAAAAAAAAAAAAAAF3
:10FD7000AAAAAAAAAAAAAAAAAAAAAA02AAAA02AA33
:10FD8000A00AAAAA02AAA802AA800AAAAAAAAAAA99
:10FD9000AAAAAAAA00AAAAA802AAAAA02AAAAAAAA1
:10FDA000AAAAAAA02A020AA8AA8000000002AA8081
:10FDB000AAAAA00AAAAAAAAAAAAAAAAAAAAAAAAA4D
:10FDC000AAAAAAAAAAAAAAAAAAAAAAAAAAAAAAAA93
:10FDD000AAAAAAAAAAAAAAAAAAAAAAAAAAAAAA022B
:10FDE000AAAA00AAA00AAAAA02AAAA000000AAAA6D
:10FDF000AAAAAAAAAAAAAAAA00AAAAA802AAAAA0C1
:10FE00002AAAAAAAAAAAAAA02A2A00A8AA80000006
:10FE10000002AA80AAAAA00AAAAAAAAAAAAAAAAA68
:10FE2000AAAAAAAAAAAAAAAAAAAAAAAAAAAAAAAA32
:10FE3000AAAAAAAAAAAAAAAAAAAAAAAAAAAAAAAA22
:10FE4000AAAAAA02AAAA00AAA00AAAAA02AAAA0060
:10FE50000000AAAAAAAAAAAAAAAAAAAA00AAAAA802
:10FE600002AAAAA02AAAAAAAAAAAAAA02A2A00A8DA
:10FE7000AA8000000002AA80AAAAA00AAAAAAAAA86
:10FE8000AAAAAAAAAAAAAAAAAAAAAAAAAAAAAAAAD2
:10FE9000AAAAAAAAAAAAAAAAAAAAAAAAAAAAAAAAC2
:10FEA000AAAAAAAAAAAAA000000000AAA00AAAAA0E
:10FEB00002AAA808002AAAAAAAAAAAAAAAAAAAAA18
:10FEC00000AAAAA802AAAAA02AAAAAAAAAAAAAA07A
:10FED000202A00A8AA802AAAAAAAAA80AAAAA00AB6
:10FEE000AAAAAAAAAAAAAAAAAAAAAAAAAAAAAAAA72
:10FEF000AAAAAAAAAAAAAAAAAAAAAAAAAAAAAAAA62
:10FF0000AAAAAAAAAAAAAAAAAAAAA000000000AA03
:10FF1000A002AAAA02AA800AAAAAAAAAAAAAAAAA65
:10FF2000AAAAAAAA00AAAAAA02AAAAA02AAAAAAA0D
:10FF3000AAAAAAA0202AA080AA802AAAAAAAAA803D
:10FF4000AAAA800AAAAAA80AAAAAAAAAAAAAAAAA7D
:10FF5000AAAAAAAAAAAAAAAAAAAAAAAAAAAAAAAA01
:10FF6000AAAAAAAAAAAAAAAAAAAAAAAAAAAAA000A5
:10FF7000000000AAA002AAAA02AA800AAAAAAAAA03
:10FF8000AAAAAAAAAAAAAAAA00AAAAAA02AAAAA02D
:10FF90002AAAAAAAAAAAAAA0202AA080AA802AAA33
:10FFA000AAAAAA80AAAA800AAAAAA80AAAAAAAAA47
:10FFB000AAAAAAAAAAAAAAAAAAAAAAAAAAAAAAAAA1
:10FFC000AAAAAAAAAAAAAAAAAAAAAAAAAAAAAAAA91
:10FFD000AAAAA02AAAAA800AA002AAA802AA800AFB
:10FFE000AAAAAAAAAAAAAAAAAAAAAAAA00AAAAAA1B
:10FFF00002AAAA802AAAAAAAAAAAAAA020AAA000FB
:020000040801F1
:10000000AAA02AAAAAAAAA80AAA8000AAAAAA00004
:10001000AAAAAAAAAAAAAAAAAAAAAAAAAAAAAAAA40
:10002000AAAAAAAAAAAAAAAAAAAAAAAAAAAAAAAA30
:10003000AAAAAAAAAAAAA02AAAAA800AA002AAA828
:1000400002AA800AAAAAAAAAAAAAAAAAAAAAAAAA82
:1000500000AAAAAA02AAAA802AAAAAAAAAAAAAA006
:1000600020AAA000AAA02AAAAAAAAA80AAA8000A2E
:10007000AAAAA000AAAAAAAAAAAAAAAAAAAAAAAA94
:10008000AAAAAAAAAAAAAAAAAAAAAAAAAAAAAAAAD0
:10009000AAAAAAAAAAAAAAAAAAAAA02AAAAA800A14
:1000A000AA02AA8002AA800AAAAAAAAAAAAAAAAAF4
:1000B000AAAAAAAA00AAAAAA002AA800AAAAAAAA20
:1000C000AAAAAAA000AAA000AAA000AAAAAAAA80D6
:1000D0002AA0000AAAAAA000AAAAAAAAAAAAAAAA08
:1000E000AAAAAAAAAAAAAAAAAAAAAAAAAAAAAAAA70
:1000F000AAAAAAAAAAAAAAAAAAAAAAAAAAAA802A0A
:10010000AAAAA80AAA00000202AAA80000000AAA35
:10011000AAAAAAAAAAAA000000000AAAA00000008F
:10012000AAAAAAAAAAAAAAA000AAAA00AAAA0000E1
:10013000002AAAA00000200AAAAAA000AAAAAAAA85
:10014000AAAAAAAAAAAAAAAAAAAAAAAAAAAAAAAA0F
:10015000AAAAAAAAAAAAAAAAAAAAAAAAAAAAAAAAFF
:10016000AAAA802AAAAAA80AAA00000202AAA8008B
:1001700000000AAAAAAAAAAAAAAA000000000AAA1B
:10018000A0000000AAAAAAAAAAAAAAA000AAAA0035
:10019000AAAA0000002AAAA00000200AAAAAA00079
:1001A000AAAAAAAAAAAAAAAAAAAAAAAAAAAAAAAAAF
:1001B000AAAAAAAAAAAAAAAAAAAAAAAAAAAAAAAA9F
:1001C000AAAAAAAAAAAA80AAAAAAA802AAA0002A97
:1001D00002AAA800000002AAAAAAAAAAAAAA000023
:1001E00000000AAAAA80002AAAAAAAAAAAAAAAA0C1
:1001F0000AAAAA00AAAAA80000AAAAAA000AA00AF3
:10020000AAAAA80AAAAAAAAAAAAAAAAAAAAAAAAAF0
:10021000AAAAAAAAAAAAAAAAAAAAAAAAAAAAAAAA3E
:10022000AAAAAAAAAAAAAAAAAAAA80AAAAAAA80202
:10023000AAA0002A02AAA800000002AAAAAAAAAAA2
:10024000AAAA000000000AAAAA80002AAAAAAAAAAA
:10025000AAAAAAA00AAAAA00AAAAA80000AAAAAAA8
:10026000000AA00AAAAAA80AAAAAAAAAAAAAAAAA84
:10027000AAAAAAAAAAAAAAAAAAAAAAAAAAAAAAAADE
:10028000AAAAAAAAAAAAAAAAAAAAAAAAAAAAAAAACE
:10029000AAAAAAAAAAAAAAAAAAAA800AAAAA002AB2
:1002A000AAAAAAAAAAAAAAAAAAAAAAAAAAAAAAAAAE
:1002B000AAAAAAAAAAAAAAAAAAAAAAAAAAAAAAAA9E
:1002C000AAAAAAAAAAAAAAAAAAAAAAAAAAAAAAAA8E
:1002D000AAAAAAAAAAAAAAAAAAAAAAAAAAAAAAAA7E
:1002E000AAAAAAAAAAAAAAAAAAAAAAAAAAAAAAAA6E
:1002F000AAAAAAAAAAAAAAAAAAAAAAAAAAAA800A28
:10030000AAAA002AAAAAAAAAAAAAAAAAAAAAAAAA77
:10031000AAAAAAAAAAAAAAAAAAAAAAAAAAAAAAAA3D
:10032000AAAAAAAAAAAAAAAAAAAAAAAAAAAAAAAA2D
:10033000AAAAAAAAAAAAAAAAAAAAAAAAAAAAAAAA1D
:10034000AAAAAAAAAAAAAAAAAAAAAAAAAAAAAAAA0D
:10035000AAAAAAAAAAAAAAAAAAAAAAAAAAAAAAAAFD
:10036000AAAA80AAAAAA002AAAAAAAAAAAAAAAAA41
:10037000AAAAAAAAAAAAAAAAAAAAAAAAAAAAAAAADD
:10038000AAAAAAAAAAAAAAAAAAAAAAAAAAAAAAAACD
:10039000AAAAAAAAAAAAAAAAAAAAAAAAAAAAAAAABD
:1003A000AAAAAAAAAAAAAAAAAAAAAAAAAAAAAAAAAD
:1003B000AAAAAAAAAAAAAAAAAAAAAAAAAAAAAAAA9D
:1003C000AAAAAAAAAAAA800AAAA802AAAAAAAAAA01
:1003D000AAAAAAAAAAAAAAAAAAAAAAAAAAAAAAAA7D
:1003E000AAAAAAAAAAAAAAAAAAAAAAAAAAAAAAAA6D
:1003F000AAAAAAAAAAAAAAAAAAAAAAAAAAAAAAAA5D
:10040000AAAAAAAAAAAAAAAAAAAAAAAAAAAAAAAA4C
:10041000AAAAAAAAAAAAAAAAAAAAAAAAAAAAAAAA3C
:10042000AAAAAAAAAAAAAAAAAAAA800AAAA802AAA0
:10043000AAAAAAAAAAAAAAAAAAAAAAAAAAAAAAAA1C
:10044000AAAAAAAAAAAAAAAAAAAAAAAAAAAAAAAA0C
:10045000AAAAAAAAAAAAAAAAAAAAAAAAAAAAAAAAFC
:10046000AAAAAAAAAAAAAAAAAAAAAAAAAAAAAAAAEC
:10047000AAAAAAAAAAAAAAAAAAAAAAAAAAAAAAAADC
:10048000AAAAAAAAAAAAAAAAAAAAAAAAAAAA8000A0
:1004900000000AAAAAAAAAAAAAAAAAAAAAAAAAAAB0
:1004A000AAAAAAAAAAAAAAAAAAAAAAAAAAAAAAAAAC
:1004B000AAAAAAAAAAAAAAAAAAAAAAAAAAAAAAAA9C
:1004C000AAAAAAAAAAAAAAAAAAAAAAAAAAAAAAAA8C
:1004D000AAAAAAAAAAAAAAAAAAAAAAAAAAAAAAAA7C
:1004E000AAAAAAAAAAAAAAAAAAAAAAAAAAAAAAAA6C
:1004F000AAAA800000000AAAAAAAAAAAAAAAAAAA24
:10050000AAAAAAAAAAAAAAAAAAAAAAAAAAAAAAAA4B
:10051000AAAAAAAAAAAAAAAAAAAAAAAAAAAAAAAA3B
:10052000AAAAAAAAAAAAAAAAAAAAAAAAAAAAAAAA2B
:10053000AAAAAAAAAAAAAAAAAAAAAAAAAAAAAAAA1B
:10054000AAAAAAAAAAAAAAAAAAAAAAAAAAAAAAAA0B
:10055000AAAAAAAAAAAAAAA00002AAAAAAAAAAAA57
:10056000AAAAAAAAAAAAAAAAAAAAAAAAAAAAAAAAEB
:10057000AAAAAAAAAAAAAAAAAAAAAAAAAAAAAAAADB
:10058000AAAAAAAAAAAAAAAAAAAAAAAAAAAAAAAACB
:10059000AAAAAAAAAAAAAAAAAAAAAAAAAAAAAAAABB
:100B1000AAAAAAAA001700000002001717000002E4
:100B2000000A01000001000E0E000002000000009B
:100B300000000000000000000000000000000000B5
:100B4000401700000002901717000002400A010041
:100B50000001A00E0E0000020000000000000000D6
:100B6000000000000000000000004017000000022C
:100B7000901717000002400A01000001A00E0E00AD
:100B80000002000000000000000000000000000063
:100B900000000000801700000002901717000002FC
:100BA000800A01000001500E0E000002000000004B
:100BB000000000000000000000000000000080179E
:100BC00000000002901717000002800A01000001D7
:100BD000500E0E00000200000000000000000000A7
:100BE00000000000000000000019010000010000EA
:100BF00000000000000000000000000000000000F5
:100C000000000000000000000000000000000000E4
:100C100000000000001901000001000000000000B9
:100C200000000000000000000000000000000000C4
:100C3000000000000000000000000000000080191B
:100C400001000001000000000000000000000000A2
:100C50000000000000000000000000000000000094
:100C60000000000000000000401901000001000029
:100C70000000000000000000000000000000000074
:100C80000000000000000000000000000000000064
:100C90000000001901000001000000000000000039
:100CA0000000000000000000000000000000000044
:100CB000000000000000000000000000000A00002A
:100CC0000001601414000001001400000001001372
:100CD0000A01000100000000000000000000000008
:100CE000000000000000400A000000019014140001
:100CF000000110140A000001A0130100000100000F
:100D000000000000000000000000000000000000E3
:100D1000400A0000000190141400000100140A00B1
:100D20000001990C01030401000000000000000014
:100D300000000000000000000000400A0000000168
:100D400090141400000100140A000001990B04041F
:100D50000101000000000000000000000000000091
:100D600000000000800A000000019014140000013F
:100D700020140A00000150130100000100000000CF
:100D80000000000000000000000000000000000063
:100D90000000000000000000000000101010101003
:100DA000000010000000006C484800000000000037
:100DB0000000001414287C287C28505000000010EB
:100DC00038404038487010100000002050200C704F
:100DD00008140800000000000018202054483400C7
:100DE00000000010101010000000000000000008BB
:100DF000081010101010100808000020201010100B
:100E000010101020200000107C1028280000000086
:100E100000000000101010FE101010000000000074
:100E20000000000000181030200000000000007CCE
:100E30000000000000000000000000000030300052
:100E400000000004040808101020204000000038B2
:100E50004444444444443800000000301010101052
:100E600010107C00000000384404081020447C006E
:100E70000000003844041804044438000000000C4A
:100E8000141424447E040E000000003C202038048A
:100E9000044438000000001C2040784444443800DA
:100EA0000000007C4404080808101000000000380E
:100EB0004444384444443800000000384444443C2E
:100EC00004087000000000000030300000303000E6
:100ED000000000000018180000183020000000007A
:100EE0000C10608060100C000000000000007C000E
:100EF0007C00000000000000C02018041820C00082
:100F000000000000182404081000300000003844DD
:100F1000444C54544C4044380000003010282828D9
:100F20007C44EE00000000F8444478444444F80057
:100F30000000003C4440404040443800000000F0C5
:100F4000484444444448F000000000FC44507050C1
:100F50004044FC000000007E222838282020700039
:100F60000000003C4440404E44443800000000EE85
:100F700044447C444444EE000000007C10101010F7
:100F800010107C000000003C080808484848300069
:100F9000000000EE444850704844E6000000007035
:100FA0002020202024247C00000000EE6C6C54548F
:100FB0004444EE00000000EE64645454544CEC00D1
:100FC00000000038444444444444380000000078A1
:100FD0002424243820207000000000384444444475
:100FE0004444381C000000F8444444784844E2007B
:100FF000000000344C40380404645800000000FE37
:101000009210101010103800000000EE44444444C8
:1010100044443800000000EE444428282810100002
:10102000000000EE4444545454542800000000C60C
:10103000442810102844C600000000EE4428281060
:10104000101038000000007C4408101020447C0080
:1010500000000038202020202020202038000040E0
:101060002020201010080808000000380808080890
:10107000080808083800001010284400000000008C
:1010800000000000000000000000000000FE001052
:101090000800000000000000000000000038443C90
:1010A00044443E00000000C0405864444444F800FA
:1010B00000000000003C4440404438000000000CA8
:1010C00004344C4444443E00000000000038447C9A
:1010D00040403C000000001C207C202020207C00A0
:1010E0000000000000364C4444443C04380000C07A
:1010F000405864444444EE0000000010007010109A
:1011000010107C000000001000780808080808088B
:10111000700000C0405C48705048DC0000000030A7
:101120001010101010107C000000000000E8545453
:101130005454FE000000000000D864444444EE0013
:10114000000000000038444444443800000000001F
:1011500000D8644444447840E000000000364C4429
:1011600044443C040E000000006C302020207C0031
:1011700000000000003C44380444780000000000F7
:10118000207C202020221C000000000000CC4444D1
:10119000444C36000000000000EE444428281000B3
:1011A0000000000000EE44545454280000000000E9
:1011B00000CC48303048CC000000000000EE442451
:1011C0002818101078000000007C481020447C0093
:1011D000000000081010101020101010080000105F
:1011E000101010101010101000000020101010101F
:1011F000081010102000000000000024580000001B
:101200000000C4E300000000000000001DC01D80BD
:101210003BFF3B073F777E76F870FBFEFBFE3F7798
:101220003F773E73387038703BE0000000000000EC
:1012300000000000000000000000000000000000AE
:10124000000000000000000000000000000000009E
:10125000000000000000000000000000000000008E
:10126000000000000000000000000000000000007E
:10127000000000000000000000000000000000006E
:10128000000000000000000000000000000000005E
:10129000000000000000000000000000000000004E
:1012A0000000000000000000BAC3000000000000C1
:1012B0000000300073FF700FFE1E7E3C6E38EE3073
:1012C000EFFFFC307C3038303E307E30E030C1F013
:1012D000000000000000000000000000000000000E
:1012E00000000000000000000000000000000000FE
:1012F00000000000000000000000000000000000EE
:1013000000000000000000000000000000000000DD
:1013100000000000000000000000000000000000CD
:1013200000000000000000000000000000000000BD
:1013300000000000000000000000000000000000AD
:101340000000000000000000000000000000CAF7DC
:101350000000000000000000300E300E3FEE30EEC6
:10136000FCFF76CE77FE7BFEFFFEF3DEF3CE37EE9C
:101370003E6E3C0E303E0000000000000000000009
:10138000000000000000000000000000000000005D
:10139000000000000000000000000000000000004D
:1013A000000000000000000000000000000000003D
:1013B000000000000000000000000000000000002D
:1013C000000000000000000000000000000000001D
:1013D000000000000000000000000000000000000D
:1013E00000000000000000000000000000000000FD
:1013F00000000000DDAE00000000000000000670EC
:10140000FFFF3E7038007FFFE000FFFC3B8C39CCD3
:10141000FFFF739C71DC7FFF001C01F800000000DF
:1014200000000000000000000000000000000000BC
:1014300000000000000000000000000000000000AC
:10144000000000000000000000000000000000009C
:10145000000000000000000000000000000000008C
:10146000000000000000000000000000000000007C
:10147000000000000000000000000000000000006C
:10148000000000000000000000000000000000005C
:1014900000000000000000000000C5C900000000BE
:1014A00000000000E01FFFF03E000E1FCFFBFFF822
:1014B0003FFF0FFF7FD87FDC6FCEEDFFFDF7F9C058
:1014C000000000000000000000000000000000001C
:1014D000000000000000000000000000000000000C
:1014E00000000000000000000000000000000000FC
:1014F00000000000000000000000000000000000EC
:1015000000000000000000000000000000000000DB
:1015100000000000000000000000000000000000CB
:1015200000000000000000000000000000000000BB
:1015300000000000000000000000000000000000AB
:10154000610000000000000000000000000000003A
:1015500000003E00670007800F807F80E380E78007
:10156000E7807F8000000000000000000000000015
:10157000000000000000000000000000000000006B
:10158000000000000000000000000000000000005B
:10159000000000000000000000000000000000004B
:1015A000000000000000000000000000000000003B
:1015B000000000000000000000000000000000002B
:1015C000000000000000000000000000000000001B
:1015D000000000000000000000000000000000000B
:1015E0000000000000006200000000000000000099
:1015F00070007000700070007F007B8071C071C04F
:1016000071C071C071C07B807F00000000000000CD
:1016100000000000000000000000000000000000CA
:1016200000000000000000000000000000000000BA
:1016300000000000000000000000000000000000AA
:10164000000000000000000000000000000000009A
:10165000000000000000000000000000000000008A
:10166000000000000000000000000000000000007A
:10167000000000000000000000000000000000006A
:1016800000000000000000000000000063000000F7
:1016900000000000000000000000000000003F000B
:1016A0007300F000E000E000E000F00073003F0095
:1016B000000000000000000000000000000000002A
:1016C000000000000000000000000000000000001A
:1016D000000000000000000000000000000000000A
:1016E00000000000000000000000000000000000FA
:1016F00000000000000000000000000000000000EA
:1017000000000000000000000000000000000000D9
:1017100000000000000000000000000000000000C9
:1017200000000000000000000000000000000000B9
:1017300000004100000000000000000000000E005A
:101740001F001F001F003B803B8071807FC071C065
:10175000E0E0E0E0E0E00000000000000000000049
:101760000000000000000000000000000000000079
:101770000000000000000000000000000000000069
:101780000000000000000000000000000000000059
:101790000000000000000000000000000000000049
:1017A0000000000000000000000000000000000039
:1017B0000000000000000000000000000000000029
:1017C0000000000000000000000000000000000019
:1017D0000000000000000000000000000000000009
:1017E00000000000000000000000000000000000F9
:1017F000000000000000000000000C000C000C00C5
:101800000C000C000C000C000C0000000C00000090
:101810000000000000000000000000001DC01DC00E
:101820000880088008800000000000000000000020
:10183000000000000000000000000D800D800D8001
:101840000D803FC01B003FC01B001B001B001B0086
:10185000000000000000000004001F803180318083
:1018600038001E000F000380318031803F000400EB
:101870000400000000000000000018002400240004
:1018800018C007801E003180024002400180000025
:101890000000000000000000000000000F00180021
:1018A000180018000C001D80370033001D80000058
:1018B000000000000000000000000000070007001A
:1018C0000200020002000000000000000000000012
:1018D00000000000000000000000030003000600FC
:1018E0000E000C000C000C000C000E0006000300A3
:1018F00003000000000000000000180018000C00A9
:101900000600060006000600060006000C001C008B
:1019100018000000000000000000060006003FC0A4
:101920003FC00F001F801980000000000000000071
:1019300000000000000000000000000000000400A3
:10194000040004003F8004000400040000000000C4
:101950000000000000000000000000000000000087
:1019600000000000000000000000060004000C0061
:101970000800080000000000000000000000000057
:10198000000000003F800000000000000000000098
:101990000000000000000000000000000000000047
:1019A000000000000000000000000C000C0000001F
:1019B000000000000000000000C000C001800180A5
:1019C0000300030006000C000C0018001800300093
:1019D000300000000000000000000E001B003180FD
:1019E000318031803180318031801B000E00000059
:1019F0000000000000000000000006003E0006009D
:101A00000600060006000600060006003FC00000B3
:101A1000000000000000000000000F00198031806D
:101A20003180030006000C00180030003F800000E9
:101A3000000000000000000000003F006180018005
:101A400003001F0003800180018061803F000000CF
:101A500000000000000000000000070007000F0069
:101A60000B001B00130033003F8003000F800000B9
:101A7000000000000000000000001F801800180097
:101A800018001F0011800180018021801F000000CC
:101A90000000000000000000000007801C0018008B
:101AA0003000370039803180318019800F0000000C
:101AB000000000000000000000007F004300030061
:101AC00006000600060006000C000C000C000000DA
:101AD000000000000000000000001F003180318085
:101AE00031801F0031803180318031801F00000043
:101AF000000000000000000000001E0033003180E4
:101B0000318033801D800180030007003C0000000D
:101B100000000000000000000000000000000000C5
:101B20000C000C000000000000000C000C00000085
:101B300000000000000000000000000000000000A5
:101B4000030003000000000000000600040008007D
:101B500008000000000000000000000000C00300BA
:101B600004001800600018000400030000C000001A
:101B70000000000000000000000000000000000065
:101B800000007FC000007FC00000000000000000D7
:101B900000000000000000000000000060001800CD
:101BA0000400030000C003000400180060000000EF
:101BB0000000000000000000000000001F00318055
:101BC0003180018007000C000C0000000C000000B8
:101BD000000000000000000000000E0011002100C5
:101BE00021002700290029002700200011000E00F5
:101BF0000000000000000000000000003F000F0097
:101C00000900198019801F8030C030C079E00000C1
:101C10000000000000000000000000007F00318094
:101C2000318031803F003180318031807F00000081
:101C30000000000000000000000000001F4030C055
:101C40006040600060006000604030801F00000065
:101C50000000000000000000000000007F00318054
:101C600030C030C030C030C030C031807F00000094
:101C70000000000000000000000000007F803080B5
:101C8000308032003E003200308030807F800000A3
:101C90000000000000000000000000007FC0304095
:101CA000304032003E003200300030007C00000046
:101CB0000000000000000000000000001E803180D5
:101CC00060806000600067C0618031801F0000009C
:101CD0000000000000000000000000007BC0318018
:101CE000318031803F803180318031807BC0000085
:101CF0000000000000000000000000003FC00600DF
:101D00000600060006000600060006003FC00000B0
:101D10000000000000000000000000001FC00300E1
:101D20000300030003006300630063003E00000043
:101D30000000000000000000000000007BC03180B7
:101D4000330036003C003E003300318079C0000093
:101D50000000000000000000000000007E001800ED
:101D60001800180018001840184018407FC00000E4
:101D7000000000000000000000000000E0E060C083
:101D800071C07BC06AC06EC064C060C0FBE0000070
:101D900000000000000000000000000073C031805F
:101DA00039803D80358037803380318079800000F4
:101DB0000000000000000000000000001F00318053
:101DC00060C060C060C060C060C031801F000000A3
:101DD0000000000000000000000000007F003180D3
:101DE0003180318031803F00300030007E000000C3
:101DF0000000000000000000000000001F00318013
:101E000060C060C060C060C060C031801F000CC096
:101E10001F80000000000000000000007F003180F3
:101E2000318031803E003300318031807CE0000021
:101E30000000000000000000000000001F80318052
:101E4000318038001F000380318031803F00000066
:101E50000000000000000000000000007F804C80B7
:101E60004C804C800C000C000C000C003F0000006B
:101E70000000000000000000000000007BC0318076
:101E80003180318031803180318031801F0000000D
:101E90000000000000000000000000007BC0318056
:101EA00031801B001B001B000A000E000E0000000A
:101EB000000000000000000000000000FBE060C027
:101EC00064C06EC06EC02A803B803B8031800000C1
:101ED0000000000000000000000000007BC0318016
:101EE0001B000E000E000E001B0031807BC00000A6
:101EF00000000000000000000000000079E030C099
:101F000019800F0006000600060006001F80000072
:101F10000000000000000000000000003F80218061
:101F20002300060004000C00188030803F80000071
:101F3000000000000000000000000780060006000E
:101F40000600060006000600060006000600060061
:101F5000078000000000000030003000180018006A
:101F60000C000C000600030003000180018000C08B
:101F700000C000000000000000001E000600060077
:101F80000600060006000600060006000600060021
:101F90001E0000000000000004000A000A001100FA
:101FA00020802080000000000000000000000000F1
:101FB0000000000000000000000000000000000021
:101FC0000000000000000000000000000000000011
:101FD000000000000000FFE0080004000200000014
:101FE00000000000000000000000000000000000F1
:101FF00000000000000000000000000000000000E1
:102000001F00018001801F80318033801DC00000CF
:1020100000000000000000000000700030003000F0
:102020003700398030C030C030C0398077000000C0
:1020300000000000000000000000000000000000A0
:102040001E80318060806000608031801F00000051
:1020500000000000000000000000038001800180FB
:102060001D80338061806180618033801DC00000ED
:102070000000000000000000000000000000000060
:102080001F00318060C07FC0600030C01F80000032
:102090000000000000000000000007E00C000C0041
:1020A0003F800C000C000C000C000C003F80000076
:1020B0000000000000000000000000000000000020
:1020C0001DC0338061806180618033801D8001800C
:1020D00001801F0000000000000070003000300090
:1020E0003700398031803180318031807BC0000001
:1020F00000000000000000000000060006000000D4
:102100001E00060006000600060006003FC0000094
:1021100000000000000000000000060006000000B3
:102120003F0003000300030003000300030003005B
:1021300003003E000000000000007000300030008E
:10214000378036003C003C003600330077C000008A
:10215000000000000000000000001E000600060055
:102160000600060006000600060006003FC000004C
:10217000000000000000000000000000000000005F
:102180007F8036C036C036C036C036C076E000002C
:10219000000000000000000000000000000000003F
:1021A0007700398031803180318031807BC0000000
:1021B000000000000000000000000000000000001F
:1021C0001F00318060C060C060C031801F0000000F
:1021D00000000000000000000000000000000000FF
:1021E0007700398030C030C030C0398037003000CF
:1021F00030007C0000000000000000000000000033
:102200001DC0338061806180618033801D800180CA
:10221000018007C000000000000000000000000076
:102220007B801CC018001800180018007F000000F8
:10223000000000000000000000000000000000009E
:102240001F8031803C001F00038031803F00000070
:102250000000000000000000000018001800180036
:102260007F00180018001800180018800F000000E8
:10227000000000000000000000000000000000005E
:102280007380318031803180318033801DC0000007
:10229000000000000000000000000000000000003E
:1022A0007BC0318031801B001B000E000E0000003F
:1022B000000000000000000000000000000000001E
:1022C000F1E060C064C06EC03B803B8031800000A4
:1022D00000000000000000000000000000000000FE
:1022E0007BC01B000E000E000E001B007BC0000018
:1022F00000000000000000000000000000000000DE
:1023000079E030C0198019800B000F00060006002C
:102310000C003E0000000000000000000000000073
:102320003F80218003000E00180030803F800000B5
:102330000000000000000000000006000C000C007F
:102340000C000C000C0018000C000C000C000C0021
:102350000600000000000000000006000600060065
:10236000060006000600060006000600060006003D
:10237000060000000000000000000C00060006003F
:102380000600060006000300060006000600060020
:102390000C00000000000000000000000000000031
:1023A000000018002480030000000000000000006E
:1023B0000000000000000000C4E300000000000076
:1023C000000000000000000000000000000000000D
:1023D00000000000000001C1C00001E3E00003E3D1
:1023E000C00003C7800003C7FFFF078FFFFF078FF1
:1023F000000F0F1E001E0F3C1E1E1F3C1E3E1F180E
:102400001E3C3F001E1C7F001E007F079E70FF07C2
:102410009EF0EF0F9E786F0F1E780F0F1E3C0F1E61
:102420001E3C0F1E1E1E0F3C1E1E0F3C1E1F0F7C4F
:102430001E0F0F781E0E0F001E000F001E000F0053
:102440003C000F07FC000F07F80000000000000030
:102450000000000000000000000000000000BAC3FF
:10246000000000000000000000000000000000006C
:1024700000000000000000000F0000000F0000003E
:102480000F07FFFE0F07FFFE0F00003E1E0000FCBF
:10249000FFF801F0FFF803E01E7807C01E780F80F8
:1024A0003C780F003C780F003C780F003C780F0020
:1024B0003C7FFFFF78FFFFFF78F00F0078F00F0000
:1024C0003DE00F001FE00F000FE00F0007C00F00FE
:1024D00007E00F0007F00F000FF80F001E7C0F0041
:1024E0003C380F0078000F00F003FF006001FE0091
:1024F00000000000000000000000000000000000DC
:1025000000000000CEA2000000000000000000005B
:1025100000000000000000000000000000000307B1
:1025200001E0078701E0070701C00FF779C01EF738
:102530007BC01EF77B803CF77BFF78F77BFFF8F7CB
:102540007F9EF7FFFF9E67FFFF9E07007F9C0F00A7
:102550000F9C1E001F9C1E7FFFBC3E7FF3FC3E00B5
:1025600003FC7E0001F8FE0001F8FE7FE1F8DE7F4B
:10257000E1F81E78E0F01E78EEF01E78FFF01E788D
:10258000FDF81E79FBFC1EF1F7BC1EF0EF9E1FE06C
:102590000F0F1EC01E0F1E000C07000000000000E1
:1025A00000000000000000000000C8ED0000000076
:1025B000000000000000000000000000000000001B
:1025C00003C0780007807800078078000780F0005B
:1025D0000F00F000FFFFFFFFFFFFFFFF1E03C01F04
:1025E0001E03C01E1FE78F3E3DE78F3C3DEF0F7C73
:1025F0003DE70F7879E00F0079E00E007FFE0E00D6
:102600007FFE1F0001E01F0001E01F0001E01F80AE
:1026100001E01F8001E03F8001FF3FC00FFF7BC052
:10262000FFF079E0F9E0F1F001E1F0F001E3E0F82A
:1026300001E7C07C01FF803F01FF001F01EC000E9D
:10264000000000000000000000000000000000008A
:10265000D1C50000000000000000000000000000E4
:1026600000000000000000000000000077000000F3
:10267000FF007FFCF7807FFDE3C001C1E3C001C321
:10268000C1803DC7FFFF39C7FFFF39CF838079DFA6
:10269000838079FF838079DF838071C383807FFFAC
:1026A000FFFE7FFFFFFE03C3838007C3838007C352
:1026B00083800FC383800FC383801FC3FFFE1DC3AE
:1026C000FFFE3DC3838079C38380F1C38380F1C360
:1026D000838061C3838001C3FFFF03C3FFFF1FC368
:1026E00080001F8380000000000000000000000048
:1026F000000000000000BADA000000000000000046
:1027000000000000000000000000000000000000C9
:1027100000000000000000001FFFFFFC1FFFFFFC87
:102720001E03C03C1EC3C73C1FE3C7BC1EF3CF3C07
:102730001EFBDF3C1E7BDE3C1E33DC3C1E03C03C2C
:102740001FFFFFFC1FFFFFFC1E03C03C0003C00077
:102750000003C0003FFFFFFC3FFFFFFC0003C00081
:102760000003C0000003C000FFFFFFFFFFFFFFFFEB
:10277000000000001C3870703E78F8F83C7C787CD3
:102780007C3C3C3EF83E3C1FF01C180E0000000054
:10279000000000000000000000000000B4CB0000BA
:1027A0000000000000000000000000000000000029
:1027B0000000000000000000000000783C000078ED
:1027C0003C0000783C0000783C0000783C00007839
:1027D0003C0C3C783C1E3C783C3F3C783CF83C7FD1
:1027E000FDF03C7FFFE03C783F803C783E003C7849
:1027F0003C003C783C003C783C003C783C003C7819
:102800003C003C783C003C783C0E3C783C0F3C78EB
:102810003C0F3C79FC0F3C7FFC0F3FFF3C0F3FF02F
:102820003E1EFF001FFEF0000FFC00000000000035
:102830000000000000000000000000000000000098
:102840000000D7D6000000000000000000000000DB
:10285000000000000000000000038000000780006E
:102860000003C0000003E0000001E0007FFFFFFE66
:102870007FFFFFFE7800001E7800001E7800001E1B
:102880007800001E7BFFFFDE03FFFFC000000FC0CB
:1028900000003F0000007E000001F8000001E000A1
:1028A0000001E000FFFFFFFFFFFFFFFF0001E0006E
:1028B0000001E0000001E0000001E0000001E00094
:1028C0000001E0000003E0000003C00000FFC000C2
:1028D00000FF800000000000000000000000000079
:1028E0000000000000000000CCE500000000000037
:1028F00000000000000000000000000000000000D8
:1029000000000000000003C03C0003C03C0003C006
:102910003C0007803C0007803C0007803C000FFF24
:10292000FFFF0FFFFFFF1F01FE001F01FF003F0120
:10293000FF003F03FF007F03FF807F07BF80FF078B
:10294000BFC0EF0F3DC0CF0F3DE00F1E3DE00F1E9B
:102950003CF00F3C3C780F7C3C7C0FF83C3E0FF782
:10296000FFDF0FE7FFCF0FC03C060F003C000F005A
:102970003C000F003C000F003C000F003C0000003A
:102980000000000000000000000000000000CFC2B6
:102990000000000000000000000000000000000037
:1029A0000000000000000000000000000000000027
:1029B000FFFFFFFFFFFFFFFF000F8000000F800001
:1029C000000F8000000F8000000F8000000F8000CB
:1029D000000FE000000FF800000FFC00000FBF0028
:1029E000000F9F80000F87E0000F83F0000F80F83A
:1029F000000F807C000F8038000F8000000F8000E7
:102A0000000F8000000F8000000F8000000F80008A
:102A1000000F8000000F8000000F8000000F80007A
:102A200000000000000000000000000000000000A6
:102A300000000000B6D4000000000000000000000C
:102A40000000000000000000000000000000000086
:102A500000000000007800000078000000787FFC93
:102A600000787FFC0078003C0078003FFFFF303F9B
:102A7000FFFF783C00783C3800783E7800781E787C
:102A8000C0780F79E0780FF0F07807F0F87803F06D
:102A9000787801E03C7803F03E7803F0187807F886
:102AA000007807FC00780F3E00781F1E00783E1F5C
:102AB00000787C0E00F8F80000F0F0003FF06000B5
:102AC0003FE00000000000000000000000000000E7
:102AD00000000000000000000000D3A6000000007D
:102AE00000000000000000000000000000000000E6
:102AF0000001C0000003E0000001E0000001F00060
:102B00000000F0001FFFFFFF1FFFFFFF1E0000007F
:102B10001E0000001E01E0781E01E0781EE1E07852
:102B20001FF1F0F81EF0F0F01EF0F0F01EF8F0F0DB
:102B30001E78F1F01E78F9E01E7879E01E7C7BE0CB
:102B40001E3C7BC01E3C7BC01E3C7BC03C3E0780C5
:102B50003C1C07803C0007803C000F0078000F0001
:102B60007BFFFFFFF3FFFFFFF000000060000000AD
:102B70000000000000000000000000000000000055
:102B8000B5C40000000000000000000000000000CC
:102B90000000000000000000000003803C0007C0AF
:102BA0003E0007803C0007807C000F0078007FFE1D
:102BB0007FFE7FFEFFFE781EF01E781FE01E781F4E
:102BC000E01E781FC01E781FC01E781FF01E781EE2
:102BD000F81E781E7C1E7FFE3C1E7FFE1E1E781E89
:102BE0001F1E781E0F9E781E079E781E071E781ED9
:102BF000001E781E001E781E003E781E003C781EC7
:102C0000003C7FFE003C7FFE007C781E3FF8781E73
:102C10003FF0000000000000000000000000000085
:102C2000000000000000B5E300000000000000000C
:102C30000000000000000000000000000000000094
:102C40000003C0000003C0000003C0000003C00078
:102C50000003FFFF0003FFFF0003C0000003C000EC
:102C60000003C0000003C0000FFFFFF80FFFFFF8D4
:102C70000F0000780F0000780F0000780F00007838
:102C80000F0000780F0000780FFFFFF80FFFFFF82C
:102C90000F000078000000000C3838301E7C787877
:102CA0003E3C78783C3C3C3C7C3E3C3EF81E3C1E26
:102CB000F01E1E1F701E1C0E000000000000000011
:102CC000000000000000000000000000D5F300003C
:102CD00000000000000000000000000000000000F4
:102CE00000000000000000003C00000078007FF0C1
:102CF00078007FF0780079FFFFFF79FFFFFF79E12F
:102D0000E00079E1E0007BC1EF807BC3CF807BC333
:102D1000CF807F87CF807F878F807F878F807BCF9B
:102D20000F807BCFFFFE79EFFFFE79E00F8078E028
:102D30000F8078F00F8078F00F8078F00F8078FFA8
:102D4000FFFF79FFFFFF7FE00F807FC00F807800DB
:102D50000F8078000F8078000F8078000F80780057
:102D60000F800000000000000000000000000000D4
:102D70000000CEAA000000000000000000000000DB
:102D80000000000000000000000000000000000043
:102D9000000780000E0780001F0780000F8780005B
:102DA00007C7800001E7800000C78000000780009F
:102DB0007FFFFFFC7FFFFFFC0007803C000F803C93
:102DC000000F003C000F003C000F603C001FF03C77
:102DD000001E783C003E3C3C003C3E3C007C1F3CDE
:102DE00000780F3C00F8063C01F0003C03E0007C5A
:102DF00007C0007C0F8000781F0000F83E00FFF045
:102E00007C00FFE03800000000000000000000002F
:102E10000000000000000000CAF7000000000000F1
:102E200000000000000000000000000000000000A2
:102E30000000000000000F0000380F0000380F00F5
:102E400000380F3FF8380F3FF8380F007838FFE0B0
:102E50007FFFFFE07FFF0F0070380F18F0381F3C36
:102E6000F0381F1CFE381FDEFE383FEFEF383FFF03
:102E7000EF383FF7E7B87F67C7B87F03C3B8FF07EE
:102E8000E038EF07E038EF0FF038CF1FF0380F1EB3
:102E900078380F3C7C380F783C380FF838380F60A2
:102EA00000780F000FF80F0007F00F00000000007F
:102EB0000000000000000000000000000000DDAE87
:102EC0000000000000000000000000000000000002
:102ED0000000000000000000003C1E00003C1E003E
:102EE000003C1E00FFFFFFFFFFFFFFFF003C1E0036
:102EF00007BC1E00078000000FFFFFFC0FFFFFFC58
:102F00001E0000003C0000003C0000007FFFFFF0BE
:102F1000F7FFFFF0378380F00787C0F00783F0F0FA
:102F20000700E0F0FFFFFFFFFFFFFFFF0F0F00E0D4
:102F30000F0F81E00E03E1E01E01C1E01FFFFFFE65
:102F40001FFFFFFE000001E0000003C00000FFC003
:102F50000000FF80000000000000000000000000F2
:102F600000000000C5C900000000000000000000D3
:102F70000000000000000000000000000000000051
:102F800000003800003E7C003FFE3F3FFFF01FBFC7
:102F9000E00007BC0000033C0000003C003C003C9B
:102FA0000FFE703DFFF8F83DFF007C3DE7803F3DA0
:102FB000E7801F3DE78E0E3DE79F003DE7FE0039AD
:102FC000E7F80039E3F01C39E3C01E79E3C01E794D
:102FD000E1E01E79E1E03C79E0F03C79E0F83CF199
:102FE000E07C3CF1E37C7DF1EF3F79E1FE1F7BE18A
:102FF000F80E7BC3E0007981C000000000000000F3
:10300000000000000000000000004100000000007F
:1030100000000000000000000000000000000000B0
:10302000000000000000000000000000007C000024
:1030300000FC000000FE000000FE000001FF000098
:1030400001FF000001EF000003EF800003CF8000CC
:1030500007C7800007C7C0000787C0000F83E000D4
:103060000F83E0000F01E0001FFFF0001FFFF000E2
:103070003FFFF8003E00F8003C00F8007C007C00B8
:103080007C007C0078003C00F8003E00F8003E0028
:103090000000000000000000000000000000000030
:1030A0000000000000000000000000000000000020
:1030B00061000000000000000000000000000000AF
:1030C0000000000000000000000000000000000000
:1030D00000000000000000000000000000000000F0
:1030E000000000000000000000000000000007F8E1
:1030F00000001FFE00003FFE00003E3F0000381FA2
:103100000000000F0000000F000003FF00001FFF81
:1031100000003F8F00007C0F00007C0F0000781F34
:1031200000007C1F00007E7F00007FFF00003FFF4B
:1031300000000FCF000000000000000000000000B1
:10314000000000000000000000000000000000007F
:10315000000000000000620000000000000000000D
:10316000000000000000000000000000000000005F
:10317000000000003C0000003C0000003C0000009B
:103180003C0000003C0000003C0000003C0000004F
:103190003C0000003CFE00003DFF80003FFFC000FF
:1031A0003F8FC0003F07E0003E03E0003E03E00029
:1031B0003C01E0003C01E0003C01E0003C03E00099
:1031C0003E03E0003E03E0003F07C0003F8FC00029
:1031D0003FFF80003FFF00003CFC000000000000BB
:1031E00000000000000000000000000000000000DF
:1031F000000000000000000000000000630000006C
:1032000000000000000000000000000000000000BE
:1032100000000000000000000000000000000000AE
:10322000000000000000000000000000000000009E
:103230000000000000000000000001FC000007FE8C
:1032400000001FFE00003F8600003E0000007C00E2
:1032500000007C0000007C00000078000000780086
:1032600000007C0000007C0000007C0000003E00AC
:1032700000003F8600001FFE00000FFE000003FC60
:10328000000000000000000000000000000000003E
:10329000000000000000000000000000000000002E
:1032A0000000CEA2000000000000000000000000AE
:1032B000000000000000000000000000030701E023
:1032C000078701E0070701C00FF779C01EF77BC031
:1032D0001EF77B803CF77BFF78F77BFFF8F77F9E3C
:1032E000F7FFFF9E67FFFF9E07007F9C0F000F9C6C
:1032F0001E001F9C1E7FFFBC3E7FF3FC3E0003FCB4
:103300007E0001F8FE0001F8FE7FE1F8DE7FE1F8C3
:103310001E78E0F01E78EEF01E78FFF01E78FDF8C3
:103320001E79FBFC1EF1F7BC1EF0EF9E1FE00F0F95
:103330001EC01E0F1E000C07000000000000000051
:103340000000000000000000D1A900000000000003
:10335000000000000000000000000000000000006D
:10336000000000000000000000001FFFFFF81FFF2A
:10337000FFF80003C0000003C0007FFFFFFE7FFFD7
:10338000FFFE7803C01E7803C01E7FFFFFFE7FFF95
:10339000FFFE0003C0000003C00007FFFFE007FFBF
:1033A000FFE00003C000000000001FFFFFF81FFF48
:1033B000FFF800000078000000781FFFFFF81FFFF3
:1033C000FFF80000007800000078000000783FFF60
:1033D000FFF83FFFFFF80000007800000000000049
:1033E0000000000000000000000000000000B5E741
:1033F00000000000000000000000000000000000CD
:1034000000000000000000000007800000078000AE
:1034100000078000000780007FFFFFF87FFFFFF8B4
:10342000780780F8780780F8780780F8780780F8C0
:10343000780780F8780780F87FFFFFF87FFFFFF8B4
:10344000780780F8780780F8780780F8780780F8A0
:10345000780780F8780780F87FFFFFF87FFFFFF894
:103460007807800E7807800F0007800F0007800F15
:103470000007801F0007801E0003FFFE0001FFFC05
:10348000000000000000000000000000000000003C
:1034900000000000D7D30000000000000000000082
:1034A000000000000000000000000000000000001C
:1034B0000000000000001FFFFFF81FFFFFF80000E2
:1034C00001F8000007E000000FC000001F800000AE
:1034D0003E000000FC000001F8000003E0000003D3
:1034E000E0000003E000FFFFFFFFFFFFFFFF00031E
:1034F000E0000003E0000003E0000003E000000340
:10350000E0000003E0000003E0000003E00000032F
:10351000E0000003E0000003E0000003C00001FF42
:10352000C00000FF8000000000000000000000005C
:1035300000000000000000000000000053757070E3
:103540006F727420666F72207061727469616C2092
:10355000726566726573682C206275742074686584
:10356000207265667265736820656666656374209F
:103570006973206E6F7420676F6F642C206275749E
:10358000206974206973206E6F74207265636F6D9B
:103590006D656E6465640D0A000000004465627527
:1035A000673A206D6972726F722073686F756C6410
:1035B000206265204D4952524F525F4E4F4E452C6E
:1035C000204D4952524F525F484F52495A4F4E5424
:1035D000414C2C2020202020202020204D495252D8
:1035E0004F525F564552544943414C206F72204D13
:1035F0004952524F525F4F524947494E0D0A0000FF
:1036000044656275673A205061696E745F44726107
:1036100077537472696E675F454E20496E7075749A
:10362000206578636565647320746865206E6F72C9
:103630006D616C20646973706C61792072616E6772
:10364000650D0A0044656275673A205061696E74C1
:103650005F44726177436972636C6520496E70756F
:1036600074206578636565647320746865206E6F87
:10367000726D616C20646973706C61792072616E27
:1036800067650D0A00000000A83601080000002050
:1036900044000000A0580008EC3601084400002057
:1036A000B4A00000B05800080100000010000000A5
:1036B0000000000000A24A048E0D010807000C0063
:1036C0000212010809000B0010001500D8170108AC
:1036D0000B001000B82301081B001800200029006F
:0C36E000000000000000000000000000DE
:0400000508000131BD
:00000001FF
